:020000040800F2
:10000000D0C60020DD01000821610008A1590008C8
:100010001D6100088D0C0008E1CA00080000000006
:100020000000000000000000000000004501000882
:10003000F11500080000000089010008F1C2000865
:10004000F7010008F7010008F7010008F7010008B0
:10005000F7010008F7010008F7010008F7010008A0
:10006000F7010008F7010008F7010008F701000890
:10007000F70100087515000885150008951500089A
:10008000A5150008F7010008F7010008F7010008AE
:10009000F7010008F7010008F7010008F701000860
:1000A000F70100088DC30008F7010008F7010008F8
:1000B000F7010008F70100089DC30008F7010008D8
:1000C000F7010008F7010008F7010008F701000830
:1000D000F701000855C90008D9C900085DCA000821
:1000E000F7010008F7010008F7010008F701000810
:1000F000ADC30008F7010008F7010008F701000888
:10010000F7010008F7010008F7010008F7010008EF
:10011000F7010008F7010008F7010008F7010008DF
:10012000F7010008F7010008F7010008B5150008FD
:10013000DFF80CD000F0FAF9004800479DD3000822
:10014000D0C60020224B19680868B0E8F00F80F391
:100150000988BFF36F8F4FF0000080F311884EF0D5
:100160000D0E70470000000006480068006880F32C
:10017000088862B661B6BFF34F8FBFF36F8F00DFA1
:1001800000BF00BF08ED00E0EFF30980BFF36F8F01
:100190000F4B1A6820E9F00F106008B54FF05000BF
:1001A00080F31188BFF34F8FBFF36F8F0EF04AFFBC
:1001B0004FF0000080F31188BDE808401968086816
:1001C000B0E8F00F80F30988BFF36F8F704700BF6E
:1001D000F0090020EFF305807047000006488047D3
:1001E00006480047FEE7FEE7FEE7FEE7FEE7FEE71C
:1001F000FEE7FEE7FEE7FEE78BC3000831010008DB
:10020000202A04DB203A21FA02F00021704721FA6B
:1002100002F3D040C2F120029140084319467047D2
:10022000A0F16101192900D82038704740EA010384
:100230009B0703D009E008C9121F08C0042AFAD29C
:1002400003E011F8013B00F8013B521EF9D2704760
:10025000D2B201E000F8012B491EFBD27047002208
:10026000F6E710B513460A4604461946FFF7F0FFB5
:10027000204610BDF0B480EA0102D40F4200B2EB78
:10028000410F02D20246084611464A0042D0C30D31
:10029000DDB2C1F3C752AD1A202D35DAC1F3160114
:1002A00041F4000204B15242C5F1200602FA06F1FF
:1002B0002A411044B3EBD05F23D0C4B1012DA0EB91
:1002C000C35009DCF0BC4FF0004202EAC352DBB27B
:1002D00000F5000000F0FBB8400000F1807000EB7A
:1002E000C350A0F1807040EAD170490009E049088C
:1002F00041EAC071A0EBC35000F50000400800EBDC
:10030000C350F0BC00F0DAB86142012202EB4101B7
:10031000001BF6E7F0BC704781F00041AAE780F0CF
:100320000040A7E780EA010210B502F00043400058
:1003300022D04A001FD0010E01EB1261C0F356001B
:10034000C2F3560240F4000042F40002A0FB022077
:1003500000047F39140400D0401C50EA124001D43C
:100360004000491EC2B20C0604EBD010401C4008ED
:10037000802A02D003E0002010BD20F001000029F7
:1003800000DA0020184310BD30B480EA010202F008
:10039000004530F0004221F0004013D090B1C30D71
:1003A000D40DC2F31601C0F31600E41A41F40001A3
:1003B00040F400027D34914201D3641C00E0490006
:1003C000002C02DA30BC002070474FF400000023FC
:1003D000914201D3891A034340084FEA4101F7D102
:1003E00051B1914202D14FF0004105E002D24FF0ED
:1003F000010101E06FF0010103EBC450284430BC5F
:1004000000F05CB8C10F80EAE0700844CA07962388
:10041000002100F05CB896230022114600F057B886
:1004200000F0004220F00040C10DC0F3160040F47F
:1004300000007F2901DA00207047962903DCC1F112
:100440009601C84001E096398840002AF4D0404225
:10045000704720F00040C10DC0F3160040F40000CA
:100460007F2901DA00207047962903DCC1F196014B
:10047000C84070479639884070470000002801DB6B
:10048000C0F10040002901DBC1F100418142704709
:1004900030B50B46014600202022012409E021FA54
:1004A00002F59D4205D303FA02F5491B04FA02F551
:1004B0002844151EA2F10102F1DC30BD0029A8BFBD
:1004C0007047401C490008BF20F00100704710B47D
:1004D000B0FA80FC00FA0CF050EA010404BF10BC32
:1004E000704749B1CCF1200421FA04F411FA0CF15F
:1004F00018BF012121430843A3EB0C01CB1D4FEA98
:1005000000614FEA102042BF002010BC704700EB92
:10051000C35010440029A4BF10BC7047401C4900C0
:1005200008BF20F0010010BC70470000064C074DCA
:1005300006E0E06840F0010394E8070098471034B3
:10054000AC42F6D3FFF7F8FD9C100108BC1001087F
:1005500070B58D1810F8014B14F0030201D110F89A
:10056000012B231106D110F8013B03E010F8016BB9
:1005700001F8016B521EF9D1ABB110F8012B04F058
:100580000C048A1A0C2C03D0A2EB84129B1C08E0EA
:1005900010F8014BA2EB0422F8E712F8014B01F826
:1005A000014B5B1EF9D5A942D4D3002070BD0000D9
:1005B00010B5144A302909D1A1F13003C3EBC304AB
:1005C00004EB031302EB830358801AE0312901DAAC
:1005D0003F2909DCA1F13003C3EBC30404EB03138F
:1005E00002EB8303D8800CE0412901DA4F2908DCB3
:1005F000A1F13003C3EBC30404EB031302EB830349
:10060000988010BD802E00202DE9F0410446174649
:10061000DFF854C14FF6FF70844201D0814203D10C
:100620004FF6FF70BDE8F0810026002244F25060D2
:10063000844201DA264602E048F6A040061B40F656
:10064000E440864200DD064648480088301AB0F58E
:10065000FA7F04DD4548008800F5FA7609E0434852
:100660000088801BB0F5FA7F03DD40480088A0F5C4
:10067000FA76DFF8F880A8F80060344644F250605B
:10068000814201DA0A4602E048F6A040421A012FF0
:100690001EDD374830F81300101AB0F5FA7F05DD7B
:1006A000334830F8130000F5FA720BE0304830F8A8
:1006B0001300801AB0F5FA7F04DD2D4830F81300DE
:1006C000A0F5FA72DFF8A88028F81320114632E06E
:1006D000284830F81300101AB0F5FA7F05DD2548D8
:1006E00030F8130000F5FA720BE0224830F81300DE
:1006F000801AB0F5FA7F04DD1E4830F81300A0F52B
:10070000FA72DFF8708028F813201146A14209DB45
:10071000091BC3EBC30808EB03180CEB8808A8F807
:10072000061008E0641AC3EBC30808EB03180CEBCF
:100730008808A8F806403FB90D1B0F48854209DA22
:1007400048F6A040054405E00D1948F6A040854252
:1007500000DB2D1A46F67810854202DDA5F50C4522
:10076000A03D28465EE70000802E002052030020B6
:10077000602E0020402E0020B0B9FFFF2DE9F0418F
:1007800006468846324C00253F2E03DDA6F1400088
:10079000054402E0A6F130000544C5EBC50000EBBE
:1007A000051004EB80001C30C5EBC50101EB051101
:1007B00034F8211000EBC107264878603860608863
:1007C0004FF6FF7188422AD0A088401C70B108F013
:1007D00040039A1CC5EBC50303EB051304EB83032D
:1007E000998860882B46FFF70FFF3860A6F130002C
:1007F000C0EBC00101EB001004EB8000C088401C7E
:1008000068B108F02002C5EBC50303EB051304EB48
:100810008303D98860882B46FFF7F6FE7860C5EB26
:10082000C50000EB051034F82000401C80B2C5EB79
:10083000C50101EB051124F82100082806DB002082
:10084000C5EBC50101EB051124F82100BDE8F081DD
:10085000802E0020786FFFFF70B55E4C5E4B01204C
:1008600000225E4900BFAEE00025C0EBC00606EBEB
:10087000860601EB46067587C0EBC00606EB8606CA
:1008800001EB4606F587C0EBC00606EB860601EBDA
:100890004606F586C0EBC00606EB860601EB46066B
:1008A0007586012259E09D89012D4ED11D89EDBB30
:1008B000C0EBC00505EB001504EB85051C3505EB09
:1008C000C2056D68464EB5420EDCC0EBC00505EBB7
:1008D000850501EB45052D8F6D1CC0EBC00606EBB1
:1008E000860601EB46063587C0EBC00505EB001513
:1008F00004EB85051C3505EBC2056D686D42B1F84A
:100900004260B5420DDCC0EBC00505EB001504EB01
:1009100085051C3505EBC2056D68B1F84260B5422E
:1009200011DDC0EBC00505EB850500E00DE001EB36
:1009300045052D8E6D1CC0EBC00606EB860601EB4F
:100940004606358608E000BF06E09D89012D03D1EB
:100950001D89012D00D100BF521C022AA3DBC0EB70
:10096000C00505EB850501EB4505AD8FC0EBC00665
:1009700006EB860601EB4606B6F84060B54208DB9A
:100980000025C0EBC00606EB860601EB4606F587A0
:1009900018E0C0EBC00505EB850501EB45056D8E44
:1009A000C0EBC00606EB860601EB4606B6F84060D3
:1009B000B54207DB0025C0EBC00606EB860601EB5F
:1009C0004606F586401C074D2D78A8427FF74CAFB0
:1009D00070BD0000802E0020A03800204034002090
:1009E000786FFFFF5003002070B58AB005461D4E9A
:1009F0001D4C28216846FFF732FCA17F607F41EA49
:100A00000020ADF80000207D062804D101221749FE
:100A1000684600F0B9FE01221449684600F09EFEC7
:100A2000BDF8000000122874BDF800006874BDF81D
:100A300000004FF6FF71884203D0BDF80000A6F811
:100A40006C00297C607F814209D1697CA07F814252
:100A500005D1207D062802D101200AB070BD0020FA
:100A6000FBE70000A0380020E239002050F0070822
:100A700010B50146304B314A588800285AD1187DAC
:100A800006280FD101205880987F2D4C2070062019
:100A900060700020A0700120E0700020207108200C
:100AA000607145E0B2F87A00C0B1472088747F20B9
:100AB000C874FF20087500204875472088757F207E
:100AC000C875FF20087600204876472088767F206A
:100AD000C876FF2008770020487729E0B2F90000A7
:100AE000000E8874B2F90000000CC8741088000A67
:100AF000087510784875B2F92800000E8875B2F9AB
:100B00002800000CC875108D000A087692F828009D
:100B10004876B2F95000000E8876B2F95000000C09
:100B2000C876B2F85000000A087792F8500048776B
:100B3000002010BD0120FCE7E2390020184300200E
:100B40005639002030B58BB0244D282101A8FFF77D
:100B500086FB00240122224901A800F0FFFDBDF818
:100B600004004FF6FF71884203D0BDF8040068808E
:100B700001E00120688008221A4901A800F0EEFD7A
:100B8000002415E001A830F814004FF6FF718842E8
:100B900007D001A830F8141005F1440020F8141013
:100BA00004E0012105F1440020F81410601CC4B2D7
:100BB0002888A042E6DC00240AE005F1440030F871
:100BC000140009490988084407490880601CC4B218
:100BD0002888A042F1DC0BB030BD0000A038002016
:100BE00024F0070860E00708DC0900202DE9F04147
:100BF0000746244D00240026287D062840D10120E8
:100C00006880AA7F2046611CCCB21F490A54062284
:100C10002046611CCCB21C490A5412222046611C99
:100C2000CCB219490A54EA7F2046611CCCB216495D
:100C30000A542020425D2046611CCCB212490A545D
:100C4000EA7F2046611CCCB20F490A542020425D45
:100C50002046611CCCB20C490A5408210A4804F011
:100C6000A1FE064632122046611CCCB206490A5447
:100C70002046611CCCB204490E540120BDE8F0812D
:100C80000020FBE7E23900209C39002000BFFEE78E
:100C900070B58AB00646204D28216846FFF7DFFA76
:100CA000002400BF08E004F1100005F10D01085C0C
:100CB0002DF81400601CC4B2287EA042F3DC287D0D
:100CC000062804D1F27A1549684600F05DFDF27AF3
:100CD0001249684600F042FD00F038F9002415E0A2
:100CE0003DF8142004F1100005F10D01085C82426A
:100CF00005D0287D062802D100200AB070BD1DF85D
:100D0000141004F110003154601CC4B2287EA042BB
:100D1000E6DC0120F1E70000E239002000F00708DE
:100D20002DE9F04F85B080460E4615461F4600203F
:100D30000490774C012F06D0022F18D0032F2AD011
:100D4000042F54D13CE04046E16CFFF7E5FA7149CD
:100D5000086008460168E1624FF03F410068FFF714
:100D60008DFB03D24FF03F406A49086040E04046A7
:100D7000616FFFF7D1FA674908600846016861654D
:100D80004FF03F410068FFF779FB03D24FF03F403F
:100D9000604908602CE09C2001594046FFF7BCFAEE
:100DA0005C49086008460168E1674FF03F41006810
:100DB000FFF764FB03D24FF03F405649086017E04D
:100DC000C42001594046FFF7A7FA52490860084677
:100DD0000168A42001514FF03F414E480068FFF7E1
:100DE0004DFB03D24FF03F404A49086000E000BF8E
:100DF00000BF494947480068FFF794FA8146FFF76A
:100E000028FB4649088000204549088039E04448CD
:100E1000008835F810004149098888422CDA40489A
:100E20000088401C35F810003C490988884223DBC3
:100E30003B49098836F81100FFF7EDFA3949086097
:100E400037490988491C36F81100FFF7E4FA36499A
:100E500008603349098835F81100FFF7DCFA334997
:100E600008602F490988491C35F81100FFF7D3FAAB
:100E70002F49086000BF08E029480088401C284925
:100E8000088027480088C828C1DD00BF23480088A3
:100E900000280ADC00202349086023490860234910
:100EA0000860234908601D4908801E4801681E48E3
:100EB0000068FFF731FA03901C4801681C4800687D
:100EC000FFF72AFA029015480088FFF7A4FA00906D
:100ED000164801680098FFF71FFA01900299FFF782
:100EE00053FA83460399FFF71DFA82460D480168BD
:100EF0005046FFF7BFF98146FFF7ABFA0D4908806E
:100F000008460088FFF787FA05B0BDE8F08F0000BB
:100F100098400020B409002000007A44C409002051
:100F2000C0090020C8090020CC090020D0090020F9
:100F3000D4090020C20900207047704770477047ED
:100F40007047704770477047704770472DE9F04F02
:100F5000A1B0FD4CFD4FDFF8F883DFF8F893DFF820
:100F6000F8A3FE4EDFF8F8B3802101A8FFF777F968
:100F700000250622FB4901A800F0F0FBBDF80400A3
:100F80004FF6FF71884216D1C822F749F74800F0A2
:100F9000FBFBC822F649F74800F0F6FBC822F649E9
:100FA000F64800F0F1FBC822F549F64800F0ECFBEA
:100FB0000320208002E0BDF804002080BDF8060078
:100FC0004FF6FF7188420ED1002508E0012104F19F
:100FD000340020F815100120A081681C85B22088FB
:100FE000A842F3DC0FE000250AE0BDF8061004F18A
:100FF000340020F81510BDF80600A081681C85B2E9
:101000002088A842F1DCBDF808004FF6FF71884245
:1010100002D10020608102E0BDF808006081BDF8C7
:101020000A004FF6FF7188420ED1002508E001202A
:101030002082022104F1140020F81510681C85B2EA
:101040002088A842F3DC0EE0002509E00120208280
:10105000BDF80A1004F1140020F81510681C85B2C0
:101060002088A842F2DCBDF80C004FF6FF718842E0
:101070000ED1002508E001206082012104F1240046
:1010800020F81510681C85B22088A842F3DC0EE019
:10109000002509E001206082BDF80C1004F1240055
:1010A00020F81510681C85B22088A842F2DC0122C5
:1010B000AC49203101A800F051FBBDF804004FF607
:1010C000FF71884202D10120208102E0BDF80400B6
:1010D00020810122A349283101A800F03FFBBDF87F
:1010E00004004FF6FF71884202D10020A08002E088
:1010F000BDF80400A08001229A49303101A800F017
:101100002DFBBDF804004FF6FF71884202D101208B
:10111000E08002E0BDF80400E08008229A4901A8BE
:1011200000F01CFB002517E001A830F8150000288E
:101130000BDD01A830F81500082806DA01A830F800
:10114000151004F1340020F81510012104F13400C9
:1011500020F81510681C85B2082DE5DB08228A49A5
:10116000203901A800F0FAFA002517E001A830F8AC
:10117000150000280BDD01A830F81500082806DA54
:1011800001A830F8151004F1140020F81510022100
:1011900004F1140020F81510681C85B2082DE5DB59
:1011A00008227949203101A800F0D8FA002517E07B
:1011B00001A830F8150000280BDD01A830F8150053
:1011C000082806DA01A830F8151004F1240020F8E8
:1011D0001510012104F1240020F81510681C85B2B7
:1011E000082DE5DB01225F49383101A800F0B6FA8D
:1011F000BDF804004FF6FF71884203D10120A4F826
:101200006E0003E0BDF80400A4F86E000122554909
:10121000403101A800F0A2FABDF804004FF6FF71BA
:10122000884203D10220A4F8640003E0BDF8040062
:10123000A4F864000822554901A800F08FFABDF80F
:1012400004004FF6FF71884220D1002050490870F9
:1012500048708870C8700021F1644D49087048706A
:101260008870C8700021716749490870487088709B
:10127000C87000219C2081510020454908704870A9
:101280008870C8700021C42081514DE0BDF8040071
:1012900000123F49C870BDF804008870BDF8060010
:1012A00000124870BDF80600087008460168F16435
:1012B00000BFBDF8080000123549C870BDF808002D
:1012C0008870BDF80A0000124870BDF80A00087066
:1012D00008460168716700BFBDF80C0000122C4978
:1012E000C870BDF80C008870BDF80E000012487080
:1012F000BDF80E000870084601689C20815100BFAF
:10130000BDF8100000122249C870BDF810008870A6
:10131000BDF8120000124870BDF8120008700846AF
:101320000168C420815100BF01220E49483101A843
:1013300000F014FABDF804004FF6FF71884229D17D
:101340000120A4F8660029E0A038002040340020E5
:10135000363A00209C4B0020184300209840002083
:101360009C43002000F0070800D00708600300201D
:1013700000D40708F004002000D8070880060020E9
:1013800000DC07081008002020E0070800C007085C
:10139000F4020020BDF80400A4F8660001222549EB
:1013A00001A800F0DBF9BDF804004FF6FF71884298
:1013B00003D10120A4F86C0003E0BDF80400A4F8F8
:1013C0006C0001221B49143101A800F0C7F9BDF8D7
:1013D00004004FF6FF7188420DD10521A7F8861051
:1013E000A8F82C110520A9F84E00AAF87C0030843A
:1013F000ABF87C001BE0BDF80410A7F88610BDF820
:101400000410A7F8CC10BDF80400A8F86000BDF8DF
:101410000400A9F84E0000BFBDF80400AAF87C0043
:10142000BDF804003084BDF80400ABF87C0021B0A6
:10143000BDE8F08F50F007082DE9F0478146484E8F
:10144000484C002500274FF00308F08800284DD1B4
:10145000102D47DA4FF48041434802F00FFE04F1AB
:10146000520121F815004FF400413F4802F006FEFA
:1014700004F1A40121F8150040213C4802F0FEFDD2
:1014800004F1F60121F815008021384802F0F6FD3C
:1014900004F5A47121F815004FF48071334802F06F
:1014A000EDFD04F5CD7121F815004FF400712F48C2
:1014B00002F0E4FD04F5F67121F815004FF4807197
:1014C0002B4802F0DBFD04F23E2121F815004FF419
:1014D0000061274802F0D2FD04F5247121F81500BF
:1014E000681CC5B2102D39DB002537E0F0880128D3
:1014F00034D181031C4802F0C1FDA4F852004FF41E
:101500000041194802F0BAFDA4F8A4004021174890
:1015100002F0B4FDA4F8F6008021144802F0AEFDFC
:10152000A4F848014FF48071104802F0A7FDA4F818
:101530009A014FF400710D4802F0A0FDA4F8EC01EF
:101540004FF480710A4802F099FDA4F83E024FF46E
:101550000061074802F092FDA4F89002BDE8F08710
:10156000A03800209C4B0020000C014000100140DE
:101570000008014010B5024802F09AF810BD0000C2
:101580001C0D002010B5024802F092F810BD0000BA
:10159000940C002010B5024802F08AF810BD00003B
:1015A000500C002010B5024802F082F810BD000077
:1015B000D80C002010B5024802F07AF810BD0000E7
:1015C0007C0A002030B590F840500124AC40C56B37
:1015D0006C60046863604468102C04D10468A260E5
:1015E0000468E16003E00468A1600468E26030BD63
:1015F000704772B600BFFEE70021074AD161074974
:10160000096941F00401054A11611146096941F077
:101610004001116170470000880F00200020024047
:101620000021074AD1610749096941F00201054AD1
:10163000116111464861096941F04001116170472B
:10164000880F0020002002400022054BDA61054A85
:10165000126942F00102034B1A61018070470000D9
:10166000880F00200020024000201E49C96801F0B8
:10167000100139B11C49C96941F002011A4AD1610E
:1016800040F010001749C96801F0040139B116494A
:10169000C96941F00101144AD16140F004001149C7
:1016A000C96901F0010169B10F49C96941F004013B
:1016B0000D4AD16100BF0B49C96921F00101094AF6
:1016C000D16100BF00BF40F20111884206D1054937
:1016D000C96921F00101034AD16101E00149C860F3
:1016E00000BF704700200240880F002070B50446FC
:1016F00002F0DCFC054609E0601C38B124B102F0C0
:10170000D5FC401BA04201D9032070BD1248C0681F
:1017100000F001000028EFD10F48C06800F0200061
:1017200020B100BF20200C49C86000BF0A48C06833
:1017300000F0100048B90848C06900F0010020B965
:101740000548C06800F0040018B1FFF78DFF0120C4
:10175000DBE70020D9E7000000200240F0B5034697
:101760001C4600250026084607E010F8015B10F82B
:10177000016B45EA062724F8027B171EA2F1010C33
:101780001FFA8CF2F1D1F0BD2DE9F04786B080460A
:101790000E4691464FF0000A00270025C6F30A0ABC
:1017A000A6EB0A0700200590019000BF03970120D7
:1017B0000490820239461648FFF7D0FF002507E063
:1017C00038F8150005EB5A01114A22F811006D1C7A
:1017D0004D45F5D302F09AFA00BF05A901A802F021
:1017E000DBF900BF00240BE0094830F814C007EB18
:1017F000440162460023012002F030FA601C84B2EA
:10180000B4F5806FF0DB02F01FFA06B0BDE8F08798
:10181000001000202DE9F04794B00446DFF870A4D2
:101820004FF00008002700260025A94628210AA815
:10183000FEF715FD28216846FEF711FD00BF24E0E4
:10184000152000EB48010AF10D00415C142000EB6B
:1018500048020AF10D00805C41EA00200AA921F843
:101860001800152000EB48010AF10D00415C14201E
:1018700000EB48020AF10D00805C41EA00202DF8DF
:10188000180008F1010000F0FF08B8F1140FD7DBD1
:101890009AF81400062841F0D683FE4890F810907C
:1018A0004FF6FF7000EA0929FA48407C40EA09092E
:1018B000F848877CB9F1010F7ED1012F47D114225E
:1018C000F5490AA8FFF760FF1422F3490AA8FFF7B9
:1018D00045FF00250AE03DF815000AA931F815106A
:1018E000884201D1701CC6B2681C85B2142DF2DB8F
:1018F000142E1DD1E9480088401CE8490880E548BD
:10190000007C2074E348407C6074E248807CA074D2
:10191000E048C07CE074084600880A2802D1022012
:10192000207501E001202075012014B0BDE8F0878A
:10193000D848007C2074D748407C6074D548807CAF
:10194000A074D448C07CE07400202075EDE7022F1D
:1019500049D11422D04928310AA8FFF715FF1422D3
:10196000CD4928310AA8FFF7F9FE00250AE03DF825
:1019700015000AA931F81510884201D1701CC6B2B1
:10198000681C85B2142DF2DB142E1DD1C3480088CB
:10199000401CC2490880BF48007C2074BD48407C80
:1019A0006074BC48807CA074BA48C07CE07408466F
:1019B0000088282804D100E070E20220207501E0B0
:1019C000012020750120B0E7B248007C2074B148A6
:1019D000407C6074AF48807CA074AE48C07CE074EA
:1019E00000202075A1E7032F47D11422AA495031C6
:1019F0000AA8FFF7C9FE1422A74950310AA8FFF729
:101A0000ADFE00250AE03DF815000AA931F81510D1
:101A1000884201D1701CC6B2681C85B2142DF2DB5D
:101A2000142E1BD19D480088401C9C490880994871
:101A3000007C20749748407C60749648807CA07439
:101A40009448C07CE074084600880A2802D102202D
:101A5000207501E001202075012066E78D48007C9B
:101A600020748C48407C60748A48807CA0748948CB
:101A7000C07CE0740020207557E7042F47D1142262
:101A8000854978310AA8FFF77FFE14228249783110
:101A90000AA8FFF763FE00250AE03DF815000AA931
:101AA00031F81510884201D1701CC6B2681C85B28D
:101AB000142DF2DB142E1BD178480088401C774986
:101AC00008807448007C20747248407C60747148BF
:101AD000807CA0746F48C07CE074084600880A28A7
:101AE00002D10220207501E00120207501201CE7B1
:101AF0006848007C20746748407C60746548807C3E
:101B0000A0746448C07CE074002020750DE7052FA8
:101B100047D114226049A0310AA8FFF735FE1422EC
:101B20005D49A0310AA8FFF719FE00250AE03DF83B
:101B300015000AA931F81510884201D1701CC6B2EF
:101B4000681C85B2142DF2DB142E1BD1534800887B
:101B5000401C524908804F48007C20744D48407C0E
:101B600060744C48807CA0744A48C07CE07408468D
:101B700000880A2802D10220207501E0012020758A
:101B80000120D2E64348007C20744248407C6074C7
:101B90004048807CA0743F48C07CE07400202075E1
:101BA000C3E6062F47D114223B49C8310AA8FFF7E4
:101BB000EBFD14223849C8310AA8FFF7CFFD0025F4
:101BC0000AE03DF815000AA931F81510884201D144
:101BD000701CC6B2681C85B2142DF2DB142E1BD10A
:101BE0002E480088401C2D4908802A48007C20741B
:101BF0002848407C60742748807CA0742548C07CBD
:101C0000E074084600880A2802D10220207501E00D
:101C100001202075012088E61E48007C20741D48A4
:101C2000407C60741B48807CA0741A48C07CE074BF
:101C30000020207579E6072F50D114221649F03183
:101C40000AA8FFF7A1FD14221349F0310AA8FFF7F3
:101C500085FD00250AE03DF815000AA931F81510A8
:101C6000884201D1701CC6B2681C85B2142DF2DB0B
:101C7000142E24D109480088401C084908800548D2
:101C8000007C20740348407C60740248807C07E03C
:101C9000E23900200029002000D00708D8090020E0
:101CA000A074FE48C07CE074084600880A2802D16F
:101CB0000220207501E001202075012035E6F7485B
:101CC000007C2074F548407C6074F448807CA074EB
:101CD000F248C07CE0740020207526E6082F45D12C
:101CE0001422EF490AA8FFF74FFD1422EC490AA875
:101CF000FFF734FD00250AE03DF815000AA931F888
:101D00001510884201D1701CC6B2681C85B2142D12
:101D1000F2DB142E1BD1E3480088401CE149088007
:101D2000DE48007C2074DD48407C6074DB48807CA9
:101D3000A074DA48C07CE074084600880A2802D102
:101D40000220207501E0012020750120EDE5D34837
:101D5000007C2074D148407C6074D048807CA074A2
:101D6000CE48C07CE07400202075DEE5092F47D105
:101D70001422CB4928310AA8FFF706FD1422C849CE
:101D800028310AA8FFF7EAFC00250AE03DF8150013
:101D90000AA931F81510884201D1701CC6B2681C1E
:101DA00085B2142DF2DB142E1BD1BE480088401CD6
:101DB000BC490880B948007C2074B848407C6074F5
:101DC000B648807CA074B548C07CE07408460088A2
:101DD0000A2802D10220207501E00120207501208F
:101DE000A3E5AE48007C2074AC48407C6074AB48EE
:101DF000807CA074A948C07CE0740020207594E524
:101E00000A2F41F020811422A54950310AA8FFF77A
:101E1000BBFC1422A24950310AA8FFF79FFC002501
:101E20000AE03DF815000AA931F81510884201D1E1
:101E3000701CC6B2681C85B2142DF2DB142E1ED1A4
:101E400098480088401C974908809448007C20747A
:101E50009248407C60749148807CA0748F48C07C1C
:101E6000E074084600880A2802D10220207501E0AB
:101E70000120207500208B490880012055E5874806
:101E8000007C20748548407C60748448807CA07409
:101E90008248C07CE0740020207546E5B9F1020F4D
:101EA0007ED1012F45D114227F490AA8FFF76CFC8F
:101EB00014227D490AA8FFF751FC00250AE03DF8ED
:101EC00015000AA931F81510884201D1701CC6B25C
:101ED000681C85B2142DF2DB142E1BD171480088CA
:101EE000401C704908806D48007C20746B48407C21
:101EF00060746A48807CA0746848C07CE0740846BE
:101F000000880A2802D10220207501E001202075F6
:101F100001200AE56148007C20746048407C6074C0
:101F20005E48807CA0745D48C07CE0740020207511
:101F3000FBE4022F48D114225B4928310AA8FFF79D
:101F400023FC1422584928310AA8FFF707FC002572
:101F50000AE03DF815000AA931F81510884201D1B0
:101F6000701CC6B2681C85B2142DF2DB142E1CD175
:101F70004C480088401C4B4908804848007C20742D
:101F80004648407C60744548807CA0744348C07CCF
:101F9000E07408460088282803D10220207502E05A
:101FA0006CE2012020750120BFE43C48007C2074D5
:101FB0003A48407C60743948807CA0743748C07CC3
:101FC000E07400202075B0E4032F47D11422364975
:101FD00050310AA8FFF7D8FB1422334950310AA820
:101FE000FFF7BCFB00250AE03DF815000AA931F80F
:101FF0001510884201D1701CC6B2681C85B2142D20
:10200000F2DB142E1BD127480088401C254908808C
:102010002248007C20742148407C60741F48807CEA
:10202000A0741E48C07CE074084600880A2802D1CB
:102030000220207501E001202075012075E4174879
:10204000007C20741548407C60741448807CA07427
:102050001248C07CE0740020207566E4042F50D143
:102060001422114978310AA8FFF78EFB14220E4979
:1020700078310AA8FFF772FB00250AE03DF8150049
:102080000AA931F81510884201D1701CC6B2681C2B
:1020900085B2142DF2DB142E24D107E00029002094
:1020A00018D10708D809002000D40708FC48008888
:1020B000401CFB490880FB48007C2074F948407CA8
:1020C0006074F848807CA074F648C07CE0740846D0
:1020D00000880A2802D10220207501E00120207525
:1020E000012022E4EF48007C2074EE48407C6074BC
:1020F000EC48807CA074EB48C07CE0740020207524
:1021000013E4052F45D11422E7490AA8FFF73CFB49
:102110001422E5490AA8FFF721FB00250AE03DF853
:1021200015000AA931F81510884201D1701CC6B2F9
:10213000681C85B2142DF2DB142E1BD1D848008800
:10214000401CD7490880D748007C2074D548407C83
:102150006074D448807CA074D248C07CE074084687
:1021600000880A2802D10220207501E00120207594
:10217000012028E4CB48007C2074CA48407C60746D
:10218000C848807CA074C748C07CE07400202075DB
:1021900019E4062F47D11422C34928310AA8FFF7B2
:1021A000F3FA1422C04928310AA8FFF7D7FA00250C
:1021B0000AE03DF815000AA931F81510884201D14E
:1021C000701CC6B2681C85B2142DF2DB142E1BD114
:1021D000B3480088401CB2490880B248007C207493
:1021E000B048407C6074AF48807CA074AD48C07C2F
:1021F000E074084600880A2802D10220207501E018
:1022000001202075012028E4A648007C2074A54800
:10221000407C6074A348807CA074A248C07CE074B9
:102220000020207519E4072F47D114229E49503110
:102230000AA8FFF7A9FA14229B4950310AA8FFF710
:102240008DFA00250AE03DF815000AA931F81510AD
:10225000884201D1701CC6B2681C85B2142DF2DB15
:10226000142E1BD18E480088401C8D4908808D4853
:10227000007C20748B48407C60748A48807CA07409
:102280008848C07CE074084600880A2802D10220F1
:10229000207501E001202075012028E48148007CA0
:1022A00020748048407C60747E48807CA0747D48A7
:1022B000C07CE0740020207519E4082F47D1142257
:1022C000794978310AA8FFF75FFA14227649783104
:1022D0000AA8FFF743FA00250AE03DF815000AA90D
:1022E00031F81510884201D1701CC6B2681C85B245
:1022F000142DF2DB142E1BD169480088401C68495C
:1023000008806848007C20746648407C607465489A
:10231000807CA0746348C07CE074084600880A286A
:1023200002D10220207501E001202075012028E45F
:102330005C48007C20745B48407C60745948807C19
:10234000A0745848C07CE0740020207519E4092F5F
:1023500047D114225449A0310AA8FFF715FA1422D4
:102360005149A0310AA8FFF7F9F900250AE03DF824
:1023700015000AA931F81510884201D1701CC6B2A7
:10238000681C85B2142DF2DB142E1BD14448008842
:10239000401C434908804348007C20744148407CED
:1023A00060744048807CA0743E48C07CE07408465D
:1023B00000880A2802D10220207501E00120207542
:1023C000012028E43748007C20743648407C607443
:1023D0003448807CA0743348C07CE07400202075B1
:1023E00019E40A2F5BD114222F49C8310AA8FFF73C
:1023F000CBF914222C49C8310AA8FFF7AFF9002500
:102400000AE03DF815000AA931F81510884201D1FB
:10241000701CC6B2681C85B2142DF2DB142E1ED1BE
:102420001F480088401C1E4908801E48007C2074FC
:102430001C48407C60741B48807CA0741948C07C98
:10244000E074084600880A2802D10220207501E0C5
:102450000120207500201249088001202EE4114837
:10246000007C20740F48407C60740E48807CA0740F
:102470000C48C07CE074002020751FE4B9F1030F04
:102480007ED1012F4ED1142208490AA8FFF77CF90A
:10249000142206490AA8FFF761F9002513E015E3A5
:1024A000D809002000290020A0D4070800D8070878
:1024B0003DF815000AA931F81510884201D1701CA9
:1024C000C6B2681C85B2142DF2DB142E1BD1FB485A
:1024D0000088401CF9490880F948007C2074F848BD
:1024E000407C6074F648807CA074F548C07CE07441
:1024F000084600880A2802D10220207501E0012048
:102500002075012022E4EE48007C2074EC48407CD9
:102510006074EB48807CA074E948C07CE0740020C3
:10252000207513E4022F47D11422E6490AA8FFF7C9
:102530002BF91422E3490AA8FFF710F900250AE055
:102540003DF815000AA931F81510884201D1701C18
:10255000C6B2681C85B2142DF2DB142E1DD1D748EB
:102560000088401CD5490880D548007C2074D44898
:10257000407C6074D248807CA074D148C07C00E06C
:1025800071E2E07408460088282802D102202075F4
:1025900001E001202075012022E4C948007C20745C
:1025A000C748407C6074C648807CA074C448C07C26
:1025B000E0740020207513E4032F47D11422C14991
:1025C00028310AA8FFF7E0F81422BE4928310AA8EA
:1025D000FFF7C4F800250AE03DF815000AA931F814
:1025E0001510884201D1701CC6B2681C85B2142D2A
:1025F000F2DB142E1BD1B1480088401CAF49088083
:10260000AF48007C2074AE48407C6074AC48807C4D
:10261000A074AB48C07CE074084600880A2802D148
:102620000220207501E001202075012026E4A44845
:10263000007C2074A248407C6074A148807CA07417
:102640009F48C07CE0740020207517E4042F47D118
:1026500014229C4950310AA8FFF796F81422994990
:1026600050310AA8FFF77AF800250AE03DF8150076
:102670000AA931F81510884201D1701CC6B2681C35
:1026800085B2142DF2DB142E1BD18C480088401C1F
:102690008A4908808A48007C20748948407C60749C
:1026A0008748807CA0748648C07CE0740846008817
:1026B0000A2802D10220207501E0012020750120A6
:1026C00027E47F48007C20747D48407C60747C480F
:1026D000807CA0747A48C07CE0740020207518E4E7
:1026E000052F47D11422774978310AA8FFF74CF813
:1026F0001422744978310AA8FFF730F800250AE05F
:102700003DF815000AA931F81510884201D1701C56
:10271000C6B2681C85B2142DF2DB142E1BD167489B
:102720000088401C654908806548007C2074644826
:10273000407C60746248807CA0746148C07CE07416
:10274000084600880A2802D10220207501E00120F5
:102750002075012028E45A48007C20745848407CA9
:1027600060745748807CA0745548C07CE074002099
:10277000207519E4062F47D114225249A0310AA826
:10278000FFF702F814224F49A0310AA8FEF7E6FF2E
:1027900000250AE03DF815000AA931F81510884215
:1027A00001D1701CC6B2681C85B2142DF2DB142E48
:1027B0001BD142480088401C404908804048007CAA
:1027C00020743F48407C60743D48807CA0743C4845
:1027D000C07CE074084600880A2802D102202075D7
:1027E00001E001202075012028E43548007C207498
:1027F0003348407C60743248807CA0743048C07C90
:10280000E0740020207519E4072F47D114222D49C8
:10281000C8310AA8FEF7B8FF14222A49C8310AA80D
:10282000FEF79CFF00250AE03DF815000AA931F8E3
:102830001510884201D1701CC6B2681C85B2142DD7
:10284000F2DB142E1BD11D480088401C1B49088058
:102850001B48007C20741A48407C60741848807CB7
:10286000A0741748C07CE074084600880A2802D18A
:102870000220207501E001202075012031E410487C
:10288000007C20740E48407C60740D48807CA074ED
:102890000B48C07CE0740020207522E4082F4DD145
:1028A00014220849F0310AA8FEF76EFF14220549E8
:1028B000F0310AA8FEF752FF002510E0D8090020E9
:1028C0000029002028D807083DF815000AA931F88A
:1028D0001510884201D1701CC6B2681C85B2142D37
:1028E000F2DB142E1BD1FD480088401CFB490880F8
:1028F000FB48007C2074FA48407C6074F848807C77
:10290000A074F748C07CE074084600880A2802D109
:102910000220207501E001202075012029E4F04803
:10292000007C2074EE48407C6074ED48807CA0748C
:10293000EB48C07CE074002020751AE4092F45D1D3
:102940001422E8490AA8FEF71FFF1422E5490AA845
:10295000FEF704FF00250AE03DF815000AA931F84A
:102960001510884201D1701CC6B2681C85B2142DA6
:10297000F2DB142E1BD1D9480088401CD7490880AF
:10298000D748007C2074D648407C6074D448807C52
:10299000A074D348C07CE074084600880A2802D19D
:1029A0000220207501E00120207501202BE4CC4895
:1029B000007C2074CA48407C6074C948807CA07444
:1029C000C748C07CE074002020751CE40A2F7DD12C
:1029D0001422C44928310AA8FEF7D6FE1422C149A0
:1029E00028310AA8FEF7BAFE00250AE03DF81500D6
:1029F0000AA931F81510884201D1701CC6B2681CB2
:102A000085B2142DF2DB142E1ED1B4480088401C70
:102A1000B2490880B248007C2074B148407C6074A0
:102A2000AF48807CA074AE48C07CE0740846008843
:102A30000A2802D10220207501E001202075002023
:102A4000A6490880012028E4A548007C2074A448F9
:102A5000407C6074A248807CA074A148C07CE07473
:102A60000020207519E4B9F1040FB0D1012F47D12E
:102A700014229D490AA8FEF787FE14229A490AA843
:102A8000FEF76CFE00250AE03DF815000AA931F8B2
:102A90001510884201D1701CC6B2681C85B2142D75
:102AA000F2DB142E1DD18D480088401C8B49088014
:102AB0008B48007C20748A48407C60748848807C05
:102AC000A0748748C07CE074084600E0BBE2008840
:102AD0000A2802D10220207501E001202075012082
:102AE00025E47F48007C20747D48407C60747C48ED
:102AF000807CA0747A48C07CE0740020207516E4C5
:102B0000022F47D11422784928310AA8FEF73CFE4B
:102B10001422754928310AA8FEF720FE00250AE094
:102B20003DF815000AA931F81510884201D1701C32
:102B3000C6B2681C85B2142DF2DB142E1BD1674877
:102B40000088401C654908806548007C2074644802
:102B5000407C60746248807CA0746148C07CE074F2
:102B600008460088282802D10220207501E00120B3
:102B70002075012025E45A48007C20745848407C88
:102B800060745748807CA0745548C07CE074002075
:102B9000207516E4032F47D11422534950310AA857
:102BA000FEF7F2FD1422504950310AA8FEF7D6FD77
:102BB00000250AE03DF815000AA931F815108842F1
:102BC00001D1701CC6B2681C85B2142DF2DB142E24
:102BD0001BD142480088401C404908804048007C86
:102BE00020743F48407C60743D48807CA0743C4821
:102BF000C07CE074084600880A2802D102202075B3
:102C000001E001202075012028E43548007C207473
:102C10003348407C60743248807CA0743048C07C6B
:102C2000E0740020207519E4042F47D114222E49A6
:102C300078310AA8FEF7A8FD14222B4978310AA89A
:102C4000FEF78CFD00250AE03DF815000AA931F8D1
:102C50001510884201D1701CC6B2681C85B2142DB3
:102C6000F2DB142E1BD11D480088401C1B49088034
:102C70001B48007C20741A48407C60741848807C93
:102C8000A0741748C07CE074084600880A2802D166
:102C90000220207501E001202075012032E4104857
:102CA000007C20740E48407C60740D48807CA074C9
:102CB0000B48C07CE0740020207523E4052F4FD121
:102CC00014220949A0310AA8FEF75EFD1422064924
:102CD000A0310AA8FEF742FD002512E0D809002025
:102CE0000029002040D9070800DC07083DF815003E
:102CF0000AA931F81510884201D1701CC6B2681CAF
:102D000085B2142DF2DB142E1BD1D0480088401C54
:102D1000CE490880CE48007C2074CD48407C607449
:102D2000CB48807CA074CA48C07CE0740846008808
:102D30000A2802D10220207501E00120207501201F
:102D40002AE4C348007C2074C148407C6074C048B9
:102D5000807CA074BE48C07CE074002020751BE419
:102D6000062F45D11422BB490AA8FEF70DFD1422F7
:102D7000B8490AA8FEF7F2FC00250AE03DF8150064
:102D80000AA931F81510884201D1701CC6B2681C1E
:102D900085B2142DF2DB142E1BD1AC480088401CE8
:102DA000AA490880AA48007C2074A948407C607425
:102DB000A748807CA074A648C07CE07408460088C0
:102DC0000A2802D10220207501E00120207501208F
:102DD0002CE49F48007C20749D48407C60749C4893
:102DE000807CA0749A48C07CE074002020751DE4AB
:102DF000072F47D11422974928310AA8FEF7C4FCAF
:102E00001422944928310AA8FEF7A8FC00250AE0FC
:102E10003DF815000AA931F81510884201D1701C3F
:102E2000C6B2681C85B2142DF2DB142E1BD1874864
:102E30000088401C854908808548007C20748448AF
:102E4000407C60748248807CA0748148C07CE074BF
:102E5000084600880A2802D10220207501E00120DE
:102E6000207501202CE47A48007C20747848407C4E
:102E700060747748807CA0747548C07CE074002042
:102E800020751DE4082F47D11422724950310AA839
:102E9000FEF77AFC14226F4950310AA8FEF75EFC57
:102EA00000250AE03DF815000AA931F815108842FE
:102EB00001D1701CC6B2681C85B2142DF2DB142E31
:102EC0001BD162480088401C604908806048007C33
:102ED00020745F48407C60745D48807CA0745C48CE
:102EE000C07CE074084600880A2802D102202075C0
:102EF00001E00120207501202CE45548007C20745D
:102F00005348407C60745248807CA0745048C07C18
:102F1000E074002020751DE4092F47D114224D498B
:102F200078310AA8FEF730FC14224A4978310AA801
:102F3000FEF714FC00250AE03DF815000AA931F857
:102F40001510884201D1701CC6B2681C85B2142DC0
:102F5000F2DB142E1BD13D480088401C3B49088001
:102F60003B48007C20743A48407C60743848807C40
:102F7000A0743748C07CE074084600880A2802D153
:102F80000220207501E00120207501202CE430484A
:102F9000007C20742E48407C60742D48807CA07496
:102FA0002B48C07CE074002020751DE40A2F4AD114
:102FB00014222849A0310AA8FEF7E6FB142225496D
:102FC000A0310AA8FEF7CAFB00250AE03DF815006B
:102FD0000AA931F81510884201D1701CC6B2681CCC
:102FE00085B2142DF2DB142E1ED118480088401C27
:102FF000164908801648007C20741548407C60748F
:103000001348807CA0741248C07CE0740846008895
:103010000A2802D10220207501E00120207500203D
:103020000A490880012029E40948007C20740848E6
:10303000407C60740648807CA0740548C07CE074C5
:10304000002020751AE4002018E40000D8090020B0
:1030500000290020C8DC070870B500250026264C92
:103060002648407905022548807905432348407861
:10307000032805D021484078062801D001260CE01D
:103080001E488078022801D0012606E005211B4851
:1030900002F088FCA84200D0012618484078032896
:1030A00021D1012115480078803800EB800202EB25
:1030B000801004EB4000A0F888101048C178007818
:1030C000803800EB800202EB801024F810100B48CF
:1030D00001790078803800EB800202EB801004EB6D
:1030E0004000018507E005484078062803D10348E1
:1030F000C0780249C87070BDBC500020002B002071
:103100000146064A01EBC10000EB411032F8100005
:1031100008B9012070470020FCE700009C4B00200C
:1031200070B50025234C2448407905022248807957
:10313000054321484078032807D01F4840780628D7
:1031400003D001201D49088010E01B488078022828
:1031500003D001201949088008E00521164802F033
:1031600021FCA84202D00120144908800121124804
:103170000078803800EB0012C2EBC01004EB400076
:10318000A0F8B6100C48C1780078803800EB001227
:10319000C2EBC01004EB400081820748017900783F
:1031A000803800EB0012C2EBC01004EB40008187B6
:1031B00070BD00005C590020002B0020DE090020BB
:1031C00010B5002150480123504A1278203A02EBF2
:1031D000C20404EB421200EB4202A2F850304C4A07
:1031E0001278212A03D04A4A1278222A3CD1484A2E
:1031F0005278032A04D0464A5278062A00D0012188
:10320000434A5278032A24D119BB0023404A12783A
:10321000203A02EBC20404EB421200EB4202A2F895
:103220004A3001233A4A1278203A02EBC20404EBF6
:10323000421200EB4202A2F85030354AD37812789D
:10324000203A02EBC20404EB421220F8123000BF15
:1032500059E02F4A5278062A55D1002953D12C4AD9
:10326000D2782B4BDA704EE0294A1278232A03D009
:10327000274A1278242A46D1254A5278032A04D0B4
:10328000234A5278062A00D00121214A5278032A83
:1032900030D171BB00231E4A1278203A02EBC204DF
:1032A00004EB421200EB4202A2F84A300123184A12
:1032B0001278203A02EBC20404EB421200EB420205
:1032C000A2F85030124A1278223A02EBC20404EB00
:1032D000421200EB420253840D4A1278223A02EB6A
:1032E000C20404EB421200EB4202A2F8423000BFDB
:1032F00009E0FFE7064A5278062A04D119B9044AC0
:10330000D278034BDA7010BD9C4B002000250020C2
:10331000002B002010B504460CB9012010BD6079C7
:1033200020B900202071204600F004F801206071CF
:103330000020F3E708B5094A016891420DD100BFAA
:103340000749496941F04001054A516111464969FF
:1033500001F04001009100BF00BF08BD00300240F5
:1033600000100240F0B5034600BF5879012801D192
:103370000220F0BD0120587100BF022018711868AA
:10338000046802F0100640F6FE70B0408443D1E9B4
:10339000000640EA060502F0100005FA00F00443BA
:1033A000186804601868006802F01007C026BE4064
:1033B000B0431E6830601868006802F01007C0262D
:1033C000BE40B0431E6830600120187100BF00206D
:1033D000587100BF00BFCCE710B504460CB90120FE
:1033E00010BD207920B900206071204600F008F857
:1033F0000220207100202061012020710020EFE7D1
:1034000010B586B004460020029003900490059009
:103410002249206888423ED100BF2148C06940F05F
:1034200000501F49C8610846C06900F00050019073
:1034300000BF00BF00BF0846806940F004008861FB
:103440000846806900F00400019000BF00BF202002
:1034500002900320039002A9124800F06FFC12486A
:1034600012490860102048600021104881608021C6
:10347000C160490001618900416120218161002111
:10348000C16100F0E1FA08B1FEF7B3F800BF0748E8
:10349000E060446200BF06B010BD00000074004050
:1034A0000010024000080140440402407C0A002051
:1034B0000146002291F82100022808D004208863E8
:1034C00000BF002081F8200000BF0120704708687D
:1034D000006820F00E000B6818600868006820F093
:1034E00001000B68186091F8403001209840CB6BC8
:1034F0005860012081F8210000BF002081F82000E1
:1035000000BF1046E2E7000070B50446002594F8BD
:103510002100022803D00420A0630125C1E0206817
:10352000006820F00E00216808602068006820F024
:103530000100216808605C492068884252D95A49D4
:1035400078392068884201D1012047E05649643922
:103550002068884201D1102040E05349503920684A
:10356000884201D1801539E04F493C3920688842B2
:1035700001D1801432E04C4928392068884202D1B8
:103580004FF480302AE0484914392068884202D13B
:103590004FF4801022E044492068884201D1400461
:1035A0001CE042492068884201D1012016E03F49D1
:1035B00014312068884201D110200FE03B492831A6
:1035C0002068884201D1801508E038493C312068E4
:1035D000884201D1801401E04FF480303349091F43
:1035E000086051E0304978392068884201D10120D3
:1035F00047E02D4964392068884201D1102040E01D
:10360000294950392068884201D1801539E026497E
:103610003C392068884201D1801432E0224928399F
:103620002068884202D14FF480302AE01E491439C4
:103630002068884202D14FF4801022E01A492068A5
:10364000884201D140041CE018492068884201D119
:10365000012016E0154914312068884201D110205C
:103660000FE0124928312068884201D1801508E016
:103670000E493C312068884201D1801401E04FF4AA
:103680008030094980394860012084F8210000BF5A
:10369000002084F8200000BF606B10B12046616BF1
:1036A0008847284670BD00008000024008040240A0
:1036B00070B50446E06B05682068066894F8401011
:1036C000042088402840002875D006F00400002817
:1036D000FAD02068006800F0200028B9206800684F
:1036E00020F0040021680860D5492068884254D938
:1036F000D34978392068884201D1042049E0D04973
:1037000064392068884201D1402042E0CC495039D8
:103710002068884201D100153BE0C9493C39206846
:10372000884202D14FF4804033E0C54928392068EF
:10373000884202D14FF480202BE0C149143920681F
:10374000884202D14FF4800023E0BD4920688842BE
:1037500001D1C0041DE0BB492068884201D104208A
:1037600017E0B84914312068884201D1402010E0A8
:10377000B44928312068884201D1001509E0B149D7
:103780003C312068884202D14FF4804001E04FF480
:103790008020AC49091F086054E0A94978392068A5
:1037A000884201D104204AE0A54964392068884252
:1037B00002D1402043E04CE0A149503920688842C2
:1037C00001D100153BE09E493C392068884202D176
:1037D0004FF4804033E09A4928392068884202D16A
:1037E0004FF480202BE0964914392068884202D19A
:1037F0004FF4800023E092492068884201D1C00440
:103800001DE090492068884201D1042017E08D49CD
:1038100014312068884201D1402010E089492831C4
:103820002068884201D1001509E086493C312068B2
:10383000884202D14FF4804001E04FF4802080495B
:1038400080394860E06A002802D02046E16A884753
:10385000F4E094F84010022088402840002871D0FD
:1038600006F002000028FAD02068006800F020006E
:1038700040B92068006820F00A0021680860012033
:1038800084F821006E492068884254D96C497839FF
:103890002068884201D1022049E0694964392068E2
:1038A000884201D1202042E0654950392068884291
:1038B00001D140153BE062493C392068884202D181
:1038C0004FF4005033E05E4928392068884202D125
:1038D0004FF400302BE05A4914392068884202D155
:1038E0004FF4001023E056492068884201D180043B
:1038F0001DE054492068884201D1022017E0514957
:1039000014312068884201D1202010E04D4928312F
:103910002068884201D1401509E04A493C312068BD
:10392000884202D14FF4005001E04FF40030454985
:10393000091F086054E0424978392068884202D162
:1039400002204AE057E03E4964392068884201D1AC
:10395000202042E03A4950392068884201D1401580
:103960003BE037493C392068884202D14FF400508F
:1039700033E0334928392068884202D14FF40030BF
:103980002BE02F4914392068884202D14FF40010EF
:1039900023E02B492068884201D180041DE0294999
:1039A0002068884201D1022017E02649143120689E
:1039B000884201D1202010E0224928312068884225
:1039C00001D1401509E01F493C312068884202D1ED
:1039D0004FF4005001E04FF400301949803948603D
:1039E00000BF002084F8200000BFA06A30B320464A
:1039F000A16A884722E094F84010082088402840B7
:103A0000E0B106F00800C8B12068006820F00E00A0
:103A10002168086094F8401001208840E16B4860FC
:103A20000120A06384F8210000BF002084F820005A
:103A300000BF206B10B12046216B884770BD00008D
:103A400080000240080402400146002209B901201A
:103A500070471E4B086898420BD21D4B0868C01A6D
:103A60001423B0FBF3F08000086419480838C863D9
:103A70000AE0164B0868C01A1423B0FBF3F080006C
:103A8000086412480838C863022081F821000868D9
:103A9000026843F6F0708243D1E901031843CB6812
:103AA00018430B6918434B6918438B691843CB695A
:103AB000184302430868026000208863012081F8EF
:103AC0002100002081F8200000BFC1E70804024067
:103AD000080002402DE9F04104460D4616461F46F7
:103AE0004FF0000800BF94F82000012802D1022006
:103AF000BDE8F081012084F8200000BF94F8210087
:103B000001282CD1022084F821000020A063206825
:103B1000006820F00100216808603B4632462946D3
:103B20002046FDF74FFDE06A30B12068006840F0A4
:103B30000E00216808600BE02068006820F0040097
:103B4000216808602068006840F00A002168086069
:103B50002068006840F001002168086006E000BFAE
:103B6000002084F8200000BF4FF002084046BFE765
:103B700070B5044600F09AFA06462546681C10B156
:103B800004480078054400BF00F090FA801BA8426A
:103B9000FAD370BDEC0900202DE9F04104460E4631
:103BA0000127002500BF2648007E012802D10220FF
:103BB000BDE8F08101202249087600BF2068022874
:103BC00013D14CF25030FDF791FD90BB0120FDF771
:103BD00013FD4CF25030FDF789FD07461948006986
:103BE00020F004001749086123E04CF25030FDF743
:103BF0007DFDF0B94FF0FF303060A56812E0284637
:103C0000FDF70EFD4CF25030FDF770FD07460D48F4
:103C1000006920F002000B4908610FB1356007E030
:103C200005F50065D4E9021001EBC020A842E6D8F2
:103C300000BF00BF00200249087600BF3846B7E742
:103C4000880F0020002002400348006940F08000F7
:103C50000149086100207047002002402DE9FE4F15
:103C600005468B4617469846012600240020029000
:103C700000BF2448007E012802D10220BDE8FE8F4B
:103C800001202049087600BF4CF25030FDF72EFD90
:103C9000064686BB012D02D10120029006E0022DCE
:103CA00002D10220029001E00420029000241EE0D4
:103CB0002201B946C24648465146FCF7A1FA80B2F5
:103CC0000190022000FB04B000900199FDF7BCFCBC
:103CD0004CF25030FDF70AFD06460B48006920F013
:103CE00001000949086106B104E0601CC4B20298F1
:103CF0008442DDDB00BF00BF00200249087600BF20
:103D00003046BBE7880F0020002002400020084911
:103D1000096901F0800151B10649054A516006491F
:103D200051601146096901F0800101B1012070471D
:103D30000020024023016745AB89EFCD2DE9F8470C
:103D4000024600239C467BE14FF0010808FA03F489
:103D5000D1F8008008EA0400A0427DD1DFF8F4A287
:103D6000D1F80480A8EB0A09D0453AD014DCB8F1A8
:103D7000030F50D009DCB8F1000F31D0B8F1010FBA
:103D80001CD0B8F1020F49D120E0B8F1110F18D0C2
:103D9000B8F1120F42D11EE0B9F5881F25D006DC1C
:103DA000B9F5803F20D0B9F5801F37D11AE0B9F5B9
:103DB000001F18D0B9F5041F30D117E0D1F80CC09E
:103DC0002DE0D1F80C8008F1040C28E0D1F80C802B
:103DD00008F1080C23E0D1F80C8008F10C0C1EE06F
:103DE00000BF00BF00BF00BF00BF00BFD1F8088008
:103DF000B8F1000F02D14FF0040C0BE0D1F80880AD
:103E0000B8F1010F03D14FF0080C146102E04FF03C
:103E1000080C546103E04FF0000C00E000BF00BF4D
:103E2000FF2801D8904601E002F104084646FF2829
:103E300002D84FEA830803E0A3F108084FEA880894
:103E40004746D6F800804FF00F0909FA07F928EA2B
:103E500009080CFA07F900E07AE048EA0908C6F810
:103E60000080D1F8048008F08058B8F1805F6FD1ED
:103E700000BFDFF8E481D8F8188048F00108DFF8C7
:103E8000D891C9F81880C846D8F8188008F00108F9
:103E9000CDF8008000BF00BF4FEAB9384FEA930960
:103EA00058F829504FEA83784FEA18794FF00F08F5
:103EB00008FA09F825EA0805DFF8A081424502D191
:103EC0004FF0000824E0DFF89881424502D14FF01E
:103ED00001081DE0DFF88C81424502D14FF0020855
:103EE00016E0DFF88481424502D14FF003080FE06D
:103EF000DFF87881424502D14FF0040808E0DFF88E
:103F00007081424502D14FF0050801E04FF00608EC
:103F10004FEA83794FEA197908FA09F848EA050562
:103F2000DFF850814FEA930948F82950D1F804800E
:103F300008F48038B8F5803F0BD1DFF83C81D8F821
:103F4000008048EA0008DFF83091C9F800800AE0F4
:103F500075E0DFF82481D8F8008028EA0008DFF84F
:103F60001891C9F80080D1F8048008F40038B8F539
:103F7000003F0ED1DFF8008108F10408D8F8008076
:103F800048EA0008DFF8F09009F10409C9F8008058
:103F90000DE0DFF8E48008F10408D8F8008028EA92
:103FA0000008DFF8D49009F10409C9F80080D1F8BD
:103FB000048008F48018B8F5801F0ED1DFF8B880AF
:103FC00008F10808D8F8008048EA0008DFF8A8904F
:103FD00009F10809C9F800800DE0DFF89C8008F1BC
:103FE0000808D8F8008028EA0008DFF88C9009F16A
:103FF0000809C9F80080D1F8048008F40018B8F561
:10400000001F0ED1DFF8708008F10C08D8F800808E
:1040100048EA0008DFF8609009F10C09C9F800804F
:104020000DE0DFF8548008F10C08D8F8008028EA89
:104030000008DFF8449009F10C09C9F800805B1C06
:10404000D1F8008028FA03F8B8F1000F7FF47CAEB5
:10405000BDE8F88700001110001002400008014080
:10406000000C014000100140001401400018014004
:10407000001C014008000140000401400246936812
:104080000B400BB1012000E00020704710B5C26862
:1040900021EA020302EA010443EA0443036110BD7A
:1040A0000AB1016101E00B04036170470148006837
:1040B00070470000E40900200348006803490978BC
:1040C0000844014908607047E4090020EC09002019
:1040D00010B50848006840F0100006490860032049
:1040E00000F0CCF8002000F007F800F049F80020BC
:1040F00010BD00000020024070B588B004460025C5
:104100000026002221462C2000F07AF82C2000F016
:1041100067F800BF1648806940F400501449886170
:104120000846806900F40050019000BF00BF02A95A
:1041300003A800F07DF900F0B3F905460D48B5FB82
:10414000F0F0461E0C480D49086040F2E7310B487C
:10415000C160466000210161816000F07DFC20B9F2
:10416000064800F0D9FC08B070BD0120FBE7000054
:104170000010024040420F00003401403C0F00207C
:1041800008B500BF1448806940F0010012498861F9
:104190000846806900F00100009000BF00BF00BF2A
:1041A0000846C06940F08050C8610846C06900F008
:1041B0008050009000BF00BF00220F21901E00F031
:1041C0001FF800BF0549486820F0E06040F000702B
:1041D000486000BF08BD0000001002400000014020
:1041E00001460846002809DB00F01F0301229A401F
:1041F00043099B0003F1E023C3F8002100BF70478F
:104200002DE9F05F80460D461646002708F0E2FED5
:10421000074639462A46334601F00700C0F1070A2F
:10422000BAF1040F02D94FF0040A01E0C0F1070A05
:10423000D14600F1040ABAF1070F02D24FF0000A8A
:1042400001E0A0F1030AD4464FF0010A0AFA09FA84
:10425000AAF1010A0AEA020A0AFA0CFA4FF0010B63
:104260000BFA0CFBABF1010B0BEA030B4AEA0B0454
:104270002146404608F0B6FEBDE8F09F00BF00F0C2
:104280000702064B19684FF6FF031940044B0B4316
:1042900043EA0221014B196000BF70470CED00E0BA
:1042A0000000FA0570B504460D460CB9012070BD3A
:1042B0005A48006800F00700A8420ED2574800682C
:1042C00020F007002843554908600846006800F0C0
:1042D0000700A84201D00120E9E7207800F00200A1
:1042E00002281DD1207800F00400042805D14C4894
:1042F000406840F4E0604A494860207800F00800D7
:10430000082805D14648406840F460504449486058
:104310004348406820F0F000A168084340494860E5
:10432000207800F0010078B36068012806D13C488D
:10433000006800F4003090B90120B8E760680228F6
:1043400006D13748006800F0007040B90120AEE7A0
:104350003348006800F0020008B90120A7E73048A0
:10436000406820F00300616808432D494860FFF76A
:104370009DFE064609E0FFF799FE801B41F2883159
:10438000884202D9032092E707E02548406800F000
:104390000C006168B0EB810FEDD12048006800F09F
:1043A0000700A8420ED91D48006820F007002843E6
:1043B0001A4908600846006800F00700A84201D0CA
:1043C000012074E7207800F00400042807D1144885
:1043D000406820F4E060E1680843114948602078B3
:1043E00000F00800082808D10D48406820F460500B
:1043F000216940EAC1000A49486000F061F80849B3
:104400004968C1F30311074A515CC8400649086076
:1044100006480068FFF770FE002048E700200240D1
:1044200000100240640D0108E0090020E8090020A6
:104430000F2202600D4A526802F0030242600B4AEA
:10444000526802F0F0028260084A526802F4E062A8
:10445000C260064A526802F46052D2080261044AFD
:10446000126802F007020A60704700000010024064
:10447000002002400148006870470000E009002069
:1044800000B5FFF7F7FF04494968C1F30221034A69
:10449000515CC84000BD000000100240740D0108CE
:1044A00000B5FFF7E7FF04494968C1F3C221034A99
:1044B000515CC84000BD000000100240740D0108AE
:1044C000F0B585B00FF26C0C9CE8E01001A8A0E8F4
:1044D000E0101CA52D680095002100220023002477
:1044E0000020194D696801F00C05F5B1042D02D0CA
:1044F000082D19D101E0154819E001ADC1F383463B
:10450000AC5D01F4803555B10F4D6D68C5F3404584
:104510001DF805200D4D6543B5FBF2F302E00C4D8F
:1045200004FB05F3184602E000BF084800BF00BFC7
:1045300005B0F0BD02030405060708090A0B0C0DBF
:104540000E0F1010010200000010024000127A004D
:1045500000093D00F8B504460CB90120F8BD2078EB
:1045600000F00100002878D0F848406800F00C0006
:1045700004280CD0F548406800F00C00082811D140
:10458000F248406800F48030B0F5803F0AD1EF482F
:10459000006800F4003000285FD0606800285CD11B
:1045A0000120DBE700BF6068B0F5803F06D1E74837
:1045B000006840F48030E549086028E0606858B938
:1045C000E248006820F48030E0490860084600684E
:1045D00020F4802008601AE06068B0F5A02F0BD1AD
:1045E000DA48006840F48020D8490860084600682E
:1045F00040F4803008600AE0D448006820F480303D
:10460000D24908600846006820F48020086000BF96
:10461000606888B1FFF74AFD054606E0FFF746FDF2
:10462000401B642801D9032098E7C848006800F4BB
:1046300000300028F2D010E0FFF738FD054606E014
:10464000FFF734FD401B642801D9032086E7BF48EB
:10465000006800F400300028F2D1207800F0020059
:10466000022857D1B948406800F00C0050B1B74853
:10467000406800F00C00082818D1B448406800F4E5
:10468000803098B9B148006800F0020020B120697C
:10469000012801D0012061E7AC48006820F0F80053
:1046A000616940EAC100A949086033E02069E8B1C6
:1046B0000120A7490860FFF7F9FC054606E0FFF76F
:1046C000F5FC401B022801D9032047E79F480068FA
:1046D00000F002000028F2D09C48006820F0F800AA
:1046E000616940EAC1009949086013E000209849D7
:1046F0000860FFF7DBFC054606E0FFF7D7FC401B30
:10470000022801D9032029E79048006800F0020040
:104710000028F2D1207800F0080008282DD1A069E7
:10472000B8B101208B490860FFF7C0FC054606E0E0
:10473000FFF7BCFC401B022801D903200EE7834889
:10474000406A00F002000028F2D0012001F0EAFCEB
:1047500013E000207F490860FFF7A8FC054606E04B
:10476000FFF7A4FC401B022801D90320F6E6774896
:10477000406A00F002000028F2D1207800F0040026
:10478000042873D100277148C06900F0805070B9C7
:1047900000BF6E48C06940F080506C49C86108464F
:1047A000C06900F08050009000BF00BF01276A4838
:1047B000006800F48070B0B96748006840F4807009
:1047C00065490860FFF772FC054606E0FFF76EFCDE
:1047D000401B642801D90320C0E65F48006800F44C
:1047E00080700028F2D000BFE068012806D1574849
:1047F000006A40F001005549086227E0E06858B9B6
:104800005248006A20F00100504908620846006AD8
:1048100020F00400086219E0E06805280BD14B483D
:10482000006A40F00400494908620846006A40F006
:10483000010008620AE04548006A20F0010043498F
:1048400008620846006A20F00400086200BFE068C1
:10485000A0B1FFF72BFC054609E0FFF727FC401B42
:1048600041F28831884202D9032077E622E03748B6
:10487000006A00F002000028EFD012E0FFF716FCFB
:10488000054608E0FFF712FC401B41F288318842E0
:1048900001D9032062E62D48006A00F002000028DA
:1048A000F0D1012F05D12948C06920F08050274957
:1048B000C86100BFE069C8B32448406800F00C003C
:1048C000082860D0E069022848D100202049086605
:1048D000FFF7ECFB054606E0FFF7E8FB401B02286C
:1048E00001D903203AE61948006800F0007000285A
:1048F000F2D1206AB0F5803F07D11448406820F417
:104900000030A168084311494860D4E90801084310
:104910000E49496821F4741108430C49486001208C
:104920000B490866FFF7C2FB054607E03DE0FFF7CD
:10493000BDFB401B022801D903200FE60348006895
:1049400000F000700028F2D02FE0000000100240BC
:10495000000042428004424200700040002014499E
:104960000866FFF7A3FB054606E0FFF79FFB401B29
:10497000022801D90320F1E50E48006800F000701C
:104980000028F2D111E0E069012800D1E6E50948EC
:10499000466806F48031206A814204D106F4701121
:1049A000606A814201D00120D8E50020D6E50000F0
:1049B00000004242001002407047704730B5024686
:1049C0000B4600BF92F83C00012801D1022030BD07
:1049D000012082F83C0000BF022082F83D001068F0
:1049E00044681068816824F07004186804431068F3
:1049F0004460144D1068A84213D0134D1068A842AB
:104A00000FD01068B0F1804F0BD0104D1068A84245
:104A100007D00F4D1068A84203D00E4D1068A84271
:104A200005D121F0800158680143106881600120A0
:104A300082F83D0000BF002082F83C0000BF00BFAC
:104A4000C5E70000002C0140003401400004004094
:104A500000080040000C004010B504460CB90120CD
:104A600010BD94F83D0028B9002084F83C00204691
:104A700000F026F8022084F83D00211D206807F090
:104A80009DFC012084F8460000BF84F83E0001210F
:104A90003F200155402001554120015500BF00BF76
:104AA000012084F84200432001554420015545204F
:104AB000015500BF012084F83D000020D0E7000030
:104AC00008B5124A016891420DD100BF10498969A9
:104AD00041F400610E4A91611146896901F4006157
:104AE000009100BF11E00B4A016891420DD100BF57
:104AF0000749C96941F00401054AD1611146C969F4
:104B000001F00401009100BF00BF08BD002C01406E
:104B10000010024000080040014691F83D000128C5
:104B200001D001207047022081F83D000868C0686C
:104B300040F001000B68D860164B0868984213D00B
:104B4000154B086898420FD00868B0F1804F0BD021
:104B5000124B0868984207D0114B0868984203D05E
:104B6000104B086898420CD10868806800F0070272
:104B7000062A0CD00868006840F001000B68186035
:104B800005E00868006840F001000B68186000202C
:104B9000C8E70000002C0140003401400004004040
:104BA00000080040000C00402DE9F04104460D468D
:104BB00000BF94F83C00012802D10220BDE8F0813A
:104BC000012084F83C0000BF022084F83D002068EA
:104BD000866826F0770626F47F4620688660286877
:104BE000502833D00CDC202850D004DC00284BD0D7
:104BF000102851D149E0302849D040284CD139E023
:104C000060282DD0702807D0B0F5805F03D0B0F5B4
:104C1000005F41D10DE040E0D5E902136A682068E9
:104C200007F01AFC2068866846F0770620688660E0
:104C300033E0D5E902136A68206807F00DFC2068AC
:104C4000806840F480402168886026E0EA686968EE
:104C5000206807F015FC5021206807F008FC1CE0D4
:104C6000EA686968206807F01EFC6021206807F088
:104C7000FEFB12E0EA686968206807F001FC402149
:104C8000206807F0F4FB08E000BF00BF00BF296800
:104C9000206807F0ECFB00E000BF00BF012084F8B3
:104CA0003D0000BF002084F83C0000BF00BF85E746
:104CB000704710B5044620680069C0F34000D8B1C1
:104CC0002068C068C0F34000B0B16FF002002168F6
:104CD0000861012020772068806900F0030018B186
:104CE0002046FFF7E5FF05E0204600F0ADF820463E
:104CF00000F0ABF80020207720680069C0F3800046
:104D0000D8B12068C068C0F38000B0B16FF0040073
:104D100021680861022020772068806900F44070D3
:104D200018B12046FFF7C4FF05E0204600F08CF8DC
:104D3000204600F08AF80020207720680069C0F340
:104D4000C000D8B12068C068C0F3C000B0B16FF037
:104D5000080021680861042020772068C06900F0FD
:104D6000030018B12046FFF7A3FF05E0204600F03E
:104D70006BF8204600F069F8002020772068006971
:104D8000C0F30010D8B12068C068C0F30010B0B103
:104D90006FF0100021680861082020772068C06942
:104DA00000F4407018B12046FFF782FF05E020466E
:104DB00000F04AF8204600F048F8002020772068EC
:104DC000006900F0010058B12068C06800F00100DF
:104DD00030B16FF0010021680861204600F036F81C
:104DE00020680069C0F3C01058B12068C068C0F3E3
:104DF000C01030B16FF08000216808612046FFF7D5
:104E0000DBFD20680069C0F3801058B12068C068DD
:104E1000C0F3801030B16FF0400021680861204677
:104E200000F020F820680069C0F3401058B12068F5
:104E3000C068C0F3401030B16FF0200021680861F5
:104E40002046FFF7BAFD10BD7047704710B5044605
:104E500003492068884201D1FFF72EF910BD0000F8
:104E600000340140704770B5044600252068406951
:104E7000C0F3C01594F8390021280ED16DB1206817
:104E8000406920F0800021684861206B10B1206BE0
:104E9000FEF70EFB204607F01EFC20684069C0F3B9
:104EA000801594F83A0022280ED16DB1206840692F
:104EB00020F0400021684861606B10B1606BFEF724
:104EC000F7FA204607F0E7FB002070BD70470000AE
:104ED0002DE9F0470446206805682068C668206808
:104EE00047694FF00008C14605F00F08B8F1000F00
:104EF0000AD105F0200038B106F0200020B120468C
:104F000007F0F3FBBDE8F087B8F1000F71D007F0B0
:104F1000010018B906F4907000286AD005F001006D
:104F200030B106F4807018B1E06B40F00100E0632E
:104F300005F0040030B107F0010018B1E06B40F05B
:104F40000200E06305F0020030B107F0010018B183
:104F5000E06B40F00400E06305F0080048B106F0A3
:104F6000200010B907F0010018B1E06B40F0080014
:104F7000E063E06B68B305F0200028B106F0200084
:104F800010B1204607F0B1FB20684069C0F38019DA
:104F9000E06B00F0080010B9B9F1000F22D02046F4
:104FA00007F079FB2068406900F04000B0B120684C
:104FB000406920F0400021684861606B50B118489A
:104FC000616B4863606BFEF79FFA10B1606B416BD9
:104FD00088470CE02046FFF779FF08E02046FFF7FE
:104FE00075FF04E02046FFF771FF0020E06389E7CA
:104FF000FFE705F0800030B106F0800018B12046D0
:1050000007F042FC7EE705F0400030B106F04000BA
:1050100018B1204607F04FFB74E700BF72E70000AD
:10502000DFC5000810B504460CB9012010BDA06909
:1050300000B100E000BF94F8390028B9002084F8DE
:105040003800204600F028F8242084F83900206831
:10505000C06820F400502168C860204607F096FB25
:105060002068006920F49040216808612068406948
:1050700020F02A00216848612068C06840F4005090
:105080002168C8600020E063202084F8390084F89B
:105090003A000020CAE7000010B586B004460020A0
:1050A0000290039004900590A249206888423BD169
:1050B00000BFA148C06940F480109F49C8610846FC
:1050C000C06900F48010019000BF00BF00BF084617
:1050D000806940F0100088610846806900F0100087
:1050E000019000BF00BF00BF0846806940F020006B
:1050F00088610846806900F02000019000BF00BF71
:1051000088140290022003900320059002A98B4886
:10511000FEF714FE0420029000200390049002A9E0
:105120008748FEF70BFE02E186492068884263D17A
:1051300000BF8148806940F480407F49886108460B
:10514000806900F48040019000BF00BF00BF0846A6
:10515000806940F0040088610846806900F004001E
:10516000019000BF00BF4815029002200390032069
:10517000059002A97448FEF7E1FD4FF480600290AB
:1051800000200390049002A96F48FEF7D7FD6F48F6
:105190006F4908600020486000216D4881608021CF
:1051A000C160002101614161202181610902C16169
:1051B000FEF74AFC08B1FCF71CFA00BF64486063C4
:1051C000446200BF6148143862490860102048609A
:1051D0000021604881608021C1600021016141613E
:1051E0008161C161FEF730FC08B1FCF702FA00BF33
:1051F0005848206344629AE057492068884249D160
:1052000000BF4D48C06940F400304B49C8610846B2
:10521000C06900F40030019000BF00BF00BF084625
:10522000806940F0040088610846806900F004004D
:10523000019000BF00BF04200290022003900320D1
:10524000059002A94048FEF779FD08200290002051
:105250000390049002A93C48FEF770FD3B481430CF
:105260003E4908600020486000213C488160802160
:10527000C160002101614161202181610902C16198
:10528000FEF7E2FB08B1FCF7B4F900BF33486063F6
:1052900044624CE032492068884248D100BF264829
:1052A000C06940F480202449C8610846C06900F400
:1052B0008020019000BF00BF00BF0846806940F019
:1052C000080088610846806900F00800019000BF6E
:1052D00000BF08150290022003900320059002A948
:1052E0002048FEF72BFD4FF4006002900020039051
:1052F000049002A91B48FEF721FD144828381A49DA
:105300000860002048600021174881608021C1604A
:105310000021016141618161C161FEF795FB08B126
:10532000FCF767F900BF10486063446200BF06B035
:1053300010BD00000050004000100240001001406D
:1053400000140140003801400008014058000240AC
:10535000500C0020940C002000440040D80C002089
:1053600000480040000C01401C0D002077B581B0C2
:105370000446154694F83A00202850D1029800B10E
:1053800015B9012004B070BD00BF94F838000128A1
:1053900001D10220F6E7012084F8380000BF02980E
:1053A000A062A5850020E063222084F83A001D4811
:1053B000616B88621C48616BC8621C48616B086342
:1053C0000020616B486302AE32682368191D2B46CA
:1053D000606BFEF77FFB00BF002000902068006834
:1053E000009020684068009000BF00BF00BF002010
:1053F00084F8380000BF2068C06840F480702168DD
:10540000C8602068406940F0010021684861206858
:10541000406940F04000216848610020B2E7022066
:10542000B0E7000043C6000889C60008F3C50008BD
:10543000704770472DE9F84F04460E4617469946C7
:105440004FF0000A94F8390020285AD106B117B954
:105450000120BDE8F88F00BF94F83800012801D181
:105460000220F6E7012084F8380000BF0020E06346
:10547000212084F83900FEF719FE8246A784E784CC
:10548000A068B0F5805F04D1206910B90025B0464E
:1054900002E035464FF0000800BF002084F83800D5
:1054A00000BF1BE05346002280212046CDF800902B
:1054B00007F01AFA08B10320CBE745B9B8F80000A5
:1054C000C0F308002168486008F1020803E028786A
:1054D000216848606D1CE08C401EE084E08C002850
:1054E000E0D15346002240212046CDF8009007F03D
:1054F000FBF908B10320ACE7202084F83900002034
:10550000A7E70220A5E770472DE9F0410746364D91
:10551000002400266888002862D1287D06285CD1F6
:1055200001206880AA7F2046611CCCB22F490A5412
:1055300006222046611CCCB22C490A540022204687
:10554000611CCCB229490A54A5222046611CCCB268
:1055500026490A542046611CCCB224490A542046EC
:10556000611CCCB221490A542046611CCCB21F49AF
:105570000A542046611CCCB21C490A542046611CC6
:10558000CCB21A490A542046611CCCB217490A54BD
:105590002046611CCCB215490A542046611CCCB28D
:1055A00012490A542046611CCCB210490A542046C4
:1055B000611CCCB20D490A540E210C4800F0F2F9DE
:1055C000064632122046611CCCB208490A542046D5
:1055D000611CCCB205490E5404E00020BDE8F08106
:1055E0000020FBE70120F9E7E23900209C39002088
:1055F000F0B58BB00646344F344D282101A8FAF798
:105600002EFE002400BF09E004F1100005F10D0199
:10561000085C01A921F81400601CC4B2287EA042D5
:10562000F2DC287D062804D10122294901A8FCF7D3
:10563000ABF80122264901A8FCF790F8BDF8040058
:105640003074BDF80400052802DABDF80400F880C3
:10565000287D062805D108221E490DF10600FCF719
:1056600093F808221B490DF10600FCF777F8002497
:1056700024E001A9601C31F81020103005F10D0163
:10568000085C824205D0287D062802D100200BB09C
:10569000F0BD01A9601C31F8100008280CDA601C6C
:1056A00031F8101007F1240020F8141001A9601C33
:1056B00011F8101010303154601CC4B2287EA04282
:1056C000D7DC0120E3E70000A0380020E239002009
:1056D00030F0070840E007082DE9F0410746374D54
:1056E000002400266888002864D1287D06285ED121
:1056F00001206880AA7F2046611CCCB230490A5440
:1057000006222046611CCCB22D490A5410222046A4
:10571000611CCCB22A490A542020425D2046611CFB
:10572000CCB227490A54A5222046611CCCB2244998
:105730000A542046611CCCB221490A542046611CFF
:10574000CCB21F490A542046611CCCB21C490A54F1
:105750002046611CCCB21A490A542046611CCCB2C6
:1057600017490A542046611CCCB215490A542046F8
:10577000611CCCB212490A542046611CCCB21049BB
:105780000A542046611CCCB20D490A540E210C4823
:1057900000F008F9064632122046611CCCB20849D6
:1057A0000A542046611CCCB205490E5404E0002086
:1057B000BDE8F0810020FBE70120F9E7E239002095
:1057C0009C3900202DE9F0410746374D0024002682
:1057D0006888002864D1287D06285ED10120688071
:1057E000AA7F2046611CCCB230490A5406222046CA
:1057F000611CCCB22D490A5412222046611CCCB245
:105800002A490A542020425D2046611CCCB2274917
:105810000A54A5222046611CCCB224490A542046D1
:10582000611CCCB221490A542046611CCCB21F49EC
:105830000A542046611CCCB21C490A542046611C03
:10584000CCB21A490A542046611CCCB217490A54FA
:105850002046611CCCB215490A542046611CCCB2CA
:1058600012490A542046611CCCB210490A54204601
:10587000611CCCB20D490A540E210C4800F092F87C
:10588000064632122046611CCCB208490A54204612
:10589000611CCCB205490E5404E00020BDE8F08143
:1058A0000020FBE70120F9E7E23900209C390020C5
:1058B0002DE9F0410746384D00240026688800286D
:1058C00065D1287D06285FD101206880AA7F204607
:1058D000611CCCB231490A5406222046611CCCB26C
:1058E0002E490A5414222046611CCCB22B490A547A
:1058F000EA7F2046611CCCB228490A542020425D30
:105900002046611CCCB225490A54A5222046611CC0
:10591000CCB222490A542046611CCCB21F490A5419
:105920002046611CCCB21D490A542046611CCCB2F1
:105930001A490A542046611CCCB218490A54204620
:10594000611CCCB215490A542046611CCCB21349E3
:105950000A542046611CCCB210490A542046611CEE
:10596000CCB20E490A540E210C4800F01BF8064632
:1059700032122046611CCCB208490A542046611CF0
:10598000CCB206490E5404E00020BDE8F0810020AE
:10599000FBE70120F9E70000E23900209C390020F4
:1059A00000BFFEE770B502460B46FF24FF2509E065
:1059B00012F8010B80EA04010748405C80EA050404
:1059C0000648455C181EA3F10106B3B2F0D105EB01
:1059D000042080B270BD00004400010844010108A9
:1059E00004E0002200F8012B4A1E91B20029F8DCE5
:1059F0007047000070B58AB005466D4C6D4E282189
:105A00006846FAF72CFCA17F607F41EA0020ADF8E0
:105A100000002020015DE07F41EA0020ADF8020097
:105A20002220015D2120005D41EA0020ADF8040044
:105A30002420015D2320005D41EA0020ADF806002E
:105A40002620015D2520005D41EA0020ADF8080018
:105A50002820015D2720005D41EA0020ADF80A0002
:105A60002A20015D2920005D41EA0020ADF80C00EC
:105A70002C20015D2B20005D41EA0020ADF80E00D6
:105A8000207D062804D108224B496846FBF77CFE9E
:105A9000082249496846FBF761FEBDF80000001284
:105AA0002874BDF800006874BDF802000012A874E4
:105AB000BDF80200E874BDF8040000122875BDF8B6
:105AC00004006875BDF806000012A875BDF8060050
:105AD000E875BDF8080000122876BDF80800687661
:105AE000BDF80A000012A876BDF80A00E876BDF8F5
:105AF0000C0000122877BDF80C006877BDF80E0086
:105B00000012A877BDF80E00E877297C607F8142FB
:105B10004CD1697CA07F814248D1207D062845D1A7
:105B2000607F2649C870A07F8870E07F4870202081
:105B3000005D087008460168F16400BF2120005D27
:105B40001E49C8702220005D88702320005D4870C7
:105B50002420005D087008460168716700BF252099
:105B6000005D1649C8702620005D88702720005D02
:105B700048702820005D0870084601689C2081510B
:105B800000BF2920005D0D49C8702A20005D887083
:105B90002B20005D48702C20005D087008460168CD
:105BA000C420815100BF01200AB070BD0020FBE776
:105BB000E23900209840002000C007085803002068
:105BC00070B58AB005461D4E1D4C28216846FAF76F
:105BD00046FBA17F607F41EA0020ADF80000207DF8
:105BE000062804D1012217496846FBF7CDFD0122A2
:105BF00014496846FBF7B2FDBDF800000012287496
:105C0000BDF800006874BDF800004FF6FF718842CF
:105C100003D0BDF80000A6F86400297C607F8142B3
:105C200009D1697CA07F814205D1207D062802D15F
:105C300001200AB070BD0020FBE70000A038002062
:105C4000E239002040F007082DE9F0410646377898
:105C500096F801803846FAF7E3FA3038C4B2092CD6
:105C600001DDE01FC4B24046FAF7DAFA3038C5B2B7
:105C7000092D01DDE81FC5B205EB0410C0B2BDE877
:105C8000F081000010B50548054908600846FDF799
:105C900041FB08B1FBF7ADFC10BD00000030024035
:105CA000FC0100201CB50020009001900A480B491F
:105CB00008600846FDF790FB08B1FBF79AFC3C2012
:105CC000009000200190102269460448FDF74AFB2D
:105CD00008B1FBF78EFC1CBD00740040680A002070
:105CE00008B500BF1548406940F0010013494861FC
:105CF0000846406900F00100009000BF00BF00BFEF
:105D00000846406940F0020048610846406900F0DA
:105D10000200009000BF00BF002205210E20FEF708
:105D20006FFA0E20FEF75CFA002205213B20FEF7F9
:105D300067FA3B20FEF754FA08BD0000001002404D
:105D400000B585B00020019002900390049000BF40
:105D50004548806940F020004349886108468069D1
:105D600000F02000009000BF00BF00BF084680691F
:105D700040F0040088610846806900F0040000904B
:105D800000BF00BF00BF0846806940F0080088617E
:105D90000846806900F00800009000BF00BF00BF07
:105DA0000846806940F0100088610846806900F06C
:105DB0001000009000BF00BF002213212B48FEF707
:105DC0006FF900224FF440512948FEF769F900228B
:105DD0004FF480612748FEF763F9132001900120FA
:105DE0000290002003900220049001A91F48FDF7B3
:105DF000A5FF4FF440500190012002900020039035
:105E00000220049001A91A48FDF798FF4FF4404082
:105E1000019000200290039001A91548FDF78EFF24
:105E20004FF47070019000200290039001A9114876
:105E3000FDF784FF4FF41060019000200290039062
:105E400001A90A48FDF77AFF4FF480600190012014
:105E50000290002003900220049001A90548FDF75C
:105E60006DFF05B000BD00000010024000080140B9
:105E7000000C01400010014010B500220521272030
:105E8000FEF7BEF92720FEF7ABF9002205212520F9
:105E9000FEF7B6F92520FEF7A3F9002205212620FA
:105EA000FEF7AEF92620FEF79BF9002205211E2001
:105EB000FEF7A6F91E20FEF793F90022052119200E
:105EC000FEF79EF91920FEF78BF90022052110201C
:105ED000FEF796F91020FEF783F9002205210F2026
:105EE000FEF78EF90F20FEF77BF9002205210D2029
:105EF000FEF786F90D20FEF773F910BD00B587B0E7
:105F0000002003900490059006900190029016489E
:105F100016490860002048600021144881604FF64F
:105F2000FF71C1604FF40071016100214161816125
:105F3000FEF792FD08B1FBF75CFB4FF48050039035
:105F400003A90A48FEF730FE08B1FBF752FB002018
:105F50000190029001A90548FEF730FD08B1FBF75A
:105F600048FB07B000BD0000002C0140C00A002023
:105F700000B587B000200390049005900690019032
:105F8000029014481449086000204860002112481B
:105F900081604FF6FF71C160002101618161FEF7F0
:105FA0005BFD08B1FBF725FB4FF48050039003A97C
:105FB0000948FEF7F9FD08B1FBF71BFB0020019033
:105FC000029001A90448FEF7F9FC08B1FBF711FBA8
:105FD00007B000BD00080040080B002010B50B48BA
:105FE0000B4908604FF4E1304860002108488160A7
:105FF000C16001610C21416100218161C161FFF734
:1060000011F808B1FBF7F5FA10BD00000050004090
:10601000500B002010B51248124908604FF416507A
:10602000486000210F488160C16001610C2141611D
:1060300000218161C161FEF7F5FF08B1FBF7D9FAD4
:1060400008480068C06840F0100006490968C86048
:106050004FF4807204490348FFF788F910BD00002F
:1060600000380140900B00200024002010B5124899
:10607000124908604FF41640486000210F488160C3
:10608000C16001610C21416100218161C161FEF7A4
:10609000C9FF08B1FBF7ADFA08480068C06840F0D6
:1060A000100006490968C8604FF48072044903482B
:1060B000FFF75CF910BD000000440040D00B002049
:1060C0000027002010B51248124908604FF41650FE
:1060D000486000210F488160C16001610C2141616D
:1060E00000218161C161FEF79DFF08B1FBF781FAD4
:1060F00008480068C06840F0100006490968C86098
:106100004FF4807204490348FFF730F910BD0000D6
:1061100000480040100C0020002A002000BFFEE7CD
:1061200000BFFEE708B508490968C9084FF47A724C
:10613000B1FBF2F14143009100BF00BF00994A1E3C
:1061400000920029F9D108BDE0090020F0B58BB01C
:106150003C4F3D4C3D4E002508223D4901A8FBF730
:10616000FDFA00BF0FE001A830F815004FF6FF71EF
:10617000884206D001A830F8151007F1340020F845
:106180001510681CC5B23888A842ECDC01223149E0
:1061900001A8FBF7E3FABDF804004FF6FF7188424F
:1061A00002D0BDF80400388101222A49383101A803
:1061B000FBF7D4FABDF804004FF6FF7188420DD109
:1061C0004FF41670A4F842000146A4F88810A4F811
:1061D000CE10A4F81411A4F85A1113E0BDF804006D
:1061E000A4F84200BDF80410A4F88810BDF804100B
:1061F000A4F8CE10BDF80410A4F81411BDF80410D2
:10620000A4F85A1100250EE0002030804FF6FF70F0
:10621000F080B0807080402106F11C00FFF7E0FBA9
:10622000681CC5B25C36082DEEDB002504E00220B8
:1062300009490870681CC5B23888A842F7DC0BB061
:10624000F0BD0000A038002040340020802E002047
:1062500020E0070820F007085003002070B586B042
:1062600004461A4E1A4D142101A8F9F7F8FFA97F28
:10627000687F41EA0020ADF80400287D062804D19B
:106280000122144901A8FBF77FFA0020ADF80400B1
:106290000122104901A8FBF761FABDF80400A6F835
:1062A0004200BDF8040000122074BDF804006074C0
:1062B000217C687F814206D1617CA87F814202D126
:1062C000012006B070BD0020FBE700004034002034
:1062D000E239002058F00708F0B58BB00646344F7D
:1062E000344D282101A8F9F7BAFF002400BF09E0C6
:1062F00004F1100005F10D01085C01A921F814005A
:10630000601CC4B2287EA042F2DC287D062804D19D
:106310000122294901A8FBF737FA0122264901A8E1
:10632000FBF71CFABDF804003074BDF80400052822
:1063300002DABDF804003881287D062805D108223C
:106340001E490DF10600FBF71FFA08221B490DF14B
:106350000600FBF703FA002424E001A9601C31F8D1
:106360001020103005F10D01085C824205D0287D17
:10637000062802D100200BB0F0BD01A9601C31F845
:10638000100008280CDA601C31F8101007F13400F6
:1063900020F8141001A9601C11F8101010303154AD
:1063A000601CC4B2287EA042D7DC0120E3E70000D5
:1063B000A0380020E239002020F0070820E007087C
:1063C0002DE9FC4180462E4D2E4F00240026002052
:1063D00000900190288800284ED1287D062848D1B9
:1063E00001202880AA7F2046611CCCB226490A548D
:1063F00006222046611CCCB223490A5400222046C2
:10640000611CCCB220490A5410222046611CCCB237
:106410001D490A5400222046611CCCB21A490A5474
:10642000FF222046611CCCB217490A54A87F8DF880
:10643000000006208DF8010000208DF802001020D9
:106440008DF8030000208DF80400FF208DF8050072
:1064500006216846FFF7A6FA064632122046611C5E
:10646000CCB209490A542046611CCCB206490E54EC
:1064700004E00020BDE8FC810020FBE70120F9E7F3
:10648000E2390020A0380020103900202DE9F04723
:1064900004468F4E8F4FDFF84092DFF84082002590
:1064A00099F81E50012D01DB082D02DD0020BDE80A
:1064B000F0872020E07299F81E00607407EBC51089
:1064C000B0F87A00C0B14720A0747F20E074FF20AC
:1064D0002075002060754720A0757F20E075FF20A3
:1064E0002076002060764720A0767F20E076FF208F
:1064F00020770020607741E007EBC510B0F900007D
:10650000000EA07407EBC510B0F90000000CE07499
:1065100007EBC5100088000A207507EBC51000784E
:10652000607507EBC510B0F92800000EA07507EBE9
:10653000C510B0F92800000CE07507EBC510008D00
:10654000000A207607EBC51090F82800607607EB6C
:10655000C510B0F95000000EA07607EBC510B0F9D9
:106560005000000CE07607EBC510B0F85000000AB0
:10657000207707EBC51090F850006077B6F87A00E6
:10658000D0B1472004F81E0F7F206070FF20A0705C
:106590000020E070472020717F206071FF20A071F3
:1065A0000020E071472020727F206072FF20A072DF
:1065B0000020E0721E3C2BE0B6F90000000E04F84B
:1065C0001E0FB6F90000000C60703088000AA07041
:1065D0003078E070B6F92800000E2071B6F9280076
:1065E000000C6071308D000AA07196F82800E071EF
:1065F000B6F95000000E2072B6F95000000C60721F
:10660000B6F85000000AA07296F85000E0721E3CE6
:1066100005EB850008EBC000C08B90B1472004F863
:106620002A0F7F206070FF20A0700020E0704720BC
:1066300020717F206071FF20A0710020E0712A3C52
:1066400043E005EB850158F83100F9F7E9FE000E4B
:1066500004F82A0F05EB850158F83100F9F7E0FE40
:10666000000C607005EB850158F83100F9F7D8FE91
:10667000000AA07005EB850158F83100F9F7D0FE4B
:10668000E07005EB850108EBC1018869F9F7C8FEE8
:10669000000E207105EB850108EBC1018869F9F74F
:1066A000BFFE000C607105EB850108EBC101886934
:1066B000F9F7B6FE000AA07105EB850108EBC101F0
:1066C0008869F9F7ADFEE0712A3C0120EFE6000091
:1066D000184300209C430020E2390020984000200D
:1066E0002DE9F04F8BB00446DFF8E4A3F94EFA48E9
:1066F0000A90DFF8E883DFF8E8B3FA480990FA482F
:106700000890FA480790FA480690012500270020D3
:106710000490814603900290012D01DB082D03DDDA
:1067200000200BB0BDE8F08F002720E00BF1240023
:1067300010F8171004980844C0B204900BF114002C
:1067400010F81700484400F0FF090BF1340010F86E
:10675000171003980844C0B203900BF1440010F8DE
:10676000171002980844C0B20290781CC7B2681E85
:10677000B842DBDC002705E0002107F110002154BE
:10678000781CC7B2042FF7DB05EBC50000EB451101
:106790000A9800EB4100807804F8140F0020607024
:1067A000A070E07005EBC50000EB45110A9800EB06
:1067B000410090F84000207100206071A071E071EC
:1067C00005EB850000EB851018F810002072002002
:1067D0006072A072E07205EB850000EB851008EB9B
:1067E000400090F82800207300206073A073E073CD
:1067F00005EB850000EB851018F8100020740020D0
:106800006074A074E07405EB850000EB851008EB64
:10681000400090F82800207500206075A075E07594
:10682000143C0498401C00EBC00101EB40110A9895
:1068300000EB4100B0F84C0018B1032084F82C00A4
:1068400006E00499491CC8B2FCF75AFC84F82C00F5
:1068500009F1010000EB001000EB4001079800EB8C
:106860004100B0F85E0018B1032084F830000CE05D
:1068700009F1010000EB001000EB4001079800EB6C
:10688000410090F8580084F830000398401CC0EB99
:10689000C00000EB8001089800EB4100408F28B158
:1068A000032084F8340084F8380019E00398401C71
:1068B000C0EBC00000EB8001089800EB410090F8AD
:1068C000340084F834000398401CC0EBC00000EB97
:1068D0008001089800EB410090F8360084F83800F9
:1068E00009F1010000EB001000EB4001079800EBFC
:1068F0004100B0F85E0018B1032084F83C000CE0C1
:1069000009F1010000EB001000EB4001079800EBDB
:10691000410090F85A0084F83C00002004F82D0F44
:106920006070A07020716071A07120726072A0729E
:1069300020736073A07320746074A07405EB8500ED
:1069400000EB851008EB400090F82800E074002070
:1069500020756075A07505EB850000EB851008EBD0
:10696000400090F82800E075002020766076A07640
:106970002D3C002705E0002107F148002154781C38
:10698000C7B2202FF7DB05EB850006EBC000C08BFC
:1069900038B1002004F8680F6070A070E070683CA7
:1069A00013E005EB850006EBC000406805909DF8FC
:1069B000140004F8680F9DF8150060709DF816002B
:1069C000A0709DF81700E070683C05EB850006EBB1
:1069D000C000C08B38B1002004F86C0F6070A0704C
:1069E000E0706C3C18E00AEBC511B1F92A00F9F728
:1069F00009FD40490190F9F795FC05909DF81400B8
:106A000004F86C0F9DF8150060709DF81600A070DA
:106A10009DF81700E0706C3C05EB850006EBC000AC
:106A2000C08B38B1002004F8700F6070A070E07067
:106A3000703C18E00AEBC511B1F90200F9F7E2FC6D
:106A40002C490190F9F76EFC05909DF8140004F8AC
:106A5000700F9DF8150060709DF81600A0709DF8ED
:106A60001700E070703C05EB850006EBC000C08BA2
:106A700038B1002004F8740F6070A070E070743CAE
:106A800018E00AEBC511B1F92A00F9F7BBFC194966
:106A90000190F9F747FC05909DF8140004F8740F75
:106AA0009DF8150060709DF81600A0709DF8170005
:106AB000E070743C05EB850006EBC000C08BD8B1DC
:106AC000002004F8780F6070A070E070783C2CE033
:106AD0009C430020984000209C4B0020BC5000208C
:106AE000A0380020E239002040340020363A00204F
:106AF0005C590020CDCCCC3D0AEBC511B1F9520058
:106B0000F9F780FC64490190F9F70CFC05909DF8B9
:106B1000140004F8780F9DF8150060709DF81600B9
:106B2000A0709DF81700E070783C05EB850006EB3F
:106B3000C000C08B50B1762004F87C0F7F206070BD
:106B4000FF20A0700020E0707C3C14E0284600EBA1
:106B5000800006EBC000806905909DF8140004F8E1
:106B60007C0F9DF8150060709DF81600A0709DF8D0
:106B70001700E0707C3C05EB850006EBC000C08B85
:106B800038B1002004F8800F6070A070E070803C85
:106B90000CE005EB850006EBC00080690590002045
:106BA00004F8800F6070A070E070803C05EB8500F9
:106BB00006EBC000C08B38B1002004F8840F607071
:106BC000A070E070843C0CE005EB850006EBC00093
:106BD00080690590002004F8840F6070A070E07058
:106BE000843C05EB850006EBC000C08B38B100206B
:106BF00004F8880F6070A070E070883C0CE005EB32
:106C0000850006EBC00080690590002004F8880F1D
:106C10006070A070E070883C05EB850006EBC0005A
:106C2000C08B38B1002004F88C0F6070A070E07049
:106C30008C3C13E005EB850006EBC00080690590F5
:106C40009DF8140004F88C0F9DF8150060709DF8F5
:106C50001600A0709DF81700E0708C3C05EB8500D5
:106C600006EBC000C08B38B1002004F8900F6070B4
:106C7000A070E070903C0CE005EB850006EBC000D6
:106C800080690590002004F8900F6070A070E0709B
:106C9000903C012045E50000CDCCCC3D78B50246C6
:106CA000FE4B0121002400BF05E0A52504F11000E2
:106CB0001554601CC4B2082CF7DD002412E000203B
:106CC000182505EB84055055192505EB840550550D
:106CD0001A2505EB840550551B2505EB84055055F9
:106CE000601CC4B2082CEADD0121FDE301EB810048
:106CF00003EBC000C08B28B30025481E00EB400604
:106D000006EBC000382606EB80001554481E00EB49
:106D1000400606EBC000392606EB80001554481EDD
:106D200000EB400606EBC0003A2606EB8000155447
:106D3000481E00EB400606EBC0003B2606EB800039
:106D4000155430E001EB810053F8300000909DF8BD
:106D50000050481E00EB400606EBC000382606EB4C
:106D6000800015549DF80150481E00EB400606EBCC
:106D7000C000392606EB800015549DF80250481ECD
:106D800000EB400606EBC0003A2606EB80001554E7
:106D90009DF80350481E00EB400606EBC0003B2662
:106DA00006EB8000155401EB810003EBC000C08BA3
:106DB00028B30025481E00EB400606EBC0003C2629
:106DC00006EB80001554481E00EB400606EBC000A1
:106DD0003D2606EB80001554481E00EB400606EBEE
:106DE000C0003E2606EB80001554481E00EB40060E
:106DF00006EBC0003F2606EB8000155431E001EBA6
:106E0000810003EBC000806800909DF80050481E90
:106E100000EB400606EBC0003C2606EB8000155454
:106E20009DF80150481E00EB400606EBC0003D26D1
:106E300006EB800015549DF80250481E00EB4006FA
:106E400006EBC0003E2606EB800015549DF803506B
:106E5000481E00EB400606EBC0003F2606EB800014
:106E6000155401EB810003EBC000C08B28B3002553
:106E7000481E00EB400606EBC000402606EB8000F3
:106E80001554481E00EB400606EBC000412606EBF9
:106E900080001554481E00EB400606EBC000422659
:106EA00006EB80001554481E00EB400606EBC000C0
:106EB000432606EB8000155431E001EB810003EB23
:106EC000C000C06800909DF80050481E00EB4006CE
:106ED00006EBC000402606EB800015549DF80150DB
:106EE000481E00EB400606EBC000412606EB800082
:106EF00015549DF80250481E00EB400606EBC000FA
:106F0000422606EB800015549DF80350481E00EB06
:106F1000400606EBC000432606EB8000155401EB4B
:106F2000810003EBC000C08B28B30025481E00EB96
:106F3000400606EBC000442606EB80001554481EB0
:106F400000EB400606EBC000452606EB800015541A
:106F5000481E00EB400606EBC000462606EB80000C
:106F60001554481E00EB400606EBC000472606EB12
:106F70008000155431E001EB810003EBC000006993
:106F800000909DF80050481E00EB400606EBC00044
:106F9000442606EB800015549DF80150481E00EB76
:106FA000400606EBC000452606EB800015549DF810
:106FB0000250481E00EB400606EBC000462606EBDA
:106FC000800015549DF80350481E00EB400606EB68
:106FD000C000472606EB8000155401EB810003EB4F
:106FE000C000C08B28B30025481E00EB400606EB0E
:106FF000C000482606EB80001554481E00EB4006F2
:1070000006EBC000492606EB80001554481E00EB35
:10701000400606EBC0004A2606EB80001554481EC9
:1070200000EB400606EBC0004B2606EB8000155433
:1070300031E001EB810003EBC000406900909DF856
:107040000050481E00EB400606EBC000482606EB49
:10705000800015549DF80150481E00EB400606EBD9
:10706000C000492606EB800015549DF80250481ECA
:1070700000EB400606EBC0004A2606EB80001554E4
:107080009DF80350481E00EB400606EBC0004B265F
:1070900006EB8000155401EB810001E098400020D0
:1070A00003EBC000C08B40B37625481E00EB4006C2
:1070B00006EBC0004C2606EB800015547F25481EC9
:1070C00000EB400606EBC0004D2606EB8000155491
:1070D000FF25481E00EB400606EBC0004E2606EBDF
:1070E000800015540025481E00EB400606EBC0004A
:1070F0004F2606EB8000155431E001EB810003EBD5
:10710000C000806900909DF80050481E00EB4006CA
:1071100006EBC0004C2606EB800015549DF801508C
:10712000481E00EB400606EBC0004D2606EB800033
:1071300015549DF80250481E00EB400606EBC000B7
:107140004E2606EB800015549DF80350481E00EBB8
:10715000400606EBC0004F2606EB8000155401EBFD
:10716000810003EBC000C08B40B37625481E00EBC6
:10717000400606EBC000502606EB800015547F2524
:10718000481E00EB400606EBC000512606EB8000CF
:107190001554FF25481E00EB400606EBC0005226A2
:1071A00006EB800015540025481E00EB400606EB58
:1071B000C000532606EB8000155431E001EB81003E
:1071C00003EBC000806900909DF80050481E00EB62
:1071D000400606EBC000502606EB800015549DF8D3
:1071E0000150481E00EB400606EBC000512606EB9E
:1071F000800015549DF80250481E00EB400606EB37
:10720000C000522606EB800015549DF80350481E1E
:1072100000EB400606EBC000532606EB8000155439
:1072200001EB810003EBC000C08B40B37625481E04
:1072300000EB400606EBC000542606EB8000155418
:107240007F25481E00EB400606EBC000552606EBE6
:1072500080001554FF25481E00EB400606EBC000D9
:10726000562606EB800015540025481E00EB40060C
:1072700006EBC000572606EB8000155431E001EB09
:10728000810003EBC000806900909DF80050481E0B
:1072900000EB400606EBC000542606EB80001554B8
:1072A0009DF80150481E00EB400606EBC000552635
:1072B00006EB800015549DF80250481E00EB400676
:1072C00006EBC000562606EB800015549DF80350CF
:1072D000481E00EB400606EBC000572606EB800078
:1072E000155401EB810003EBC000C08B40B3762541
:1072F000481E00EB400606EBC000582606EB800057
:1073000015547F25481E00EB400606EBC0005926A9
:1073100006EB80001554FF25481E00EB400606EBE7
:10732000C0005A2606EB800015540025481E00EBCD
:10733000400606EBC0005B2606EB8000155431E0EA
:1073400001EB810003EBC000806900909DF80050C4
:10735000481E00EB400606EBC000582606EB8000F6
:1073600015549DF80150481E00EB400606EBC00086
:10737000592606EB800015549DF80250481E00EB7C
:10738000400606EBC0005A2606EB800015549DF817
:107390000350481E00EB400606EBC0005B2606EBE0
:1073A0008000155401EB810003EBC000C08B40B39B
:1073B0007625481E00EB400606EBC0005C2606EB77
:1073C000800015547F25481E00EB400606EBC000E8
:1073D0005D2606EB80001554FF25481E00EB400695
:1073E00006EBC0005E2606EB800015540025481E03
:1073F00000EB400606EBC0005F2606EB800015544C
:1074000031E001EB810003EBC000806900909DF842
:107410000050481E00EB400606EBC0005C2606EB61
:10742000800015549DF80150481E00EB400606EB05
:10743000C0005D2606EB800015549DF80250481EE2
:1074400000EB400606EBC0005E2606EB80001554FC
:107450009DF80350481E00EB400606EBC0005F2677
:1074600006EB8000155401EB810003EBC000C08BDC
:1074700040B37625481E00EB400606EBC0006026B0
:1074800006EB800015547F25481E00EB400606EBF6
:10749000C000612606EB80001554FF25481E00EB56
:1074A000400606EBC000622606EB8000155400255E
:1074B000481E00EB400606EBC000632606EB80008A
:1074C000155433E001EB810003EBC00080690090AC
:1074D0009DF80050481E00EB400606EBC0006026F9
:1074E00006EB8000155400E022E09DF80150481E94
:1074F00000EB400606EBC000612606EB8000155449
:107500009DF80250481E00EB400606EBC0006226C4
:1075100006EB800015549DF80350481E00EB400612
:1075200006EBC000632606EB80001554481CC1B270
:1075300004297FF7DBAB012078BD00002DE9F04F77
:107540008BB00446DFF8E4A3F94EFA480A90DFF85E
:10755000E883DFF8E8B3FA480990FA480890FA4857
:107560000790FA48069002250027002004908146E3
:1075700003900290012D01DB082D03DD00200BB0EC
:10758000BDE8F08F002720E00BF1240010F8171061
:1075900004980844C0B204900BF1140010F81700CE
:1075A000484400F0FF090BF1340010F8171003985D
:1075B0000844C0B203900BF1440010F81710029871
:1075C0000844C0B20290781CC7B2681EB842DBDC27
:1075D000002705E0002107F110002154781CC7B2F4
:1075E000042FF7DB05EBC50000EB45110A9800EB13
:1075F0004100807804F8140F00206070A070E070E3
:1076000005EBC50000EB45110A9800EB410090F82E
:107610004000207100206071A071E07105EB8500D1
:1076200000EB851018F81000207200206072A07224
:10763000E07205EB850000EB851008EB400090F848
:107640002800207300206073A073E07305EB8500B1
:1076500000EB851018F81000207400206074A074EE
:10766000E07405EB850000EB851008EB400090F816
:107670002800207500206075A075E075143C049802
:10768000401C00EBC00101EB40110A9800EB4100E7
:10769000B0F84C0018B1032084F82C0006E00499DF
:1076A000491CC8B2FBF72CFD84F82C0009F101003D
:1076B00000EB001000EB4001079800EB4100B0F830
:1076C0005E0018B1032084F830000CE009F10100DD
:1076D00000EB001000EB4001079800EB410090F830
:1076E000580084F830000398401CC0EBC00000EB49
:1076F0008001089800EB4100408F28B1032084F8F6
:10770000340084F8380019E00398401CC0EBC00036
:1077100000EB8001089800EB410090F8340084F8F9
:1077200034000398401CC0EBC00000EB80010898B7
:1077300000EB410090F8360084F8380009F10100B0
:1077400000EB001000EB4001079800EB4100B0F89F
:107750005E0018B1032084F83C000CE009F1010040
:1077600000EB001000EB4001079800EB410090F89F
:107770005A0084F83C00002004F82D0F6070A070BF
:1077800020716071A07120726072A07220736073AA
:10779000A07320746074A07405EB850000EB851065
:1077A00008EB400090F82800E07400202075607518
:1077B000A07505EB850000EB851008EB400090F804
:1077C0002800E075002020766076A0762D3C00270A
:1077D00005E0002107F148002154781CC7B2202F92
:1077E000F7DB05EB850006EBC000C08B38B100204D
:1077F00004F8680F6070A070E070683C13E005EB5F
:10780000850006EBC000406805909DF8140004F860
:10781000680F9DF8150060709DF81600A0709DF827
:107820001700E070683C05EB850006EBC000C08BDC
:1078300038B1002004F86C0F6070A070E0706C3CF0
:1078400018E00AEBC511B1F92A00F8F7DBFD404951
:107850000190F8F767FD05909DF8140004F86C0F8F
:107860009DF8150060709DF81600A0709DF8170037
:10787000E0706C3C05EB850006EBC000C08B38B1B6
:10788000002004F8700F6070A070E070703C18E089
:107890000AEBC511B1F90200F8F7B4FD2C490190CB
:1078A000F8F740FD05909DF8140004F8700F9DF85E
:1078B000150060709DF81600A0709DF81700E0702C
:1078C000703C05EB850006EBC000C08B38B1002092
:1078D00004F8740F6070A070E070743C18E00AEB5C
:1078E000C511B1F92A00F8F78DFD19490190F8F793
:1078F00019FD05909DF8140004F8740F9DF815000B
:1079000060709DF81600A0709DF81700E070743C40
:1079100005EB850006EBC000C08BD8B1002004F851
:10792000780F6070A070E070783C2CE09C430020E1
:10793000984000209C4B0020BC500020A038002024
:10794000E239002040340020363A00205C59002003
:10795000CDCCCC3D0AEBC511B1F95200F8F752FD80
:1079600060490190F8F7DEFC05909DF8140004F8DA
:10797000780F9DF8150060709DF81600A0709DF8B6
:107980001700E070783C05EB850006EBC000C08B6B
:1079900050B1762004F87C0F7F206070FF20A0702B
:1079A0000020E0707C3C14E0284600EB800006EBF1
:1079B000C000806905909DF8140004F87C0F9DF8C4
:1079C000150060709DF81600A0709DF81700E0701B
:1079D0007C3C05EB850006EBC000C08B38B1002075
:1079E00004F8800F6070A070E070803C0CE005EB44
:1079F000850006EBC00080690590002004F8800F28
:107A00006070A070E070803C05EB850006EBC00064
:107A1000C08B38B1002004F8840F6070A070E07053
:107A2000843C0CE005EB850006EBC0008069059006
:107A3000002004F8840F6070A070E070843C05EBB7
:107A4000850006EBC000C08B38B1002004F8880F19
:107A50006070A070E070883C0CE005EB850006EBE0
:107A6000C00080690590002004F8880F6070A07045
:107A7000E070883C05EB850006EBC000C08B38B198
:107A8000002004F88C0F6070A070E0708C3C0CE05B
:107A900005EB850006EBC00080690590002004F826
:107AA0008C0F6070A070E0708C3C05EB850006EBDD
:107AB000C000C08B38B1002004F8900F6070A07037
:107AC000E070903C0CE005EB850006EBC00080699F
:107AD0000590002004F8900F6070A070E070903C5A
:107AE00001204CE5CDCCCC3DF8B50146FD4BFE4E1A
:107AF000FE4C0322002500BF05E0002705F1100021
:107B00000F54681CC5B2042DF7DB02EBC20000EB7A
:107B1000421006EB4000807801F8140F00204870F6
:107B20008870C87002EBC20000EB421006EB400008
:107B300090F840000871002048718871C87102EB0C
:107B4000820000EB821014F81000087200204872C6
:107B50008872C87202EB820000EB821004EB4000D6
:107B600090F828000873002048738873C87302EBEC
:107B7000820000EB821014F8100008740020487492
:107B80008874C87402EB820000EB821004EB4000A2
:107B900090F828000875002048758875C87502EBB4
:107BA000820000EB821014F810000876002048765E
:107BB0008876C87602EB820000EB821004EB40006E
:107BC00090F828000877002048778877C87702EB7C
:107BD000820000EB821014F8100081F820000020D1
:107BE00081F8210081F8220081F8230002EB820055
:107BF00000EB821004EB400090F8280081F824008C
:107C0000002081F8250081F8260081F8270002EB8A
:107C1000820000EB821004EB400090F8280081F80D
:107C20002800002081F8290081F82A0081F82B0023
:107C300002EB820000EB821004EB400090F8280079
:107C400081F82C00002081F82D0081F82E0081F8A9
:107C50002F0002EB820000EB821004EB400090F852
:107C6000280081F83000002081F8310081F83200CE
:107C700081F833001439002505E0002705F148009C
:107C80000F54681CC5B2202DF7DB02EB820003EB1A
:107C9000C000C08B38B1002001F8680F48708870B0
:107CA000C870683912E002EB820053F8300000908F
:107CB0009DF8000001F8680F9DF8010048709DF8DC
:107CC000020088709DF80300C870683902EB8200DA
:107CD00003EBC000C08B38B1002001F86C0F487076
:107CE0008870C8706C3913E002EB820003EBC000AF
:107CF000806800909DF8000001F86C0F9DF801006D
:107D000048709DF8020088709DF80300C8706C39B7
:107D100002EB820003EBC000C08B38B1002001F8F9
:107D2000700F48708870C870703913E002EB8200E1
:107D300003EBC000C06800909DF8000001F8700FD0
:107D40009DF8010048709DF8020088709DF80300BE
:107D5000C870703902EB820003EBC000C08B38B1F1
:107D6000002001F8740F48708870C870743913E0EF
:107D700002EB820003EBC000006900909DF8000058
:107D800001F8740F9DF8010048709DF8020088709A
:107D90009DF80300C870743902EB820003EBC00049
:107DA000C08B38B1002001F8780F48708870C87017
:107DB000783913E002EB820003EBC00040690090C9
:107DC0009DF8000001F8780F9DF8010048709DF8BB
:107DD000020088709DF80300C870783902EB8200B9
:107DE00003EBC000C08B50B1762001F87C0F7F20E0
:107DF0004870FF2088700020C8707C3913E002EBC7
:107E0000820003EBC000806900909DF8000001F83B
:107E10007C0F9DF8010048709DF8020088709DF865
:107E20000300C8707C3902EB820003EBC000C08BFA
:107E300038B1002001F8800F48708870C870803910
:107E40000CE002EB820003EBC00080690090002090
:107E500001F8800F48708870C870803902EB82008A
:107E600003EBC000C08B38B1002001F8840F4870CC
:107E70008870C87084390CE002EB820003EBC0000C
:107E800080690090002001F8840F48708870C870E5
:107E9000843902EB820003EBC000C08B38B10020B4
:107EA00001F8880F48708870C87088390CE002EBC0
:107EB000820003EBC00080690090002001F8880F69
:107EC00048708870C870883902EB820003EBC000EC
:107ED000C08B68B1002001F88C0F48708870C870A2
:107EE0008C3912E0984000209C4B0020BC500020B0
:107EF00002EB820003EBC00080690090002001F8D3
:107F00008C0F48708870C8708C3902EB820003EBCC
:107F1000C000C08B38B1002001F8900F4870887005
:107F2000C87090390CE002EB820003EBC00080695E
:107F30000090002001F8900F48708870C870903948
:107F40000120F8BDF8B50146FD4BFE4EFE4C042263
:107F5000002500BF05E0002705F110000F54681C44
:107F6000C5B2042DF7DB02EBC20000EB421006EBBA
:107F70004000807801F8140F002048708870C870A5
:107F800002EBC20000EB421006EB400090F840000C
:107F90000871002048718871C87102EB820000EB03
:107FA000821014F810000872002048728872C8729B
:107FB00002EB820000EB821004EB400090F82800F6
:107FC0000873002048738873C87302EB820000EBCB
:107FD000821014F810000874002048748874C87463
:107FE00002EB820000EB821004EB400090F82800C6
:107FF0000875002048758875C87502EB820000EB93
:10800000821014F810000876002048768876C8762A
:1080100002EB820000EB821004EB400090F8280095
:108020000877002048778877C87702EB820000EB5A
:10803000821014F8100081F82000002081F821003F
:1080400081F8220081F8230002EB820000EB82100D
:1080500004EB400090F8280081F82400002081F80B
:10806000250081F8260081F8270002EB820000EB52
:10807000821004EB400090F8280081F828000020CE
:1080800081F8290081F82A0081F82B0002EB820098
:1080900000EB821004EB400090F8280081F82C00DF
:1080A000002081F82D0081F82E0081F82F0002EBCE
:1080B000820000EB821004EB400090F8280081F869
:1080C0003000002081F8310081F8320081F833005F
:1080D0001439002505E0002705F148000F54681CFD
:1080E000C5B2202DF7DB02EB820003EBC000C08B92
:1080F00038B1002001F8680F48708870C87068397E
:1081000012E002EB820053F8300000909DF800006E
:1081100001F8680F9DF8010048709DF80200887012
:108120009DF80300C870683902EB820003EBC000C1
:10813000C08B38B1002001F86C0F48708870C8708F
:108140006C3913E002EB820003EBC0008068009002
:108150009DF8000001F86C0F9DF8010048709DF833
:10816000020088709DF80300C8706C3902EB820031
:1081700003EBC000C08B38B1002001F8700F4870CD
:108180008870C870703913E002EB820003EBC00006
:10819000C06800909DF8000001F8700F9DF8010084
:1081A00048709DF8020088709DF80300C87070390F
:1081B00002EB820003EBC000C08B38B1002001F855
:1081C000740F48708870C870743913E002EB820035
:1081D00003EBC000006900909DF8000001F8740FE7
:1081E0009DF8010048709DF8020088709DF803001A
:1081F000C870743902EB820003EBC000C08B38B149
:10820000002001F8780F48708870C870783913E042
:1082100002EB820003EBC000406900909DF8000073
:1082200001F8780F9DF8010048709DF802008870F1
:108230009DF80300C870783902EB820003EBC000A0
:10824000C08B50B1762001F87C0F7F204870FF2052
:1082500088700020C8707C3913E002EB820003EBC9
:10826000C000806900909DF8000001F87C0F9DF827
:10827000010048709DF8020088709DF80300C870E6
:108280007C3902EB820003EBC000C08B38B10020C8
:1082900001F8800F48708870C87080390CE002EBDC
:1082A000820003EBC00080690090002001F8800F7D
:1082B00048708870C870803902EB820003EBC00000
:1082C000C08B38B1002001F8840F48708870C870E6
:1082D00084390CE002EB820003EBC000806900905F
:1082E000002001F8840F48708870C870843902EB50
:1082F000820003EBC000C08B38B1002001F8880F6A
:1083000048708870C87088390CE002EB820003EB7B
:10831000C00080690090002001F8880F48708870C4
:10832000C870883902EB820003EBC000C08B68B1D3
:10833000002001F88C0F48708870C8708C3912E0EA
:10834000984000209C4B0020BC50002002EB820093
:1083500003EBC00080690090002001F88C0F48708A
:108360008870C8708C3902EB820003EBC000C08BB0
:1083700038B1002001F8900F48708870C8709039AB
:108380000CE002EB820003EBC0008069009000204B
:1083900001F8900F48708870C87090390120F8BDBE
:1083A000F8B50146FD4BFE4EFE4C0522002500BFF0
:1083B00005E0002705F110000F54681CC5B2042D1C
:1083C000F7DB02EBC20000EB421006EB40008078C6
:1083D00001F8140F002048708870C87002EBC200CA
:1083E00000EB421006EB400090F8400008710020BE
:1083F00048718871C87102EB820000EB821014F89A
:1084000010000872002048728872C87202EB820065
:1084100000EB821004EB400090F828000873002065
:1084200048738873C87302EB820000EB821014F863
:1084300010000874002048748874C87402EB82002D
:1084400000EB821004EB400090F828000875002033
:1084500048758875C87502EB820000EB821014F82D
:1084600010000876002048768876C87602EB8200F5
:1084700000EB821004EB400090F828000877002001
:1084800048778877C87702EB820000EB821014F8F7
:10849000100081F82000002081F8210081F82200DE
:1084A00081F8230002EB820000EB821004EB400015
:1084B00090F8280081F82400002081F8250081F838
:1084C000260081F8270002EB820000EB821004EB0B
:1084D000400090F8280081F82800002081F8290049
:1084E00081F82A0081F82B0002EB820000EB821059
:1084F00004EB400090F8280081F82C00002081F85F
:108500002D0081F82E0081F82F0002EB820000EB95
:10851000821004EB400090F8280081F83000002021
:1085200081F8310081F8320081F8330014390025D8
:1085300005E0002705F148000F54681CC5B2202D46
:10854000F7DB02EB820003EBC000C08B38B10020E8
:1085500001F8680F48708870C870683912E002EB43
:10856000820053F8300000909DF8000001F8680F79
:108570009DF8010048709DF8020088709DF8030086
:10858000C870683902EB820003EBC000C08B38B1C1
:10859000002001F86C0F48708870C8706C3913E0C7
:1085A00002EB820003EBC000806800909DF80000A1
:1085B00001F86C0F9DF8010048709DF8020088706A
:1085C0009DF80300C8706C3902EB820003EBC00019
:1085D000C08B38B1002001F8700F48708870C870E7
:1085E000703913E002EB820003EBC000C06800901A
:1085F0009DF8000001F8700F9DF8010048709DF88B
:10860000020088709DF80300C870703902EB820088
:1086100003EBC000C08B38B1002001F8740F487024
:108620008870C870743913E002EB820003EBC0005D
:10863000006900909DF8000001F8740F9DF801009A
:1086400048709DF8020088709DF80300C870743966
:1086500002EB820003EBC000C08B38B1002001F8B0
:10866000780F48708870C870783913E002EB820088
:1086700003EBC000406900909DF8000001F8780FFE
:108680009DF8010048709DF8020088709DF8030075
:10869000C870783902EB820003EBC000C08B50B188
:1086A000762001F87C0F7F204870FF208870002022
:1086B000C8707C3913E002EB820003EBC0008069D4
:1086C00000909DF8000001F87C0F9DF801004870B3
:1086D0009DF8020088709DF80300C8707C3902EB99
:1086E000820003EBC000C08B38B1002001F8800F7E
:1086F00048708870C87080390CE002EB820003EB90
:10870000C00080690090002001F8800F48708870D8
:10871000C870803902EB820003EBC000C08B38B117
:10872000002001F8840F48708870C87084390CE00C
:1087300002EB820003EBC00080690090002001F88A
:10874000840F48708870C870843902EB820003EB94
:10875000C000C08B38B1002001F8880F48708870C5
:10876000C87088390CE002EB820003EBC00080691E
:108770000090002001F8880F48708870C870883910
:1087800002EB820003EBC000C08B68B1002001F84F
:108790008C0F48708870C8708C3912E098400020A7
:1087A0009C4B0020BC50002002EB820003EBC00079
:1087B00080690090002001F88C0F48708870C870A4
:1087C0008C3902EB820003EBC000C08B38B1002073
:1087D00001F8900F48708870C87090390CE002EB77
:1087E000820003EBC00080690090002001F8900F28
:1087F00048708870C87090390120F8BDF8B50146FE
:10880000FD4BFE4EFE4C0622002500BF05E0002772
:1088100005F110000F54681CC5B2042DF7DB02EB04
:10882000C20000EB421006EB4000807801F8140F04
:10883000002048708870C87002EBC20000EB421044
:1088400006EB400090F840000871002048718871E4
:10885000C87102EB820000EB821014F8100008725D
:10886000002048728872C87202EB820000EB82100E
:1088700004EB400090F828000873002048738873C8
:10888000C87302EB820000EB821014F81000087429
:10889000002048748874C87402EB820000EB8210D8
:1088A00004EB400090F82800087500204875887592
:1088B000C87502EB820000EB821014F810000876F5
:1088C000002048768876C87602EB820000EB8210A2
:1088D00004EB400090F8280008770020487788775C
:1088E000C87702EB820000EB821014F8100081F8C8
:1088F0002000002081F8210081F8220081F8230067
:1089000002EB820000EB821004EB400090F828009C
:1089100081F82400002081F8250081F8260081F8E4
:10892000270002EB820000EB821004EB400090F87D
:10893000280081F82800002081F8290081F82A0009
:1089400081F82B0002EB820000EB821004EB400068
:1089500090F8280081F82C00002081F82D0081F883
:108960002E0081F82F0002EB820000EB821004EB56
:10897000400090F8280081F83000002081F8310094
:1089800081F8320081F833001439002505E0002712
:1089900005F148000F54681CC5B2202DF7DB02EB2F
:1089A000820003EBC000C08B38B1002001F8680FD3
:1089B00048708870C870683912E002EB820053F882
:1089C000300000909DF8000001F8680F9DF801004C
:1089D00048709DF8020088709DF80300C8706839DF
:1089E00002EB820003EBC000C08B38B1002001F81D
:1089F0006C0F48708870C8706C3913E002EB82000D
:108A000003EBC000806800909DF8000001F86C0F37
:108A10009DF8010048709DF8020088709DF80300E1
:108A2000C8706C3902EB820003EBC000C08B38B118
:108A3000002001F8700F48708870C870703913E01A
:108A400002EB820003EBC000C06800909DF80000BC
:108A500001F8700F9DF8010048709DF802008870C1
:108A60009DF80300C870703902EB820003EBC00070
:108A7000C08B38B1002001F8740F48708870C8703E
:108A8000743913E002EB820003EBC0000069009030
:108A90009DF8000001F8740F9DF8010048709DF8E2
:108AA000020088709DF80300C870743902EB8200E0
:108AB00003EBC000C08B38B1002001F8780F48707C
:108AC0008870C870783913E002EB820003EBC000B5
:108AD000406900909DF8000001F8780F9DF80100B2
:108AE00048709DF8020088709DF80300C8707839BE
:108AF00002EB820003EBC000C08B50B1762001F87E
:108B00007C0F7F204870FF2088700020C8707C395F
:108B100013E002EB820003EBC000806900909DF837
:108B2000000001F87C0F9DF8010048709DF80200DC
:108B300088709DF80300C8707C3902EB820003EB5B
:108B4000C000C08B38B1002001F8800F48708870D9
:108B5000C87080390CE002EB820003EBC000806932
:108B60000090002001F8800F48708870C87080392C
:108B700002EB820003EBC000C08B38B1002001F88B
:108B8000840F48708870C87084390CE002EB820052
:108B900003EBC00080690090002001F8840F48704A
:108BA0008870C870843902EB820003EBC000C08B70
:108BB00038B1002001F8880F48708870C870883973
:108BC0000CE002EB820003EBC00080690090002003
:108BD00001F8880F48708870C870883902EB8200ED
:108BE00003EBC000C08B68B1002001F88C0F487007
:108BF0008870C8708C3912E0984000209C4B00208F
:108C0000BC50002002EB820003EBC00080690090A2
:108C1000002001F88C0F48708870C8708C3902EB06
:108C2000820003EBC000C08B38B1002001F8900F28
:108C300048708870C87090390CE002EB820003EB3A
:108C4000C00080690090002001F8900F4870887083
:108C5000C87090390120F8BDF8B50146FD4BFE4EB5
:108C6000FE4C0722002500BF05E0002705F110009B
:108C70000F54681CC5B2042DF7DB02EBC20000EBF9
:108C8000421006EB4000807801F8140F0020487075
:108C90008870C87002EBC20000EB421006EB400087
:108CA00090F840000871002048718871C87102EB8B
:108CB000820000EB821014F8100008720020487245
:108CC0008872C87202EB820000EB821004EB400055
:108CD00090F828000873002048738873C87302EB6B
:108CE000820000EB821014F8100008740020487411
:108CF0008874C87402EB820000EB821004EB400021
:108D000090F828000875002048758875C87502EB32
:108D1000820000EB821014F81000087600204876DC
:108D20008876C87602EB820000EB821004EB4000EC
:108D300090F828000877002048778877C87702EBFA
:108D4000820000EB821014F8100081F8200000204F
:108D500081F8210081F8220081F8230002EB8200D3
:108D600000EB821004EB400090F8280081F824000A
:108D7000002081F8250081F8260081F8270002EB09
:108D8000820000EB821004EB400090F8280081F88C
:108D90002800002081F8290081F82A0081F82B00A2
:108DA00002EB820000EB821004EB400090F82800F8
:108DB00081F82C00002081F82D0081F82E0081F828
:108DC0002F0002EB820000EB821004EB400090F8D1
:108DD000280081F83000002081F8310081F832004D
:108DE00081F833001439002505E0002705F148001B
:108DF0000F54681CC5B2202DF7DB02EB820003EB99
:108E0000C000C08B38B1002001F8680F487088702E
:108E1000C870683912E002EB820053F8300000900D
:108E20009DF8000001F8680F9DF8010048709DF85A
:108E3000020088709DF80300C870683902EB820058
:108E400003EBC000C08B38B1002001F86C0F4870F4
:108E50008870C8706C3913E002EB820003EBC0002D
:108E6000806800909DF8000001F86C0F9DF80100EB
:108E700048709DF8020088709DF80300C8706C3936
:108E800002EB820003EBC000C08B38B1002001F878
:108E9000700F48708870C870703913E002EB820060
:108EA00003EBC000C06800909DF8000001F8700F4F
:108EB0009DF8010048709DF8020088709DF803003D
:108EC000C870703902EB820003EBC000C08B38B170
:108ED000002001F8740F48708870C870743913E06E
:108EE00002EB820003EBC000006900909DF80000D7
:108EF00001F8740F9DF8010048709DF80200887019
:108F00009DF80300C870743902EB820003EBC000C7
:108F1000C08B38B1002001F8780F48708870C87095
:108F2000783913E002EB820003EBC0004069009047
:108F30009DF8000001F8780F9DF8010048709DF839
:108F4000020088709DF80300C870783902EB820037
:108F500003EBC000C08B50B1762001F87C0F7F205E
:108F60004870FF2088700020C8707C3913E002EB45
:108F7000820003EBC000806900909DF8000001F8BA
:108F80007C0F9DF8010048709DF8020088709DF8E4
:108F90000300C8707C3902EB820003EBC000C08B79
:108FA00038B1002001F8800F48708870C87080398F
:108FB0000CE002EB820003EBC0008069009000200F
:108FC00001F8800F48708870C870803902EB820009
:108FD00003EBC000C08B38B1002001F8840F48704B
:108FE0008870C87084390CE002EB820003EBC0008B
:108FF00080690090002001F8840F48708870C87064
:10900000843902EB820003EBC000C08B38B1002032
:1090100001F8880F48708870C87088390CE002EB3E
:10902000820003EBC00080690090002001F8880FE7
:1090300048708870C870883902EB820003EBC0006A
:10904000C08B68B1002001F88C0F48708870C87020
:109050008C3912E0984000209C4B0020BC5000202E
:1090600002EB820003EBC00080690090002001F851
:109070008C0F48708870C8708C3902EB820003EB4B
:10908000C000C08B38B1002001F8900F4870887084
:10909000C87090390CE002EB820003EBC0008069DD
:1090A0000090002001F8900F48708870C8709039C7
:1090B0000120F8BDF8B50146FD4BFE4EFE4C0822DE
:1090C000002500BF05E0002705F110000F54681CC3
:1090D000C5B2042DF7DB02EBC20000EB421006EB39
:1090E0004000807801F8140F002048708870C87024
:1090F00002EBC20000EB421006EB400090F840008B
:109100000871002048718871C87102EB820000EB81
:10911000821014F810000872002048728872C87219
:1091200002EB820000EB821004EB400090F8280074
:109130000873002048738873C87302EB820000EB49
:10914000821014F810000874002048748874C874E1
:1091500002EB820000EB821004EB400090F8280044
:109160000875002048758875C87502EB820000EB11
:10917000821014F810000876002048768876C876A9
:1091800002EB820000EB821004EB400090F8280014
:109190000877002048778877C87702EB820000EBD9
:1091A000821014F8100081F82000002081F82100BE
:1091B00081F8220081F8230002EB820000EB82108C
:1091C00004EB400090F8280081F82400002081F88A
:1091D000250081F8260081F8270002EB820000EBD1
:1091E000821004EB400090F8280081F8280000204D
:1091F00081F8290081F82A0081F82B0002EB820017
:1092000000EB821004EB400090F8280081F82C005D
:10921000002081F82D0081F82E0081F82F0002EB4C
:10922000820000EB821004EB400090F8280081F8E7
:109230003000002081F8310081F8320081F83300DD
:109240001439002505E0002705F148000F54681C7B
:10925000C5B2202DF7DB02EB820003EBC000C08B10
:1092600038B1002001F8680F48708870C8706839FC
:1092700012E002EB820053F8300000909DF80000ED
:1092800001F8680F9DF8010048709DF80200887091
:109290009DF80300C870683902EB820003EBC00040
:1092A000C08B38B1002001F86C0F48708870C8700E
:1092B0006C3913E002EB820003EBC0008068009081
:1092C0009DF8000001F86C0F9DF8010048709DF8B2
:1092D000020088709DF80300C8706C3902EB8200B0
:1092E00003EBC000C08B38B1002001F8700F48704C
:1092F0008870C870703913E002EB820003EBC00085
:10930000C06800909DF8000001F8700F9DF8010002
:1093100048709DF8020088709DF80300C87070398D
:1093200002EB820003EBC000C08B38B1002001F8D3
:10933000740F48708870C870743913E002EB8200B3
:1093400003EBC000006900909DF8000001F8740F65
:109350009DF8010048709DF8020088709DF8030098
:10936000C870743902EB820003EBC000C08B38B1C7
:10937000002001F8780F48708870C870783913E0C1
:1093800002EB820003EBC000406900909DF80000F2
:1093900001F8780F9DF8010048709DF80200887070
:1093A0009DF80300C870783902EB820003EBC0001F
:1093B000C08B50B1762001F87C0F7F204870FF20D1
:1093C00088700020C8707C3913E002EB820003EB48
:1093D000C000806900909DF8000001F87C0F9DF8A6
:1093E000010048709DF8020088709DF80300C87065
:1093F0007C3902EB820003EBC000C08B38B1002047
:1094000001F8800F48708870C87080390CE002EB5A
:10941000820003EBC00080690090002001F8800FFB
:1094200048708870C870803902EB820003EBC0007E
:10943000C08B38B1002001F8840F48708870C87064
:1094400084390CE002EB820003EBC00080690090DD
:10945000002001F8840F48708870C870843902EBCE
:10946000820003EBC000C08B38B1002001F8880FE8
:1094700048708870C87088390CE002EB820003EBFA
:10948000C00080690090002001F8880F4870887043
:10949000C870883902EB820003EBC000C08B68B152
:1094A000002001F88C0F48708870C8708C3912E069
:1094B000984000209C4B0020BC50002002EB820012
:1094C00003EBC00080690090002001F88C0F487009
:1094D0008870C8708C3902EB820003EBC000C08B2F
:1094E00038B1002001F8900F48708870C87090392A
:1094F0000CE002EB820003EBC000806900900020CA
:1095000001F8900F48708870C87090390120F8BD3C
:109510002DE9F04F87B00446FD480690DFF8F4834C
:10952000FD480590DFF8F493FD4EFE480490FE4898
:1095300003904FF0000A0025002700200290834688
:109540000190059890F81EB0BBF1010F02DBBBF152
:10955000080F03DD002007B0BDE8F08F0020019068
:1095600022E008F12400019910F81100504400F0A5
:10957000FF0A08F11400019910F811002844C5B23F
:1095800008F13400019910F811003844C7B208F10D
:109590004400019910F8111002980844C0B20290DA
:1095A0000198401CC0B20190ABF1010001998842C2
:1095B000D7DC2820E0720598807F60740AF10100F2
:1095C00000EBC00101EB4011049800EB4100B0F842
:1095D0004C0010B10320A07405E00AF10101C8B2EB
:1095E000F9F78EFDA074681C00EB001000EB400042
:1095F00006EB4000B0F85E0010B10320E07409E013
:10960000681C00EB001000EB400006EB400090F8F7
:109610005800E074FAF74AFDC4490860781CC0EBB2
:10962000C00000EB800009EB4000408F18B1032020
:109630002075607513E0781CC0EBC00000EB800063
:1096400009EB400090F834002075781CC0EBC00096
:1096500000EB800009EB400090F836006075681C54
:1096600000EB001000EB400006EB4000B0F85E009D
:1096700010B10320A07509E0681C00EB001000EB9E
:10968000400006EB400090F85A00A0750298401C7C
:1096900000EB800101EB8011069800EB4100B0F86F
:1096A000840010B10320E0750BE00298401C00EB31
:1096B000800101EB8011069800EB410090F87E00DC
:1096C000E075039890F8F20020760AF1010000EBB3
:1096D000C00101EB4011049800EB4100B0F84C00D0
:1096E00060B10AF1010000EBC00101EB40110498E8
:1096F00000EB410090F8220060760BE00AF10100D7
:1097000000EBC00101EB4011049800EB410090F820
:1097100022006076A520A076E076ABF1010008F18A
:10972000240131F81000012815DD0AF1020000EBD8
:10973000C00101EB4011049800EB4100B0F84C006F
:1097400010B10320207708E00AF10201C8B2F9F74E
:10975000D7FC207701E0A5202077A81C00EB0010A3
:1097600000EB400006EB4000B0F85E0020B10320A3
:10977000607784F8200014E0A81C00EB001000EBD8
:10978000400006EB400090F858006077A81C00EB02
:10979000001000EB400006EB400090F85A0084F8FF
:1097A0002000ABF1010008F1340131F8100001286C
:1097B00021DDB81CC0EBC00000EB800009EB4000CD
:1097C000408F18B10320A077E07717E0B81CC0EBFA
:1097D000C00000EB800009EB400090F83400A07757
:1097E000B81CC0EBC00000EB800009EB400090F813
:1097F0003600E07702E0A520A077E077A52004F806
:10980000210F6070A070E0702071213CABF101006D
:1098100008F1240131F81000022817DD0AF10300D5
:1098200000EBC00101EB4011049800EB4100B0F8DF
:109830004C0018B1032084F826000AE00AF1030165
:10984000C8B2F9F75DFC84F8260002E0A52084F890
:109850002600ABF1010008F1140131F810000228D4
:1098600026DDE81C00EB001000EB400006EB40009A
:10987000B0F85E0028B1032084F8270084F82A009D
:109880001BE0E81C00EB001000EB400006EB400082
:1098900090F8580084F82700E81C00EB001000EB5B
:1098A000400006EB400090F85A0084F82A0004E0DB
:1098B000A52084F8270084F82A00ABF1010008F104
:1098C000340131F81000022837DDF81CC0EBC0006D
:1098D00000EB800009EB4000408F28B1032084F8A2
:1098E000280084F829002DE0F81CC0EBC00000EB34
:1098F000800009EB400090F8340084F82800F81C40
:10990000C0EBC00000EB800009EB400010E000005D
:10991000BC500020A0380020E23900204034002054
:10992000363A00209C4B00205C5900205403002054
:1099300090F8360084F8290004E0A52084F8280077
:1099400084F82900A52004F82B0F6070A070E07047
:1099500020712B3CABF1010008F1240131F810001B
:10996000032817DD0AF1040000EBC00101EB4011F0
:10997000049800EB4100B0F84C0018B1032084F8C3
:1099800030000AE00AF10401C8B2F9F7B9FB84F823
:10999000300002E0A52084F83000ABF1010008F1AE
:1099A000140131F81000032825DD281D00EB0010FC
:1099B00000EB400006EB4000B0F85E0020B1032051
:1099C00084F8310084F83400281D00EB001000EB0F
:1099D000400006EB400090F8580084F83100281D44
:1099E00000EB001000EB400006EB400090F85A003E
:1099F00084F8340004E0A52084F8310084F83400B1
:109A0000ABF1010008F1340131F81000042825DD24
:109A1000381DC0EBC00000EB800009EB4000408F18
:109A200028B1032084F8320084F833001BE0381D8D
:109A3000C0EBC00000EB800009EB400090F8340060
:109A400084F83200381DC0EBC00000EB800009EB49
:109A5000400090F8360084F8330004E0A52084F834
:109A6000320084F83300A52004F8350F6070A07030
:109A7000E0702071353C10480068B0F5005F18D2E6
:109A80000020153404F8010C207060706070A07024
:109A90006072A072E072E0722073E07420756075ED
:109AA0006075A0756077A077E077E07784F8200094
:109AB000153C01204FE50000540300202DE9F04142
:109AC0000446934D934EDFF85082944FB87F502850
:109AD0003BDDB87F5F2838DA607C503800EB8000CF
:109AE00008EBC000C08B40B14720A0747F20E07419
:109AF000FF2020750020607507E1617C503901EB83
:109B0000810158F83100F6F78BFC000EA074617CDF
:109B1000503901EB810158F83100F6F781FC000C57
:109B2000E074617C503901EB810158F83100F6F79F
:109B300077FC000A2075617C503901EB810158F8EF
:109B40003100F6F76DFC6075DFE0B87F60287DDDE1
:109B5000B87F6F287ADA607C603806EBC010B0F806
:109B60007A00B8B14720A0747F20E074FF202075F0
:109B7000002060754720A0757F20E075FF202076CB
:109B8000002060764720A0767F20E076FF202077B7
:109B900000206077607C603806EBC010B0F90000F0
:109BA000000EA074607C603806EBC010B0F90000B5
:109BB000000CE074607C603806EBC0100088000A7E
:109BC0002075607C603806EBC01000786075607CA2
:109BD000603806EBC010B0F92800000EA075607C5C
:109BE000603806EBC010B0F92800000CE075607C0E
:109BF000603806EBC010008D000A2076607C60386B
:109C000006EBC01090F828006076607C603806EBA8
:109C1000C010B0F95000000EA076607C603806EBF2
:109C2000C010B0F95000000CE076607C603806EBA4
:109C3000C010B0F85000000A2077607C603806EB56
:109C4000C01090F8500060775FE0FFE7B87F7028A1
:109C500002DDB87F7F2858DBB87F802802DDB87F1F
:109C60008F2852DBB87FE02849DDB87FE32846DA49
:109C7000B5F87A00C0B14720A0747F20E074FF20BF
:109C80002075002060754720A0757F20E075FF20BB
:109C90002076002060764720A0767F20E076FF20A7
:109CA00020770020607730E0B5F90000000EA07446
:109CB000B5F90000000CE0742888000A20752878A7
:109CC0006075B5F92800000EA074B5F92800000CE5
:109CD000E074288D000A207595F828006075B5F9A4
:109CE0005000000EA074B5F95000000CE074B5F8F7
:109CF0005000000A207595F85000607505E0B87FA7
:109D0000E42802D00020BDE8F0810120FBE700003C
:109D1000184300209C43002098400020E239002096
:109D2000F8B50446264D0026B5F90000F6F76AFBA3
:109D300007462449F6F7F6FA00909DF800002074D3
:109D40009DF8010060749DF80200A0749DF8030066
:109D5000E074B5F92800F6F755FB07461949F6F700
:109D6000E1FA00909DF8000020759DF801006075F3
:109D70009DF80200A0759DF80300E075B5F950004C
:109D8000F6F740FB07460F49F6F7CCFA00909DF82E
:109D9000000020769DF8010060769DF80200A07614
:109DA0009DF80300E07600BF05E0A52106F11C0048
:109DB0002154701CC6B2E42EF7DB0120F8BD000070
:109DC000184300200000B43B72B621E0012080F36C
:109DD000138800BF00BF00BF00BF00BF00BFBFF3BC
:109DE0004F8F00BF00BF00BF0A48006800F4E0606A
:109DF00009490843001D0749086000BF00BF00BFB4
:109E0000BFF34F8F00BF00BF00BF00BF00BFFDE723
:109E1000DCE700000CED00E00000FA052DE9FC5F36
:109E20000446DFF8F4A1DFF8F491DFF8F4B1002084
:109E3000019000908046002500260027AA2020706F
:109E400000206070A120A0701120E070002020711F
:109E500000BFCDE07806050E0021681D2154A81D25
:109E600021544AE0701C4044C0EBC00000EB80006D
:109E700009EB4000408F30B1681D205C40F01001BC
:109E8000681D21540FE0701C4044C0EBC00000EB83
:109E9000800009EB4000808E28B1681D205C40F0F6
:109EA0000101681D2154BAF80A0000B3701C404437
:109EB000C0EBC00000EB800009EB4000C08F30B168
:109EC000681D205C40F02001681D21540FE0701CCB
:109ED0004044C0EBC00000EB800009EB4000C08EA6
:109EE00028B1681D205C40F00201681D2154701CDF
:109EF000C6B208F1010000F0FF080AF1340030F8A2
:109F00001700B042AEDC00263CE0701C284400EB99
:109F1000001000EB40000BEB4000B0F85E0060B1B9
:109F2000681D205C40F08001681D2154A81D205C44
:109F300040F05501A81D21541EE0701C284400EB80
:109F4000001000EB40000BEB4000B0F8580028B1C7
:109F5000681D205C40F00801681D2154701C2844D5
:109F600000EB001000EB40000BEB4000B0F85A0093
:109F700010B10121A81D2154701CC6B20098401CCC
:109F8000C0B20090022EC0DB002628E0711C019AAE
:109F90001144C8B2F9F7B4F8012806D1681D205C55
:109FA00040F00401681D215413E0711C019A114412
:109FB000C8B2F9F7A5F830B9681D205C20F004019B
:109FC000681D215405E0681D205C00F04001681DFB
:109FD0002154701CC6B20198401CC0B201900AF115
:109FE000240030F81700B042D0DC0026781CC7B23D
:109FF000082FFFF62FAF0B480068B0F5005F08D2BE
:10A00000002704E00021781D2154781CC7B2102FCE
:10A01000F8DBBDE8FC9F0000A038002040340020A1
:10A02000363A002054030020F0B585B004461B4E9C
:10A030001B4F1C4D14216846F6F711F9A97F687F64
:10A0400041EA0020ADF80000287D062804D1012255
:10A0500015496846F7F798FB012213496846F7F758
:10A060007DFBBDF80000A6F84000BDF80000A7F891
:10A070006000BDF8000000122074BDF8000060749C
:10A08000217C687F814206D1617CA87F814202D118
:10A09000012005B0F0BD0020FBE7000040340020A7
:10A0A000363A0020E239002064F0070800BF0120A2
:10A0B00003F0AEFCFBE7000008B50027B94600BF7F
:10A0C0000025AB46DFF8F4A3FD480090FD4CDFF817
:10A0D000F883FE4E0020FE4908800DE008F11400D0
:10A0E000FB49098830F8110058441FFA80FBF848F2
:10A0F0000088401CF6490880B8F80000F449098837
:10A100008842EBDC0020F249088000BF1E2003F0EB
:10A110007FFC4FF48061EF48F9F7B8FFEE48007814
:10A12000E0B14FF0000B0020E94908800DE008F194
:10A130001400E749098830F8110058441FFA80FBE1
:10A14000E3480088401CE2490880B8F80000E04974
:10A1500009888842EBDC0020DF49087000984088BD
:10A16000002871D1002F72D1B8F8100000286DD0EE
:10A170000621DA48FBF716FC05462812D7498871F4
:10A18000CD7100224FF48051D548F9F789FF502056
:10A1900003F0FAF864230822D049D248FBF74AF9C1
:10A1A000502003F0F1F801221103CD48F9F778FFB0
:10A1B000CA480078103800EB001000EB400004EBB8
:10A1C0004000B0F86400052817DD3C21C348007842
:10A1D000103800EB001000EB400004EB4000A0F84A
:10A1E0006410BE480078103800EB001000EB40000F
:10A1F00004EB4000A0F85C1017E0B8480078103875
:10A2000000EB001000EB400004EB4000B0F86400ED
:10A21000401C81B2B1480078103800EB001000EB10
:10A22000400004EB4000A0F86410AC4800781038FF
:10A23000082805DAA9480078401CA849087006E0FB
:10A240001120A649087002E0D5E0FFE70327B8F81F
:10A250006C0050B3032F2ED10621A348FBF7A2FBBD
:10A2600005462812A0498871CD7100224FF4805113
:10A270009B48F9F715FF502003F086F86423082265
:10A2800099499848FBF7D6F8502003F07DF8012251
:10A2900011039348F9F704FFB6F87E003C2805DD6A
:10A2A0003C20A6F87E00A6F8780004E0B6F87E0010
:10A2B000401CA6F87E00062F1FD106218B48FBF715
:10A2C00071FB0546281289498871CD7100224FF42F
:10A2D00080518348F9F7E4FE502003F055F86423D9
:10A2E000082282497F48FBF7A5F8502003F04CF87C
:10A2F000012211037A48F9F7D3FE092F58D1B8F893
:10A300001200002853D00E217948FBF74BFB05467D
:10A31000281277498873CD7300224FF4805170481A
:10A32000F9F7BEFE502003F02FF864231022704985
:10A330006C48FBF77FF8502003F026F80122110348
:10A340006748F9F7ADFE6A480078203800EBC00195
:10A3500001EB40100AEB4000B0F85000322817DC47
:10A3600063480078203800EBC00101EB40100AEB95
:10A370004000B0F85000401C81B25D4800782038A1
:10A3800000EBC00202EB40100AEB4000A0F85010B6
:10A39000574800782138032805DA55480078401CD2
:10A3A0005349087004E021205149087000E0142747
:10A3B0000C2F1FD106214F48FBF7F4FA054628124F
:10A3C0004C498871CD7100224FF480514448F9F70F
:10A3D00067FE502002F0D8FF642308224549414817
:10A3E000FBF728F8502002F0CFFF012211033C4870
:10A3F000F9F756FE8CE0B9F1030F26D100224FF495
:10A4000080513748F9F74CFE502002F0BDFF3A4822
:10A4100000780D280AD1384800780A2806D164232C
:10A420000C2235492F48FBF705F805E06423082284
:10A4300031492C48FAF7FEFF502002F0A5FF012217
:10A4400011032748F9F72CFE5EE0B9F1060F17D18A
:10A4500000224FF480512248F9F722FE502002F0EA
:10A4600093FF6423102225491E48FAF7E3FF50208A
:10A4700002F08AFF012211031948F9F711FE43E0A7
:10A48000B9F1090F40D100224FF480511448F9F777
:10A4900007FE502002F078FF64231948028817490C
:10A4A0001048FAF7C7FF502002F06EFF0122110397
:10A4B0000B48F9F7F5FD0021009823E09C4B0020A4
:10A4C000E2390020363A0020A0380020184300204E
:10A4D0001003002000100140F8020020900100202D
:10A4E000000C0140100C0020D2010020DA010020F5
:10A4F0009A010020CA010020563900209C39002012
:10A50000DA0900204180894609F1010000F0FF09C5
:10A51000F948006801287DD1F848007811280ED04C
:10A52000B4F8C200401CA4F8C200B4F8C2009628D7
:10A5300005DD9621A4F8C2100121A4F8C410EF484B
:10A54000007812280ED0B4F82801401CA4F8280185
:10A55000B4F82801962805DD9621A4F828110121D8
:10A56000A4F82A11E548007813280ED0B4F88E011B
:10A57000401CA4F88E01B4F88E01962805DD9621C2
:10A58000A4F88E110121A4F89011DC480078142859
:10A590000ED0B4F8F401401CA4F8F401B4F8F401AE
:10A5A000962805DD9621A4F8F4110121A4F8F611EE
:10A5B000D248007815280ED0B4F85A02401CA4F8EE
:10A5C0005A02B4F85A02962805DD9621A4F85A12C8
:10A5D0000121A4F85C12C948007816280ED0B4F8FE
:10A5E000C002401CA4F8C002B4F8C002962805DDE1
:10A5F0009621A4F8C0120121A4F8C212BF48007825
:10A60000172810D0B4F82603401CA4F82603B4F889
:10A61000260300E09CE1962805DD9621A4F8261388
:10A620000121A4F82813B548007818280ED0B4F8F2
:10A630008C03401CA4F88C03B4F88C03962805DD29
:10A640009621A4F88C130121A4F88E13AB4800784E
:10A65000112803D1B4F8C210A4F8C210A74800789A
:10A66000122803D1B4F82811A4F82811A3480078BF
:10A67000132803D1B4F88E11A4F88E119F480078E6
:10A68000142803D1B4F8F411A4F8F4119B4800780D
:10A69000152803D1B4F85A12A4F85A129748007832
:10A6A000162803D1B4F8C012A4F8C0129348007859
:10A6B000172803D1B4F82613A4F826138F4800787E
:10A6C000182803D1B4F88C13A4F88C138B480078A5
:10A6D00010287DDB894800781F2879DC874840797D
:10A6E00005028648807905430121844800781038A6
:10A6F00000EB001000EB400004EB4000A0F86410F9
:10A700007E484078032807D07C484078062803D04C
:10A7100001207B49088010E078488078022803D027
:10A7200001207749088008E005217448FBF73AF9D1
:10A73000A84202D001207249088071480088002890
:10A740006CD100216D480078103800EB001000EB50
:10A75000400004EB4000A0F85C1068480078103816
:10A7600000EB001000EB400004EB4000A0F85E108E
:10A7700062484078032852D16048C078012815DD2E
:10A780006048008800EB001000EB400004EB400044
:10A79000B0F85C00401C5B49098801EB011101EB3A
:10A7A000410104EB4101A1F85C002AE05548008812
:10A7B000142826DA00205349098801EB011101EB26
:10A7C000410104EB4101A1F85C004C48C17800E074
:10A7D00026E00078103800EB001000EB400024F871
:10A7E0001010464801790078103800EB001000EB9B
:10A7F000400004EB4000018542480088401C41496C
:10A80000088040480088142802D100203D49088073
:10A810003A490978103988B202F0CAFA92E091E018
:10A8200036480078702871DB344800787F286DDC6A
:10A830003248C07905023148007A05430120A6F864
:10A840007E002E484078032807D02C484078062800
:10A8500003D001202A4908800DE028488078082884
:10A8600003DB01202649088005E024488078C11CCC
:10A870002248FBF797F822480088D8BB1F48407849
:10A8800003285FD12048008814282CDA0020A6F87D
:10A8900078001A4800791949C97840EA012000B2C5
:10A8A0001949098826F81100144880791349497913
:10A8B00040EA012001B206F12800134A128820F86C
:10A8C00012100E48007A0D49C97940EA012001B200
:10A8D00006F150000C4A128820F812100A4800882D
:10A8E000401C094908800848008814282AD1002003
:10A8F0000549088026E009E04C030020002B0020D9
:10A900001403002010030020120300205048007898
:10A91000202806DB4E4800782F2802DCF8F750FC90
:10A9200010E04B480078E42802D1F8F7F9FB09E081
:10A9300047480078812805DB454800788F2801DCEE
:10A94000F8F78AFB0020434908804349086077E014
:10A95000B4F8C200401CA4F8C200B4F8C2009628A3
:10A9600005DD9621A4F8C2100121A4F8C410B4F8A2
:10A970002801401CA4F82801B4F82801962805DD18
:10A980009621A4F828110121A4F82A11B4F88E0107
:10A99000401CA4F88E01B4F88E01962805DD96219E
:10A9A000A4F88E110121A4F89011B4F8F401401C10
:10A9B000A4F8F401B4F8F401962805DD9621A4F872
:10A9C000F4110121A4F8F611B4F85A02401CA4F8BD
:10A9D0005A02B4F85A02962805DD9621A4F85A12B4
:10A9E0000121A4F85C12B4F8C002401CA4F8C00213
:10A9F000B4F8C002962805DD9621A4F8C012012102
:10AA0000A4F8C212B4F82603401CA4F82603B4F834
:10AA10002603962805DD9621A4F826130121A4F823
:10AA20002813B4F88C03401CA4F88C03B4F88C03EE
:10AA3000962805DD9621A4F88C130121A4F88E1325
:10AA4000022F03DA781CC7B2FFF760BB0027FBE7D1
:10AA5000002B0020140300204C03002086B04FF090
:10AA6000000A00BFD346002005900025DFF8F493CC
:10AA7000FD480390FD4CFE4EFE4FDFF8FC830020A6
:10AA8000FE49088011E006F13400FC49098830F8DD
:10AA9000110050441FFA80FA0BF101001FFA80FBED
:10AAA000F6480088401CF54908803088F349098839
:10AAB0008842E8DCB6F86400FF2141EA202030B982
:10AAC000B6F8660041EA202000B900E000BF00208F
:10AAD000EA49088000BF322002F09AFF4FF48061FB
:10AAE000E748F9F7D3FAE748007860B34FF0000A77
:10AAF0000020E249088011E006F13400DF490988AE
:10AB000030F8110050441FFA80FA0BF101001FFACF
:10AB100080FBDA480088401CD84908803088D74933
:10AB200009888842E8DCB6F86400FF2141EA202069
:10AB300030B9B6F8660041EA202000B900E000BF55
:10AB40000020D04908700398008800287BD1CE48A7
:10AB50000078002876D101203081B089002873D098
:10AB60000621CA48FAF71EFFC9490880084600882E
:10AB70000012C6498871C6480078C87100224FF497
:10AB80000051C448F9F78CFA502002F0FDFB3089DF
:10AB9000012805D164230822BC49BF48FAF74AFCC2
:10ABA0003089012802D1502002F0EEFB012251032E
:10ABB000B848F9F775FAB54800783038C0EBC000EE
:10ABC00000EB800004EB4000B0F844003C2816DDA8
:10ABD0003C21AE4800783038C0EBC00000EB80006C
:10ABE00004EB4000A0F84410A84800783038C0EBCF
:10ABF000C00000EB800004EB4000018717E0A34891
:10AC000000783038C0EBC00000EB800004EB40005F
:10AC1000B0F84400401C81B29C4800783038C0EB4A
:10AC2000C00000EB800004EB4000A0F84410308925
:10AC300078B996480078092807DA94480078801C8B
:10AC40009249087016E01FE211E001208F49087058
:10AC500010E08E480078092805DA8C480078801CBE
:10AC60008A49087006E001208849087002E0032044
:10AC7000854908708448007806287DD100207081BD
:10AC80007089012879D106218448FAF78BFE804922
:10AC90000880084600880012804988717C48007846
:10ACA000C87100224FF400517A48F9F7F9F95020A1
:10ACB00002F06AFB3089012805D10A230222784973
:10ACC0007548FAF7B7FB6423082274497248FAF70B
:10ACD000B1FB3089012805D10A23022270496E4850
:10ACE000FAF7A8FB502002F04FFB012251036948FC
:10ACF000F9F7D6F9694800784038C0EBC00000EB9E
:10AD0000800004EB4000B0F844003C2816DD3C21F4
:10AD1000624800784038C0EBC00000EB800004EBD4
:10AD20004000A0F844105D4800784038C0EBC000F7
:10AD300000EB800004EB4000818717E05748007863
:10AD40004038C0EBC00000EB800004EB4000B0F8DE
:10AD50004400401C81B2514800784038C0EBC0002C
:10AD600000EB800004EB4000A0F844104B48007852
:10AD70004138AAF1010101E00FE00BE0884205DA59
:10AD800046480078401C4549087006E04120434988
:10AD9000087002E009203C4908703B48007803280D
:10ADA00008D10120A6F86400B6F8640018B906209E
:10ADB00035490870F7E0B6F86400012874D106211F
:10ADC0003848FAF7EFFD324908800846008800123B
:10ADD000344988712E480078C87100224FF4005120
:10ADE0002C48F9F75DF9502002F0CEFA64230822CE
:10ADF0002C492948FAF71EFB502002F0C5FA01221F
:10AE000051032448F9F74CF926480078503800EBF4
:10AE1000800007EBC000408C3C2811DD3C2121481C
:10AE20000078503800EB800007EBC00041841D48DB
:10AE30000078503800EB800007EBC000818335E0DC
:10AE400018480078503800EB800007EBC000408CB9
:10AE5000401C81B213480078503800EB800007EBAB
:10AE6000C00022E0802E0020E23900204034002083
:10AE7000A0380020984000209C4300201A030020A6
:10AE800000100140F802002016030020AA01002053
:10AE900028030020000C0140900B0020BE01002080
:10AEA00098010020EA0100200FE04184FE4800786C
:10AEB0005038042805DAFC480078401CFA4908702C
:10AEC00071E05120F84908706DE0B6F8640002287E
:10AED00066D10621F548FAF765FDF5490880084670
:10AEE00000880012F1498871F1480078C871002289
:10AEF0004FF40051EF48F9F7D3F8502002F044FA2C
:10AF000064230822E949EC48FAF794FA502002F049
:10AF10003BFA01225103E748F9F7C2F8E748007805
:10AF20005038C0EBC00000EB800004EB4000B0F8EC
:10AF300044003C2811DD3C21E0480078503800EB0B
:10AF4000800007EBC0004184DC480078503800EBFB
:10AF5000800007EBC000818311E0D84800785038AA
:10AF600000EB800007EBC000408C401C81B2D3484E
:10AF70000078503800EB800007EBC0004184CB48DC
:10AF800000785038ABF10101884205DAC7480078F3
:10AF9000401CC649087006E05120C449087002E010
:10AFA0000620C7490870C6480078092863D10020E8
:10AFB000A6F86600B6F86600E8B303F013FE0621B3
:10AFC000C048FAF7EFFCBA4908800846008800122A
:10AFD000BC498871B6480078C87100224FF400510E
:10AFE000B448F9F75DF8502002F0CEF96423082246
:10AFF000B449B148FAF71EFA502002F0C5F901220F
:10B000005103AC48F9F74CF803F016FEAD48007850
:10B01000603808EBC010B0F87E003C2811DD3C2100
:10B02000A8480078603808EBC010A0F87E10A5484A
:10B030000078603800E023E008EBC010A0F878103A
:10B040000FE0A0480078603808EBC010B0F87E0030
:10B05000401C81B29B480078603808EBC010A0F813
:10B060007E10984800786038062805DA9548007800
:10B07000401C9449087041E06120924908703DE00D
:10B080000C208F49087039E08F480078032826D1BA
:10B0900000224FF400518748F9F702F8502002F0DF
:10B0A00073F98A4800780D280AD1884840780A2820
:10B0B00006D164230C2285497F48FAF7BBF905E0E5
:10B0C0006423082281497C48FAF7B4F9502002F041
:10B0D0005BF9012251037748F8F7E2FF09E07A486B
:10B0E0000078062805D100210398018000207649C8
:10B0F000087075480078401C7349087074480068EF
:10B1000001286ED17348807804900498C01C71495E
:10B11000085C0002664908800498001D6D49085CBF
:10B12000634909880843624908806A480078012811
:10B1300012D16848407803280ED107216548FAF7F4
:10B1400031FC5B490988884202D0012062490870BD
:10B150003020604908705BE05E480078032812D117
:10B160005C48407803280ED107215A48FAF71AFCA8
:10B170004F490988884202D0012057490870312080
:10B180005449087044E053480078052812D15148CA
:10B19000407803280ED107214E48FAF703FC4449B2
:10B1A0000988884202D001204B4908703220494961
:10B1B00008702DE047480078072813D145484078AB
:10B1C00003280FD107214348FAF7ECFB38490988D7
:10B1D000884202D001204049087033203D49087060
:10B1E00016E0EDE33B480078092811D13948407852
:10B1F00003280DD107213748FAF7D4FB2C490988D9
:10B20000884202D001203449087034203149087046
:10B2100030480078302809D0208F401C2087208FAC
:10B22000C82803DDC82020870120608729480078CE
:10B2300031280ED07E20005B401C81B27E2001535D
:10B24000005BC82805DDC8217E2001530121802034
:10B2500001532048007832280ED0C420005B401CE7
:10B2600081B2C4200153005BC82805DDC821C42079
:10B2700001530121C620015316480078332811D00C
:10B280004FF48570005B401C81B24FF48570015310
:10B29000005BC82806DDC8214FF4857001530121E9
:10B2A000801C01530B4819E0EA010020E201002054
:10B2B00028030020000C0140900B0020AA01002070
:10B2C00016030020F201002017030020103900208F
:10B2D00044030020002500201903002000783428B2
:10B2E00011D04FF4A870005B401C81B24FF4A870DD
:10B2F0000153005BC82806DDC8214FF4A870015334
:10B300000121801C0153FD48405D30287EDBFB4855
:10B31000405D3F287ADC0021F848405D3038C0EBC2
:10B32000C00000EB800004EB40000187F348405D63
:10B330003038C0EBC00000EB800004EB40004187D8
:10B340000121EE48405D3038C0EBC00000EB8000CA
:10B3500004EB4000A0F84410E849681C085C03288E
:10B3600007D0681C085C062803D00120E449087057
:10B370000CE0E249A81C085C042803D00120E04945
:10B38000087003E00721DD48FAF70CFB0721DB48D2
:10B39000FAF708FBA6F86A00D849E81C095CD74A06
:10B3A000281D105C41EA002005901146681C085CCD
:10B3B00003287CD1D24800780028FAD10021104619
:10B3C000405D3038C0EBC00000EB800004EB400073
:10B3D000018701211046405D3038C0EBC00000EB12
:10B3E000800004EB4000A0F844101046415D059831
:10B3F000F5F7DEF83089012804D1C049485D002105
:10B40000F5F7BCF9BF480088082800E0B3E021DA6E
:10B41000BA48405D30280FD1B849495D3039C1EB99
:10B42000C10101EB810104EB41012031B54A1288D1
:10B43000059821F812000DE0B049495D3039C1EBA3
:10B44000C10101EB810104EB4101AE4A128805986C
:10B4500021F81200AB480088082802D10020A94931
:10B460000880A648405D3038C0EBC00101EB0010F9
:10B4700009EB8000C088002819DBA048405D303807
:10B48000C0EBC00101EB001009EB8000C08844F262
:10B49000506188420BDC9948405D3038C0EBC001F8
:10B4A00001EB001009EB8000C088404200E0FCE0A6
:10B4B000B4F8421088420DDC9048405D3038C0EB53
:10B4C000C00101EB001009EB8000C088B4F8421005
:10B4D000884216DD8948405D3038C0EBC00000EB83
:10B4E000800004EB4000008E401C81B28348405D28
:10B4F0003038C0EBC00000EB800004EB4000018658
:10B500000AE000217D48405D3038C0EBC00000EB10
:10B51000800004EB400001867848405D3038C0EB85
:10B52000C00000EB800004EB4000008E082816DB12
:10B5300008217248405D3038C0EBC00000EB80004D
:10B5400004EB4000018601216C48405D3038C0EBBF
:10B55000C00000EB800004EB400081862AE200215D
:10B560006648405D3038C0EBC00000EB800004EB63
:10B57000400081861EE26148405D40287EDB5F48D6
:10B58000405D4F287ADC00215C48405D3038C0EBDC
:10B59000C00000EB800004EB400081870121574888
:10B5A000405D4038C0EBC00000EB800004EB400081
:10B5B000A0F844105149681C085C032807D0681C97
:10B5C000085C062803D001204D49087013E04B4960
:10B5D000A81C085C042803D00120494908700AE02F
:10B5E00007214648FAF7DEF947490988884202D020
:10B5F0000120434908704149681C085C032855D163
:10B600003F480078D8BB0B462A1D9B5C8C46EA1C41
:10B610001CF8022043EA02200A46515DF4F7C8FFF5
:10B620003A480088082839DA3449281D085C0102A4
:10B630003248405D4038C0EBC00000EB800004EBB6
:10B6400040001030314A128820F812102B48405D1B
:10B650004038C0EBC00000EB800004EB400010302D
:10B660002A49098830F81100244AE91C515C084332
:10B670001146495D4039C1EBC10101E017E015E019
:10B6800001EB810104EB41011031204A128821F8BD
:10B6900012001E480088401C1C4908801B48008876
:10B6A000082802D100201949088083E182E113486B
:10B6B000007850287DDB114800785F2879DCB6F8E7
:10B6C000640001287CD101210C480078503800EB3F
:10B6D000800007EBC0004184002108480078503802
:10B6E00000EB800007EBC000818304484078042809
:10B6F0000ED00120024908701DE000000025002046
:10B70000190300201C030020280300201E03002032
:10B71000D9488078042803D00120D84908700AE06D
:10B720000721D548FAF73EF9D5490988884202D061
:10B730000120D2490870D049681C085C04283ED119
:10B74000CE480078B0BB0846C0780002CD490880DA
:10B75000C948007909880843CA4908800846008812
:10B76000F4F759FEC8490860C34840790002C5494A
:10B770000880C148807909880843C2490880084682
:10B780000088F4F748FEC1490190F4F7FDFD0290EE
:10B79000BD4801680298F4F76DFDBB490860086870
:10B7A000BB49F4F7F1FDB449495D503901EB810122
:10B7B00002E05CE003E003E047F83100FAE0F9E082
:10B7C000B6F86400022850D10121AB480078503807
:10B7D00000EB800007EBC00041840021A648007800
:10B7E000503800EB800007EBC0008183A24840780E
:10B7F000042803D00120A149087012E09E488078F7
:10B80000042803D001209D4908700AE007219A48C6
:10B81000FAF7C8F89A490988884202D00120974966
:10B82000087007219448FAF7BDF8A6F86800924915
:10B83000681C085C042819D190480078B0B9084603
:10B840000079914908708C48C07848708A4880799E
:10B85000887089484079C870084601688648405D0C
:10B86000503800EB800047F83010A3E0A2E0824897
:10B87000007860281EDB804800786F281ADC0121E0
:10B8800084480078603808EBC010A0F87E100021D2
:10B8900080480078603808EBC010A0F8781076482F
:10B8A0004078032807D074484078062803D0012048
:10B8B000724908707EE070488078022803D0012029
:10B8C0006E49087076E005216B48FAF76BF86C4911
:10B8D0000988884203D00120684908706AE06649F7
:10B8E000681C085C032865D164480078A0BB084642
:10B8F000405D613806285BD2DFE800F003111F2F9E
:10B900003D4B5D4800795C49C97840EA012001B2AD
:10B910005948405D603808EBC010418049E0564806
:10B9200000795549C97840EA012001B25248405D8A
:10B93000613808EBC01041853BE04F4800794E4923
:10B94000C97840EA012001B24B48405D623808EBFB
:10B95000C010A0F852102CE02CE04748007946496E
:10B96000C97840EA012001B24348405D623808EBE3
:10B97000C01041801DE0404800793F49C97840EA45
:10B98000012001B23C48405D633808EBC01041859E
:10B990000FE0394800793849C97840EA012001B2FE
:10B9A0003548405D643808EBC010A0F8521000E044
:10B9B00000BF00BF002038490860304908704BE0E4
:10B9C000208F401C2087208F782803DD7820208757
:10B9D000012060877E20005B401C81B27E200153E5
:10B9E000005B782805DD78217E200153012180202D
:10B9F0000153C420005B401C81B2C4200153005B92
:10BA0000782805DD7821C42001530121C620015387
:10BA10004FF48570005B401C81B24FF48570015378
:10BA2000005B782806DD78214FF4857001530121F1
:10BA3000801C01534FF4A870005B401C81B24FF48E
:10BA4000A8700153005B782806DD78214FF4A870B8
:10BA500001530121801C015310480078032806DAA5
:10BA60000E480078401C0D490870FFF734B80020DC
:10BA70000A490870F9E7000000250020190300209A
:10BA8000280300202C0300203003002000FF7F4704
:10BA900000007A44F2010020440300201603002035
:10BAA00008B5F84C0026B046B14600BFB246B346D2
:10BAB00000200090F44D00BF322001F0A9FF4FF4A8
:10BAC0008061F248F8F7E2FAF14800680128F3D102
:10BAD0004FF00008EF4800783A2826D1ED4840782A
:10BAE000332822D1EB48807839281ED1E948C07824
:10BAF00030281AD1002710E0E649491C01EB470025
:10BB0000FAF7A2F8E449C855E249491C01EB47009D
:10BB1000FAF79AF8E149C8557F1C402FECDB402228
:10BB2000DE49DC48F4F782FB00BF00BFD94890F83B
:10BB30003E000602D74890F83F000643D5480078FB
:10BB4000392811D0D348407801280DDCD1488078BD
:10BB5000952809DCCF48C078502805DCE888401CCF
:10BB6000E8804FF0010842E0CA484079012805D03A
:10BB7000E888401CE8804FF0010838E0C548C079EB
:10BB8000032809D0C348C079062805D0E888401C9E
:10BB9000E8804FF001082AE00020E880C0490880D2
:10BBA0000DE0BC48BE490988415C05F10D00BC4A66
:10BBB00012888154BA480088401CB9490880B848A6
:10BBC00000884028EDDB0020B54908800BE0B14833
:10BBD000B3490988405CB24909886054B04800887C
:10BBE000401CAF490880AE4800881028EFDBB8F150
:10BBF000000F7DD1A748007A688168894FF6FF71F0
:10BC000001EA002068816889A249497A084368816D
:10BC1000688973286DD036DC29286BD012DCA0F13E
:10BC20001000192867D2DFE800F0797C7D82666613
:10BC300066666666666666666666868B90919293B1
:10BC400094959D0052286ED00EDC43286CD006DC03
:10BC500040286AD0412869D042284CD1A3E050281E
:10BC60006FD05128F9D1BDE070286BD006DC532885
:10BC700069D0542868D05528EFD1D3E071286ED010
:10BC80007228EAD1D9E0B0F5BF7F69D01CDC7A28F0
:10BC900067D008DCA0F174000628C3D2DFE800F00A
:10BCA000D7DFE7F1F0EF7E2877D006DC7B2875D070
:10BCB0007C2874D07D28D0D129E1A0F22110002861
:10BCC0006ED00128C9D148E141F29612811A904202
:10BCD00067D01CDC41F29312A0EB020190427DD0B0
:10BCE00010DCB0F5C07F7AD0B0F5C87F78D003E023
:10BCF00060E2A7E037E002E16FF4895108440028D0
:10BD0000ABD12BE101296CD00229A6D135E106295E
:10BD100088D2DFE801F0F4F3F2F1F0EFFEF754F827
:10BD20004FE14EE14DE162E03EE01DE03AE05D486A
:10BD3000FEF774F845E12046FDF7EAFB814640E155
:10BD40003FE132E073E06BE06BE03AE139E138E18A
:10BD500037E136E12046FAF799FB814631E167E0A9
:10BD6000E3E0BBE02DE12CE12046F4F781FE8146C3
:10BD700000204B4908800BE0464849490988405C4F
:10BD800047490988605446480088401C4449088057
:10BD9000434800884028EFDB13E1BFE0A3E0AFE0B9
:10BDA000DAE0EFE00DE10CE10BE1204600F0E4FE0B
:10BDB000814600203A4908800BE036483849098816
:10BDC000405C37490988605435480088401C344934
:10BDD0000880334800884028EFDBF2E0C3E0ABE0A6
:10BDE000B2E0C5E0204600F017FF8146E9E02046BA
:10BDF000FAF7E6FA81460020294908800BE0254839
:10BE000027490988405C26490988605424480088ED
:10BE1000401C23490880224800884028EFDBD0E0FE
:10BE2000CFE0CEE02046FDF749FE8146C9E0C8E0FC
:10BE30002046F4F7DBFE8146C3E02046FAF70EFA0F
:10BE40008146BEE02046FEF7EFF88146B9E0204685
:10BE5000F4F71EFF8146012013490870B1E0204627
:10BE6000FAF73AFA814601200F490870A9E0204606
:10BE700000F02AFF814601200B490870A1E025E06F
:10BE80001CE013E090000020E23900200010014087
:10BE900048030020002900201C000020E00D0020A5
:10BEA00034030020600E0020F80200202046F9F73D
:10BEB0009FFB81460120C149087082E02046F9F7C6
:10BEC0007FFE81460120BD4908707AE02046F4F7E4
:10BED0008BFD81460120B949087072E0204600F0D0
:10BEE0002FFB81466DE02046F9F7F6FB0120B349B0
:10BEF000087066E05FE059E053E04DE047E05FE046
:10BF00002046F9F7D5FC0120AC49087059E02046DD
:10BF1000F9F758FC0120A949087052E02046F9F7CA
:10BF2000F3FA0120A54908704BE0204600F0D0FA52
:10BF30000120A249087044E02046F5F76BFC8146D9
:10BF400001209E4908703CE02046F9F753FD8146E8
:10BF500001209A49087000BF33E032E02046FAF72A
:10BF60009DFE82462DE02046FAF7BAFB834628E084
:10BF70002046FBF7E3FA834623E02046FBF7B4FDB7
:10BF800083461EE02046FBF7DDFF834619E020468E
:10BF9000FCF706FA834614E02046FCF72FFC8346A4
:10BFA0000FE02046FCF758FE83460AE02046FDF7E6
:10BFB00081F8834605E02046FDF7B2FE009000E0E0
:10BFC00000BF00BF6889132821D13E217C48F9F7C2
:10BFD000E9FC064630127A4981F83E0081F83F605C
:10BFE000002210217748F8F75BF8502001F0CCF9D7
:10BFF0006423402272497448F9F71CFA502001F07A
:10C00000C3F9012210216F48F8F74AF8D0E0BBF1DC
:10C01000000F26D04FF0000B94212046F9F7C2FC08
:10C020000646301284F8940084F8956000221021AE
:10C030006448F8F735F8502001F0A6F902F0D2FD77
:10C0400096231A4621466048F9F7F4F902F0F4FD08
:10C05000502001F099F9012210215A48F8F720F8F0
:10C06000A6E0009830B30020009060212046F9F748
:10C0700099FC0646301284F8600084F86160002262
:10C0800010215048F8F70CF8502001F07DF902F02B
:10C09000A9FD9623622221464B48F9F7CBF902F01D
:10C0A000CBFD502001F070F9012210214548F7F72F
:10C0B000F7FF7DE0BAF1000F2CD04FF0000A00200E
:10C0C00084F8E80084F8E900EA212046F9F76AFCE0
:10C0D0000646301284F8EA0084F8EB600022102152
:10C0E0003848F7F7DDFF502001F04EF902F07AFDF5
:10C0F0004FF4FA73EC2221463348F9F79BF902F02A
:10C100009BFD502001F040F9012210212D48F7F746
:10C11000C7FF4DE0B9F1000F25D0002084F83C00A6
:10C1200084F83D003E212046F9F73CFC06463012DB
:10C1300084F83E0084F83F60002210212148F7F780
:10C14000AFFF502001F020F96423402221461E4811
:10C15000F9F770F9502001F017F901221021194860
:10C16000F7F79EFF24E0FF2084F83C0084F83D00B0
:10C170003E212046F9F716FC0646301284F83E00B0
:10C1800084F83F60002210210E48F7F789FF502005
:10C1900001F0FAF86423402221460B48F9F74AF9E6
:10C1A000502001F0F1F8012210210648F7F778FF3E
:10C1B0004FF000090020054908607DE4F8020020E6
:10C1C000600E002000080140D00B00204803002032
:10C1D000214E00BF214FDFF8888000BF4FF48061FF
:10C1E0002048F7F753FFF4F737FB002430E0052C25
:10C1F00015D2DFE804F00304080C100010E0174F1C
:10C20000DFF85C800CE0184FDFF8608008E0184F22
:10C21000DFF8608004E0184FDFF8608000E000BFC6
:10C2200000BF04EB840156F83100234642463946EC
:10C23000F4F776FD054604EB840006EBC00085614B
:10C240002046F5F7F9F8642001F0E2FB601CC4B267
:10C25000052CC3DACBE700009840002060030020E3
:10C260002407010800100140F0040020B408010870
:10C2700080060020440A010810080020D40B0108A1
:10C2800000BF012001F0C4FBFBE700BF012001F06B
:10C29000BFFBFBE700BF012001F0BAFBFBE700BFDB
:10C2A000012001F0B5FBFBE700BF012001F0B0FB6E
:10C2B000FBE700BF012001F0ABFBFBE700BF4FF441
:10C2C000FA7001F0A5FB07480068401C05490860AA
:10C2D00001210548F7F7DAFE4FF480610348F7F7CC
:10C2E000D5FEECE7040000200008014000100140EA
:10C2F00010B500BF502080F31188BFF34F8FBFF3FC
:10C300006F8F00BF03F00AFC18B14FF08050044952
:10C31000086000BF002080F3118800BF10BD00003E
:10C3200004ED00E000B58FB0282105A8F3F797FFD2
:10C3300014216846F3F793FF01200590000406904E
:10C34000002007900120099002200C90C1030D915C
:10C350004FF4E0110E9105A8F8F7FCF808B1F5F7D5
:10C3600048F90F20009002200190002002904FF425
:10C37000806003900020049002216846F7F792FF46
:10C3800008B1F5F736F90FB000BD704710B5024897
:10C39000F8F78FFC10BD0000C00A002010B502485D
:10C3A000F8F787FC10BD0000080B002010B502480C
:10C3B000F8F77FFC10BD00003C0F002010B50268AC
:10C3C000204B98420ED0204B98420BD0B0F1804FBA
:10C3D00008D01E4B984205D01D4B984202D01D4BF1
:10C3E000984203D122F070024B681A43154B9842D1
:10C3F0000ED0154B98420BD0B0F1804F08D0134BA4
:10C40000984205D0124B984202D0124B984203D169
:10C4100022F44072CB681A4322F080034C6943EA4D
:10C42000040202608B68C3620B688362054B98420A
:10C4300002D0054B984201D10B690363012343618C
:10C4400010BD0000002C01400034014000040040F9
:10C4500000080040000C004030B50C46816821F413
:10C460007F4142EA032525432943816030BD0A46C6
:10C47000816821F0700142F0070319438160704721
:10C4800030B50B461446026A056A25F001050562BF
:10C49000816921F0F00141EA041122F00A021A43F5
:10C4A0008161026230BD30B50B461446056A25F045
:10C4B000100505628169026A21F4704141EA043184
:10C4C00022F0A00242EA03128161026230BD000044
:10C4D00070B50646164D00241648847C4FF6FF7052
:10C4E00000EA04241348C07C0443032C1FD168884D
:10C4F000E8B9287D06281AD1012068800D48007D02
:10C500000D490880084600884FF6FF7101EA0020B7
:10C51000094908800748407D098808430649088082
:10C5200008460288034916310448F3F77FFE70BDC0
:10C53000E239002000290020DA0900209C3900207F
:10C5400070B58AB005461D4E1D4C28216846F3F78C
:10C5500086FEA17F607F41EA0020ADF80000207DCB
:10C56000062804D1012217496846F5F70DF9012282
:10C5700014496846F5F7F2F8BDF800000012287477
:10C58000BDF800006874BDF800004FF6FF718842E6
:10C5900003D0BDF80000A6F86600297C607F8142C8
:10C5A00009D1697CA07F814205D1207D062802D176
:10C5B00001200AB070BD0020FBE70000A038002079
:10C5C000E239002048F0070870B50546284602F019
:10C5D0007DFA044614B1D4E90010884770BD70B5E7
:10C5E00005466C6A0020E085E0842046F8F76EFC82
:10C5F00070BD70B506460025746A20684069C0F3B6
:10C60000C01594F83900212805D125B10020E08417
:10C61000204600F060F820684069C0F3801594F867
:10C620003A00222805D125B10020E085204600F0FF
:10C6300032F8E06B40F01000E0632046F8F746FC6B
:10C6400070BD70B505466C6A2868006800F020006F
:10C65000B0B90020E0852068C06820F480702168AF
:10C66000C8602068406920F00100216848612068A6
:10C67000406920F0400021684861202084F83A0099
:10C680002046F8F7D5FE70BD70B50446656A2846A9
:10C69000F8F7CFFE70BD0168C96821F49071026897
:10C6A000D1600168496921F00101026851612021CE
:10C6B00080F83A10704710B504462068C06820F032
:10C6C00040002168C860202084F839002046F8F72F
:10C6D0001AFF002010BD0168C96821F0C00102687E
:10C6E000D160202180F83910704770B5044694F865
:10C6F0003A00222847D1A068B0F5805F0CD12069AC
:10C7000050B90025A66A20684068C0F30800308050
:10C71000A06A801CA06215E0A56A0026A068B0F59A
:10C72000805F03D0A06828B9206918B920684068E4
:10C73000287004E02068406800F07F002870A06A3C
:10C74000401CA062E08D401E80B2E085C8B9206820
:10C75000C06820F020002168C8602068C06820F40C
:10C7600080702168C8602068406920F0010021685D
:10C770004861202084F83A002046F8F759FE00204E
:10C7800070BD0020FCE70220FAE7000070B5044607
:10C790002168096921F44051E2681143226811615E
:10C7A0002269A1681143626941EA02052168C968EA
:10C7B00041F20C62914329432268D16021684969A2
:10C7C00021F44071A2691143226851612D4A216808
:10C7D000914202D1F7F764FE01E0F7F751FE00EB5A
:10C7E000C00101EB001162689200B1FBF2F100EBB5
:10C7F000C00202EB001263689B00B2FBF3F26423F9
:10C80000B2FBF3F202EBC20303EB0212A1EB8201D3
:10C81000322202EB01116422B1FBF2F101F0F001CE
:10C8200000EBC00202EB001263689B00B2FBF3F264
:10C830006423B2FBF3F201EB021200EBC00101EB47
:10C84000001163689B00B1FBF3F100EBC00303EB45
:10C8500000136668B600B3FBF6F36426B3FBF6F389
:10C8600003EBC30606EB0313A1EB8301322303EBB7
:10C8700001116423B1FBF3F101F00F0111442268AF
:10C88000916070BD00380140014691F839002128BF
:10C8900028D18868B0F5805F0BD1086948B90A6A69
:10C8A0001088C0F308000B685860086A801C086292
:10C8B00005E00B6A581C086218780B685860C88C31
:10C8C000401E80B2C88458B90868C06820F0800053
:10C8D0000B68D8600868C06840F040000B68D860FA
:10C8E000002070470220FCE72DE9F04104460D4688
:10C8F00017469846069E21E0701CF8B12EB1F7F756
:10C90000D5FBA0EB0800B04218D92068C06820F41D
:10C91000D0702168C8602068406920F0010021685B
:10C920004861202084F8390084F83A0000BF0020D4
:10C9300084F8380000BF0320BDE8F081206800685B
:10C940002840A84201D1012000E00020B842D3D005
:10C950000020F1E708B51A48F8F7BAFA1848006855
:10C960000068C0F3001050B300BF002000901448CE
:10C97000006800680090124800684068009000BF9E
:10C9800000BF0F48F8F76FFA0E4800684068C0F51E
:10C9900080700D49086008460C4902680C48F3F79E
:10C9A00045FC4FF480710948F3F759FC4FF480724D
:10C9B00006490348F8F7DAFC01200649086008BD7B
:10C9C000900B0020500C0020400300200024002089
:10C9D000002500204403002008B51A48F8F778FA2B
:10C9E000184800680068C0F3001050B300BF002072
:10C9F0000090144800680068009012480068406881
:10CA0000009000BF00BF0F48F8F72DFA0E480068ED
:10CA10004068C0F580700D49086008460C490268FE
:10CA20000C48F3F703FC4FF480710948F3F717FC47
:10CA30004FF4807206490348F8F798FC0120064934
:10CA4000086008BDD00B0020D80C0020380300205F
:10CA500000270020002900204803002008B51A48BC
:10CA6000F8F736FA184800680068C0F3001050B3B1
:10CA700000BF002000901448006800680090124831
:10CA800000684068009000BF00BF0F48F8F7EBF95E
:10CA90000E4800684068C0F580700D49086008467F
:10CAA0000C4902680C48F3F7C1FB4FF48071094848
:10CAB000F3F7D5FB4FF4807206490348F8F756FCAC
:10CAC00001200649086008BD100C00201C0D002044
:10CAD0003C030020002A0020002B00204C030020F3
:10CAE00000BFFEE730B58BB01F4D282101A8F3F73A
:10CAF000B6FB002401221D4901A8F4F72FFEBDF862
:10CB000004004FF6FF71884202D0BDF80400A880EF
:10CB10000822174901A8F4F721FE00240FE001A81C
:10CB200030F814004FF6FF71884206D001A830F8A3
:10CB3000141005F1140020F81410601CC4B22888E9
:10CB4000A042ECDC00240AE005F1140030F81400E7
:10CB500008490988084407490880601CC4B228882D
:10CB6000A042F1DC0BB030BDA038002028F007084F
:10CB700000E007085C0300202DE9F0418046244DC9
:10CB8000002400270026688800283CD1287D06283C
:10CB900036D101206880AA7F2046611CCCB21D4995
:10CBA0000A5406222046611CCCB21A490A540022BB
:10CBB0002046611CCCB217490A5402222046611C4F
:10CBC000CCB214490A5400222046611CCCB211494F
:10CBD0000A5401222046611CCCB20E490A54C819DD
:10CBE0000621F8F7DFFE064632122046611CCCB261
:10CBF00008490A542046611CCCB206490E5404E090
:10CC00000020BDE8F0810020FBE70120F9E70000EB
:10CC1000E2390020563900202DE9F0478146274DA2
:10CC2000274F0024A04600266888002842D1287D8E
:10CC300006283CD101206880B888012800D100BFB7
:10CC4000AA7F2046611CCCB21E490A540622204607
:10CC5000611CCCB21B490A5400222046611CCCB294
:10CC600018490A5410222046611CCCB215490A54B6
:10CC7000EA7F2046611CCCB212490A542020425D52
:10CC80002046611CCCB20F490A5401EB0800062172
:10CC9000F8F788FE064632122046611CCCB20949DC
:10CCA0000A542046611CCCB206490E5404E0002010
:10CCB000BDE8F0870020FBE70120F9E7E23900201A
:10CCC000A038002056390020F0B58BB00646344F0E
:10CCD000344D282101A8F3F7C2FA002400BF09E06F
:10CCE00004F1100005F10D01085C01A921F8140000
:10CCF000601CC4B2287EA042F2DC287D062804D144
:10CD00000122294901A8F4F73FFD0122264901A883
:10CD1000F4F724FDBDF804003074BDF804000528C4
:10CD200002DABDF80400B880287D062805D1082263
:10CD30001E490DF10600F4F727FD08221B490DF1ED
:10CD40000600F4F70BFD002424E001A9601C31F873
:10CD50001020103005F10D01085C824205D0287DBD
:10CD6000062802D100200BB0F0BD01A9601C31F8EB
:10CD7000100008280CDA601C31F8101007F11400BC
:10CD800020F8141001A9601C11F810101030315453
:10CD9000601CC4B2287EA042D7DC0120E3E700007B
:10CDA000A0380020E239002028F0070800E007083A
:10CDB00010B502467C4800BFD1B201EB011303EB72
:10CDC000430330F81330012B35D1002301EB01145C
:10CDD00004EB440400EB4404A4F8523001EB0113CB
:10CDE00003EB430300EB4303B3F850305B1C01EB50
:10CDF000011404EB440400EB4404A4F8503001EBAC
:10CE0000011303EB430300EB4303B3F85030022B51
:10CE100011DB002301EB011404EB440400EB440498
:10CE2000A4F85030012301EB011404EB440400EB9F
:10CE30004404A4F8583001EB011303EB430330F82A
:10CE40001330A3BB002301EB011404EB440400EBFB
:10CE50004404A4F8503001EB011303EB430300EB4F
:10CE60004303B3F852305B1C01EB011404EB4404A0
:10CE700000EB4404A4F8523001EB011303EB43032D
:10CE800000EB4303B3F85230022B10DB002301EB1D
:10CE9000011404EB440400EB4404A4F8523001EB09
:10CEA000011404EB440400EB4404A4F8583001EBF3
:10CEB000011303EB430300EB43031B8D012B35D11F
:10CEC000002301EB011404EB440400EB4404A4F838
:10CED000563001EB011303EB430300EB4303B3F8BC
:10CEE00054305B1C01EB011404EB440400EB4404DC
:10CEF000A4F8543001EB011303EB430300EB4303AD
:10CF0000B3F85430022B11DB002301EB011404EBC6
:10CF1000440400EB4404A4F85430012301EB011451
:10CF200004EB440400EB4404A4F85A3001EB011371
:10CF300003EB430300EB43031B8DA3BB002301EB77
:10CF4000011404EB440400EB4404A4F8543001EB56
:10CF5000011303EB430300EB4303B3F856305B1CB0
:10CF600001EB011404EB440400EB4404A4F8563034
:10CF700001EB011303EB430300EB4303B3F856301B
:10CF8000022B10DB002301EB011404EB440400EB43
:10CF90004404A4F8563001EB011404EB440400EB04
:10CFA0004404A4F85A3010BD363A00200FB4084BA0
:10CFB00010B504A902AA039800F040F8044602A99B
:10CFC000002000F0DCF9204610BC5DF814FB0000E6
:10CFD0007FD3000802480068C0F3022070470000B9
:10CFE0000CED00E010B5002804DB0A07130E054A1B
:10CFF000135406E00A07140E034A00F00F031B1F28
:10D00000D45410BD00E400E018ED00E0EFF311800F
:10D010007047EFF305807047EFF31080704702E030
:10D0200008C8121F08C1002AFAD1704770470020B3
:10D0300001E001C1121F002AFBD170472DE9FF4F0B
:10D040008BB088460546002606E025280BD0DDE992
:10D050000D1290476D1C761C28780028F5D10FB072
:10D060003046BDE8F08F0024A146A2460122AE4919
:10D0700000E0044315F8013F203B02FA03F00842A8
:10D08000F7D128782A2810D06FF02F022878A0F145
:10D090003001092915D809EB890102EB410144F05F
:10D0A000020400EB01096D1CF0E758F8041B5FEA6D
:10D0B000010903D544F40054C9F1000944F0020405
:10D0C0006D1C28782E2817D115F8010F44F00404A0
:10D0D0002A280ED06FF02F022878A0F130010929FC
:10D0E0000AD80AEB8A0102EB410100EB010A6D1C30
:10D0F000F2E758F804AB6D1C28786C280FD006DCDA
:10D100004C2817D068280DD06A2814D104E0742860
:10D1100010D07A280FD10DE044F400140AE044F452
:10D12000801401E044F440146978814202D104F58E
:10D1300080146D1C6D1C2878692865D006DC0028D9
:10D140008DD0632827D0642806D15DE06E2808D0F2
:10D1500073282AD0752877D0DDE90D129047761C08
:10D16000E0E0C4F30250022809D003280DD0D8F81B
:10D17000001004280DD00E6008F10408D2E0D8F8A1
:10D180000010F217C1E90062F6E7D8F800100E802F
:10D19000F2E70E70F0E718F8041B8DF8001000207D
:10D1A0008DF80100EB46012003E058F804BB4FF076
:10D1B000FF3061074FF0000701D40AE07F1C57459C
:10D1C0000DDA8742FADB1BF807100029F6D106E0DA
:10D1D0007F1C8742FCDB1BF807100029F8D1DDE932
:10D1E0000D23A9EB07008146214600F0B1F8304439
:10D1F000C61904E0DDE90D121BF8010B90477F1EF4
:10D20000F8D22146484688E058F8040BC4F302518E
:10D210004FF00A0B032900D100B2042900D140B21B
:10D22000002802DA40422D2102E0210505D52B21FC
:10D230008DF82410012104E006E0E10710D0202140
:10D24000F6E708AF089113E058F8040BC4F3025155
:10D250004FF00A0B032900D180B2042900D1C0B2DB
:10D260000021EEE75946F3F713F9303107F8011DB5
:10D270000028F7D1ADEB070000F1200B600702D5C5
:10D2800024F4803401E04FF0010ADA4502DDAAEB14
:10D290000B0000E00020824600EB0B0108980144DF
:10D2A000A9EB01000A90E00306D4DDE90D23214635
:10D2B0000A9800F04DF806444FF0000908E009A96B
:10D2C00011F80900DDE90D12904709F10109761CFA
:10D2D00008998945F3DBE0030CD5DDE90D232146F0
:10D2E0000A9800F035F8064404E0DDE90D1230201C
:10D2F0009047761CBAF10001AAF1010AF5DC05E0BD
:10D30000DDE90D1217F8010B9047761CBBF1000107
:10D31000ABF1010BF4DC0A982146DDE90D2300F0A6
:10D3200005F806446D1C97E6092801002DE9F04137
:10D33000044600251E461746880404D405E03946F5
:10D340002020B0476D1C641EF9D52846BDE8F08149
:10D350002DE9F041044600251E469046C80301D53C
:10D36000302700E02027880404D505E041463846F0
:10D37000B0476D1C641EF9D52846BDE8F0810A68E7
:10D38000531C0B6010707047C200002100BF01E009
:10D3900000BF491C9142FBD3704700001FB500201D
:10D3A0000090019002900390F6F792FEF3F7CEFD05
:10D3B000F8F7CCFEFFF796FBF3F7C4FBFEF7B2FFDE
:10D3C000F8F7BEFCF8F78CFCF8F724FEF8F706FE39
:10D3D000F8F74CFEF8F776FEF8F754FCF8F762FC25
:10D3E000F8F78CFDF8F7C4FDF8F746FD012251036C
:10D3F000EF48F6F755FE01221103ED48F6F750FE0F
:10D4000001221021EB48F6F74BFE4FF480600090AC
:10D410000120019000200290022003906946E64816
:10D42000F6F78CFC00224FF40051E148F6F738FE85
:10D4300000224FF40051DE48F6F732FE00224FF48E
:10D440008051DB48F6F72CFE00221021D948F6F770
:10D4500027FE0220F6F78CFB2021D848F2F7FFFECA
:10D460000522D7A1D548FFF7A1FD0446A2B24FF48B
:10D470009673D249D748F7F7DDFF01225103CC4814
:10D48000F6F70EFE01221103C948F6F709FE012244
:10D490001021C848F6F704FE00F006FBCE4800F065
:10D4A000A1FBCE490860CE4800F09CFBCD49086046
:10D4B000CD4800F097FBCD490860CD4800F092FBC5
:10D4C000CC490860CC4800F08DFBCC490860CC48C2
:10D4D00000F088FBCB490860CB4800F083FBCB49C8
:10D4E0000860CB4800F07EFBCA490860CA4800F0DB
:10D4F00079FBCA490860CA4800F074FBC949086052
:10D50000C94800F06FFBC9490860C94800F06AFBD0
:10D51000C8490860C84A0121084600F0CBFBC7494A
:10D520000860C74A0121084600F0C4FBC5490860ED
:10D53000C54A0121084600F0BDFBC4490860C44A41
:10D540000121084600F0B6FBC2490860C24A012129
:10D55000084600F0AFFBC1490860C14A01210846F6
:10D5600000F0A8FBBF490860BF4A0121084600F04F
:10D57000A1FBBE490860BE4A0121084600F09AFBA3
:10D58000BC490860BC4A0221084600F093FBBB4935
:10D590000860BB4A0221084600F08CFBB9490860CC
:10D5A000B94A0221084600F085FBB8490860B84A2C
:10D5B0000221084600F07EFBB6490860B64B002207
:10D5C0000121B64800F05AFCB5490860B54B00226D
:10D5D0000121B54800F052FCB4490860B44B002268
:10D5E0000121B44800F04AFCB3490860B34B002263
:10D5F0000121B34800F042FCB2490860B24B00225E
:10D600000121B24800F03AFCB1490860B14B002258
:10D610000121B14800F032FCB0490860B04B002253
:10D620000121B04800F02AFCAF490860AF4B00224E
:10D630000121AF4800F022FCAE490860AE4B002249
:10D640000121AE4800F01AFCAD490860AD4B002244
:10D650000121AD4800F012FCAC490860AC4A02213F
:10D66000102000F063FAAB490860AB4A0221102099
:10D6700000F05CFAA9490860A94A0221102000F0D4
:10D6800055FAA8490860A84A0221102000F04EFA75
:10D69000A6490860A64A0221102000F047FAA549D1
:10D6A0000860A54A0221102000F040FAA349086052
:10D6B000A34A0021A34800F073FBA3490860A34AD2
:10D6C0000021A34800F06CFBA2490860A24A002197
:10D6D000A24800F065FBA2490860A24A0021A248C6
:10D6E00000F05EFBA1490860A14A0021A14800F0BA
:10D6F00057FBA1490860A14A0021A14800F050FB56
:10D70000A0490860A04A0021A04800F049FBA049B8
:10D710000860A04A0021A04800F042FB9F49086031
:10D720009F4A00219F4800F03BFB9F4908609F4AA9
:10D7300000219F4800F034FB9E4908609E4A00216A
:10D740009E4800F02DFB9E4908609E4A00219E489D
:10D7500000F026FB9D4908609D4800F075F99D4941
:10D7600008609D4800F070F99C4908609C4800F0F2
:10D770006BF99C4908609C4800F066F99B49086079
:10D780009B4800F061F99B4908609B4800F05CF9F8
:10D790009A4908609A4800F057F99A4908609A48EF
:10D7A00000F052F99949086000F09EF900BFFEE7C9
:10D7B000000C01400008014000100140600D0020F5
:10D7C0007379737974656D2072657365742E2E2E6E
:10D7D00025356400D00B00202405010874020020C8
:10D7E0003405010878020020440501087C0200206D
:10D7F000540501088002002064050108840200200D
:10D800007405010888020020840501088C020020AC
:10D810009405010890020020A4050108940200204C
:10D82000B405010898020020C40501089C020020EC
:10D83000D4050108A0020020E4050108A40200208C
:10D84000F4050108A802002004060108AC0200202B
:10D8500014060108B002002024060108B4020020CA
:10D8600034060108B802002044060108BC0200206A
:10D8700054060108C002002064060108C40200200A
:10D8800074060108C802002084060108CC020020AA
:10D8900094060108D002002084040108390F000812
:10D8A0004C020020940401083D0F000850020020A3
:10D8B000A40401083F0F000854020020B40401082A
:10D8C000410F000858020020C4040108430F00085B
:10D8D0005C020020D4040108450F0008600200200B
:10D8E000E4040108470F000864020020F404010862
:10D8F000490F000868020020040501084B0F0008CA
:10D900006C020020140501083B0F00087002002083
:10D91000F4030108340200200C040108380200203E
:10D92000240401083C0200203C04010840020020BD
:10D9300054040108440200206C040108480200203D
:10D9400044020108ADA0000804020020680201089A
:10D95000B9A00008080200208C0201085DAA000896
:10D960000C020020B0020108A1BA00081002002039
:10D97000D4020108D1C1000814020020F8020108F5
:10D9800081C20008180200201C0301088BC2000895
:10D990001C0200204003010895C20008200200205C
:10D9A000640301089FC200082402002088030108C4
:10D9B000A9C2000828020020AC030108B3C2000875
:10D9C0002C020020D0030108BDC200083002002054
:10D9D000A4060108D4020020B4060108D8020020E1
:10D9E000C4060108DC020020D4060108E002002081
:10D9F000E4060108E4020020F4060108E802002021
:10DA000004070108EC02002014070108F0020020BE
:10DA100070B50546FFF7FDFA48B9FFF7FDFA30B9D2
:10DA200008480068022805D1FFF7F0FA10B16FF03E
:10DA3000050404E0002415B1284601F023FA20462D
:10DA400070BD0000400A002070B504460026FFF7B4
:10DA5000E0FA00BBFFF7E0FAE8B9124800680228D4
:10DA600002D1FFF7D3FAB0B94FF0FF3564B1A06827
:10DA700020B1E068202801D3012506E0A06820B984
:10DA8000E06810B9002500E00025012D04D1A06850
:10DA900001F02FFB064603E015B901F01BFB06461B
:10DAA000304670BD400A002010B5FFF7B2FA48B901
:10DAB000FFF7B2FA30B90B480068022805D1FFF72A
:10DAC000A5FA10B16FF0050409E00648006820B916
:10DAD000012004490860002401E04FF0FF34204693
:10DAE00010BD0000400A002010B5FFF792FA48B9B7
:10DAF000FFF792FA30B90C480068022805D1FFF709
:10DB000085FA10B16FF005040CE0074800680128A1
:10DB100006D102200449086001F030FA002401E037
:10DB20004FF0FF34204610BD400A00202DE9F84395
:10DB300005460E4614464FF00009FFF76AFA002822
:10DB40004BD1FFF769FA002847D125480068022821
:10DB500003D1FFF75BFA00283FD1002D3DD0002E06
:10DB60003BD04FF0FF37BCB1A06858B1E0685028F7
:10DB700008D3206930B105FB06F06169814201D309
:10DB800001270AE0A06840B9E06830B9206920B9EF
:10DB9000606910B9002700E00027012F09D100209B
:10DBA000009031462846A368226901F000FC8146B6
:10DBB00006E02FB900223146284601F0C9FB814614
:10DBC000B9F1000F09D014B1D4F8008001E04FF092
:10DBD00000084146484601F0E7F84846BDE8F883AA
:10DBE000400A00202DE9F04704460026FFF711FA0D
:10DBF000002859D1FFF710FA002855D12C480068A9
:10DC0000022803D1FFF702FA00284DD10CB1676852
:10DC100000E0002707F0010008B1012500E0002521
:10DC200007F0080008283FD04FF0FF3874B1A06813
:10DC300028B1E068502802D34FF0010808E0A0683E
:10DC400030B9E06820B94FF0000801E04FF000085B
:10DC5000B8F1010F0CD12DB10420A16801F063FBD4
:10DC6000064612E00120A16801F05DFB06460CE0CB
:10DC7000B8F1000F09D125B1042001F043FB06469D
:10DC800003E0012001F03EFB06464EB114B1D4F88A
:10DC9000009001E04FF000094946304601F084F859
:10DCA00016B10DB146F001063046BDE8F087000020
:10DCB000400A00202DE9F84305460F4614464FF070
:10DCC0000008FFF7A6F9002864D1FFF7A5F900289E
:10DCD00060D132480068022803D1FFF797F9002885
:10DCE00058D1002D56D0AF4254D84FF0FF3664B112
:10DCF000A06820B1E068502801D3012606E0A068A2
:10DD000020B9E06810B9002600E00026701C70B34E
:10DD1000012D23D1012E09D10320009000221146AC
:10DD20000120A36801F043FB804605E003220021A7
:10DD3000012001F00DFB8046B8F1000F1DD0E7B1C6
:10DD400000231A461946404601F0ECFB012814D086
:10DD5000404601F03FF84FF000080EE0012E07D1D9
:10DD600039462846A26801F09BFA804605E011E09A
:10DD70003946284601F066FA8046B8F1000F09D00E
:10DD800014B1D4F8009001E04FF000094946404634
:10DD900001F00AF84046BDE8F8830000400A002080
:10DDA0002DE9F04786B0804689461446002004904D
:10DDB000FFF72FF900285DD1FFF72EF9002859D180
:10DDC0002D480068022803D1FFF720F9002851D11F
:10DDD000B8F1000F4ED080261825002005900DF1D7
:10DDE000140A471E44B3206808B1D4F800A0A06903
:10DDF00000B1A5692DB1382D03D8207900F00100BC
:10DE000018B1002006B0BDE8F087606908B160690C
:10DE10008608A06840B1E0685C2805D3206918B185
:10DE2000606908B1012708E0A06830B9E06820B94E
:10DE3000206910B9002700E00027012F0CD12169CB
:10DE4000A0684B463246CDE900510290514640460B
:10DE500001F0F2FD04900DE067B904A8B2B24B46A0
:10DE60005146CDE90050404601F0B4FD012801D0F3
:10DE7000002004900498C5E7400A00202DE9FE4FD9
:10DE80000646894692461C4600200290FFF7C1F8DC
:10DE9000002851D1FFF7C0F800284DD1284800686C
:10DEA000022803D1FFF7B2F8002845D1002E43D055
:10DEB000082000F06DFD0546002D3DD02E60C5F810
:10DEC00004A0B9F1000F01D1002700E001274FF0B5
:10DED000FF384FF0000B94B1206808B1D4F800B0BF
:10DEE000A06828B1E068302802D34FF0010808E0AC
:10DEF000A06830B9E06820B94FF0000801E04FF0A9
:10DF00000008B8F1010F0BD10E49A0682B463A4624
:10DF1000CDE900100121584601F0DDFF02900BE031
:10DF2000B8F1000F08D107482B463A46012100906E
:10DF3000584601F0B5FF02900298BDE8FE8F000040
:10DF4000400A0020C9C500082DE9F04105460E46EB
:10DF50001948076800201949096881F85A001748CC
:10DF60000068001D00F0DAFD681C38B936B11348AE
:10DF70000168091D124800F028FE1AE07C190F48BC
:10DF800000684460BC4207D20C480168091D0D4876
:10DF9000006800F000FE0CE008480168091D0A480E
:10DFA000006800F0F8FD09480068844201D2074883
:10DFB0000460BDE8F0810000040A0020F0090020A0
:10DFC000EC5E0020F8090020F4090020200A00205F
:10DFD00010B5044600F006FE24480068401C2349A2
:10DFE00008602348006840B921480460084600687A
:10DFF00001280DD100F030FA0AE01E48006838B957
:10E000001B480068C06AE16A884201D81848046069
:10E0100019480068401C1849086008460068606498
:10E020001649E06A0968884202D91449E06A086022
:10E03000E16A01EB8101124A02EB8100211D00F02F
:10E04000C4FD00F0F9FD0B48006868B1084800689D
:10E05000C06AE16A884207D24FF0805009490860DF
:10E06000BFF34F8FBFF36F8F10BD0000000A002079
:10E07000F00900200C0A00201C0A0020080A0020D9
:10E080003C5A002004ED00E008B500F0ABFD12485A
:10E090000068E8B9114800F06EFD114800F06BFD12
:10E0A0000E48104908600E480F49086000200F4BC9
:10E0B0000F4A102100900A2001F079F90649086002
:10E0C0000846006820B10BA10348006800F06CFE10
:10E0D00000F0B2FD08BD0000340A0020005F0020FF
:10E0E000145F00202C0A0020300A0020285F002046
:10E0F000785F0020546D72510000000010B516E0EA
:10E1000000F070FD0C48C068C468201D00F006FDDA
:10E110000A480068401E0949086009480068401E16
:10E120000749086000F088FD204600F05EF80448CA
:10E1300000680028E4D110BDD85E0020000A00204D
:10E14000FC09002070B504460D46206C70B1216CAE
:10E15000E0680844E0606168E068884201D32068B4
:10E16000E0602846226CE168F2F760F870BD2DE9A6
:10E17000F04104460F4615464FF00008A66B206C90
:10E1800040B9206860BB606801F06AFD80460020ED
:10E19000606025E07DB93946226CA068F2F746F848
:10E1A000216CA0680844A060D4E90110884217D30C
:10E1B0002068A06014E03946226CE068F2F736F877
:10E1C000216CE068401AE0602168E068884203D270
:10E1D000216C6068401AE060022D01D106B1761E04
:10E1E000701CA0634046BDE8F08110B5044694F869
:10E1F000590030B9206B00F03DFD204600F03AFD9B
:10E200001AE094F85900012803D1204600F032FDAD
:10E2100012E094F85900022801D1012000E000200A
:10E2200050B900BF502080F31188BFF34F8FBFF368
:10E230006F8F00BF00BFFEE710BD00000146084A17
:10E24000126812680AB9012200E000220A600A6816
:10E2500022B9034A1268D268106800E000207047B3
:10E260002C0A002030B54FF48043174800F0070413
:10E270002CB1C01D20F00700134C041B1B1B0246D1
:10E28000124C22600024114D6C60D018083820F028
:10E2900007000F4C206000240D4D2D686C600C4D64
:10E2A0002D682C601146441A4C60094C24680C609F
:10E2B000084D4C682C60084D4C682C604FF00044B1
:10E2C000064D2C6030BD0000D0660020440A0020BE
:10E2D0004C0A0020540A0020500A0020580A00204E
:10E2E00000BFFFF70BFF07480068012807D94FF070
:10E2F000805005490860BFF34F8FBFF36F8F00F068
:10E3000039FCEEE73C5A002004ED00E010B504466D
:10E310004CB1002060602060E06000231A4619467E
:10E32000204601F0FFF810BD2DE9F04106460D46EC
:10E3300017469846069C0DB9246000E02760E66306
:10E3400025640121204601F0A1F884F84C80BDE845
:10E35000F0812DE9F05F82460F4690469B460A9E6B
:10E360000C9C4FEA8801A522206BF1F771FFA8F100
:10E370000100216B01EB800929F0070909F0070072
:10E3800008B9012000E0002050B900BF502080F300
:10E390001188BFF34F8FBFF36F8F00BF00BFFEE741
:10E3A000002507E0795D04F134004155785D00B93E
:10E3B00002E06D1C102DF5D300BF00214320015554
:10E3C000382E00D33726E662E66400202065201D43
:10E3D00000F0DEFB04F1180000F0DAFB2461C6F166
:10E3E0003800A06164620020606584F8580084F8F9
:10E3F0005A005A465146484600F07EFB20600B9872
:10E4000008B10B980460BDE8F09F2DE9F04706467F
:10E410000D4617469846DDE908940DB1012000E04D
:10E42000002050B900BF502080F31188BFF34F8FF8
:10E43000BFF36F8F00BF00BFFEE75CB1FFF724FEA4
:10E440002660A561E761C4F82080C4F82490201DEF
:10E4500000F09EFBBDE8F08710B5002407E004EB58
:10E4600084010F4A02EB810000F085FB641C382C0C
:10E47000F5D30C4800F07FFB0B4800F07CFB0B4809
:10E4800000F079FB0A4800F076FB0A4800F073FBC5
:10E4900004480949086004480849086010BD0000A4
:10E4A0003C5A00209C5E0020B05E0020C45E00202C
:10E4B000D85E0020EC5E0020F4090020F80900205E
:10E4C00010B50146164800E0006803688B42FBD394
:10E4D0000246436813448B4204D143684C6823448A
:10E4E000436001460A464B6813440468A34211D1B5
:10E4F0000C4C03682468A34208D04B680468646825
:10E5000023444B6003681B680B6005E0054B1B68E8
:10E510000B6001E003680B60884200D0016010BD11
:10E52000440A00204C0A00202DE9F04104460D4623
:10E5300016461F464FF0000865602461B5420CD8AE
:10E54000F01BA169884202D34FF0010811E0211DA0
:10E550000948006800F01FFB0BE0BE4204D2BD4238
:10E5600002D34FF0010804E0211D0448006800F0C8
:10E5700012FB4046BDE8F081300A00202C0A002042
:10E5800070B5054600F02EFBA86B08B9012400E029
:10E59000002400F051FB204670BD70B5054600F028
:10E5A00021FBA86BE96B884201D1012400E0002423
:10E5B00000F042FB204670BDF8B505460F461648F0
:10E5C0000068C068C468201D00F0A8FAE06901284E
:10E5D0001DD1A06941192B463A462046FFF7A4FFFA
:10E5E000A8B1002003462A4601460090204601F0CB
:10E5F000E7FC064656B900BF502080F31188BFF3F0
:10E600004F8FBFF36F8F00BF00BFFEE700BF2046F4
:10E61000616A8847F8BD00002C0A0020F0B587B079
:10E6200082E00398002811DA04AE56B900BF5020EA
:10E6300080F31188BFF34F8FBFF36F8F00BF00BF10
:10E64000FEE7D6E90020B168904700BF0398002894
:10E650006ADB059C606908B9012000E0002010B960
:10E66000201D00F05BFA02A800F0C0F805460398F0
:10E670000A2857D2DFE800F009050731334F0608B2
:10E68000323400BF00BF00BF00BF0498A2698118E8
:10E6900003462A462046FFF747FFE8B12046616A55
:10E6A0008847E069012817D1002000900498A169EB
:10E6B000421800231946204601F082FC074657B94C
:10E6C00000BF502080F31188BFF34F8FBFF36F8FCF
:10E6D00000BF00BFFEE700BF25E000BF23E000BF92
:10E6E0000498A061A06908B1012000E0002050B9A1
:10E6F00000BF502080F31188BFF34F8FBFF36F8F9F
:10E7000000BF00BFFEE7A06941192B462A462046FC
:10E71000FFF70AFF07E094F82C0010B9204600F03C
:10E72000A9FA00E000BF00BF002203A90448006866
:10E7300001F048F800287FF474AF07B0F0BD000086
:10E74000340A0020F8B505460C4600F073FC684614
:10E7500000F04CF80646009820BB44B9B54206D8F4
:10E7600001F01CFB31462846FFF726FF1CE03CB1B8
:10E770000E480068006808B9012000E00020044647
:10E78000A91B22460A48006800F056FB01F006FB70
:10E7900050B94FF0805007490860BFF34F8FBFF367
:10E7A0006F8F01E001F0FAFAF8BD0000300A002096
:10E7B000340A002004ED00E00A490968096809B933
:10E7C000012100E0002121B14FF0FF31064A116024
:10E7D00006E004490968C968C868034A41681160CD
:10E7E00070470000F4090020200A002070B504469C
:10E7F00001F08EF9054607480068854204D200F012
:10E800000BF80120206001E0002020600148056035
:10E81000284670BD3C0A00202DE9F84332E0244828
:10E820000068C068056822480068C068C468201D88
:10E8300000F074F92046616A8847E069012821D117
:10E84000A0694619AE4207D966602461211D1848A7
:10E85000006800F0A0F915E0002003462A460146B2
:10E860000090204601F0ACFB074657B900BF50208E
:10E8700080F31188BFF34F8FBFF36F8F00BF00BFCE
:10E88000FEE700BF0A480068006808B9012000E000
:10E8900000200028C3D00648D0F800800548006852
:10E8A000034908600348C0F80080BDE8F883000011
:10E8B0002C0A0020300A00200E480068401C08B9CD
:10E8C000012000E0002050B900BF502080F31188E3
:10E8D000BFF34F8FBFF36F8F00BF00BFFEE700BFD6
:10E8E000502080F31188BFF34F8FBFF36F8F00BFAD
:10E8F00000BFFEE75C0A002008B500BF6846FFF7CE
:10E900009DFC044620460099FFF71CFFFFF786FE9A
:10E91000F4E770B5044600F065F994F9455010E04D
:10E92000606A08B9012000E0002038B904F1240031
:10E9300001F0E8F918B100F0DFFA00E003E0681E2A
:10E9400045B2002DECDC00BFFF2084F8450000F04C
:10E9500073F900F047F994F9445010E0206908B9C0
:10E96000012000E0002048B904F1100001F0CAF9CC
:10E9700008B100F0C1FA681E45B200E001E0002DC8
:10E98000ECDC00BFFF2084F8440000F055F970BDB6
:10E990002DE9F04104464FF0000800F04BFB4648DB
:10E9A000006808B9FFF75EFC444800682040002872
:10E9B0006BD1D4B1083404F00700B0B104F0070003
:10E9C000C0F10800044404F0070008B9012000E089
:10E9D000002050B900BF502080F31188BFF34F8F43
:10E9E000BFF36F8F00BF00BFFEE7002C4DD034484F
:10E9F0000068844249D8334E3046056801E02E460F
:10EA00002D686868A04202D228680028F7D12A48F9
:10EA10000068854239D0306800F108082868306005
:10EA20006868001B102819D92F1907F0070008B9CA
:10EA3000012000E0002050B900BF502080F3118871
:10EA4000BFF34F8FBFF36F8F00BF00BFFEE7686853
:10EA5000001B78606C603846FFF732FD1849686823
:10EA60000968081A164908600846006816490968C6
:10EA7000884203D212480068134908600F49686849
:10EA80000968084368600020286001F087F908F0F1
:10EA9000070008B9012000E0002050B900BF502055
:10EAA00080F31188BFF34F8FBFF36F8F00BF00BF9C
:10EAB000FEE74046BDE8F0814C0A0020580A0020DD
:10EAC000500A0020440A0020540A002070B5044671
:10EAD000254654B900BF502080F31188BFF34F8FF3
:10EAE000BFF36F8F00BF00BFFEE700F07BF82E6A18
:10EAF00000F0A2F8304670BD001F4FF08073036035
:10EB0000001F21F001030360001F034B0360143852
:10EB10000260203870470000B9E8000801460A6921
:10EB2000D1E901309860D1E901035860506888420A
:10EB300001D188685060002008611068401E106094
:10EB400010687047034B0360034B0B608023136016
:10EB5000704700001860002074600020034B0360C1
:10EB6000034B0B604FF48073136070477462002096
:10EB7000D0620020704700F1080141604FF0FF3182
:10EB8000816000F10801C1600161002101607047EE
:10EB900000210161704710B502460B685C1C0CB97E
:10EBA000106907E002F1080000E04068446824684A
:10EBB0009C42FAD944684C604C68A160886041600E
:10EBC0000A611468641C146010BD42684A6093684E
:10EBD0008B60936859609160086103685B1C0360F7
:10EBE0007047000000BF502080F31188BFF34F8FA3
:10EBF000BFF36F8F00BF0E480068401C0C490860CF
:10EC000008460068012812D10A480068C0B208B955
:10EC1000012000E0002050B900BF502080F311888F
:10EC2000BFF34F8FBFF36F8F00BF00BFFEE770478A
:10EC30005C0A002004ED00E00D48006850B900BFF8
:10EC4000502080F31188BFF34F8FBFF36F8F00BF49
:10EC500000BFFEE706480068401E054908600846F8
:10EC6000006820B9002080F3118800BF00BF704702
:10EC70005C0A002070B506463546002E3FD0083DA0
:10EC80002C461F4960680968084008B1012000E06F
:10EC9000002050B900BF502080F31188BFF34F8F80
:10ECA000BFF36F8F00BF00BFFEE7206808B90120E7
:10ECB00000E0002050B900BF502080F31188BFF35E
:10ECC0004F8FBFF36F8F00BF00BFFEE70C49606836
:10ECD0000968084098B1206888B9094960680968DE
:10ECE0008843606000F0A6F9064960680968084436
:10ECF000044908602046FFF7E3FB01F04FF870BDC0
:10ED0000580A0020500A002000204FF0E02108613E
:10ED10008861064800684FF47A71B0FBF1F0401E3C
:10ED20004FF0E0214861072008617047E0090020AA
:10ED300070B5F1F74FFA0446102C16D304F1E02019
:10ED400090F8F05315480078854201DB012000E07F
:10ED5000002050B900BF502080F31188BFF34F8FBF
:10ED6000BFF36F8F00BF00BFFEE70D48006800F4DF
:10ED7000E0600C490968884201D8012000E00020C9
:10ED800050B900BF502080F31188BFF34F8FBFF3FD
:10ED90006F8F00BF00BFFEE770BD0000600A00205B
:10EDA0000CED00E0640A0020024600200BE0084B56
:10EDB00053F8303033B9064B43F8301003EBC0033F
:10EDC0005A6002E0401C0828F1D300BF70470000E1
:10EDD000A80F002070B50446254655B900BF502045
:10EDE00080F31188BFF34F8FBFF36F8F00BF00BF59
:10EDF000FEE7284600F008F895F8460010B92846C6
:10EE0000FFF738FF70BD0000014600200EE0094A00
:10EE100002EBC00252688A4207D10022054B43F838
:10EE2000302003EBC0035A6002E0401C0828EED3F8
:10EE300000BF7047A80F00202DE9F04105460E469F
:10EE400017462C46FFF7CEFE94F94400401C10B93B
:10EE5000002084F8440094F94500401C10B90020BB
:10EE600084F84500FFF7E8FEA06B28B93A46314622
:10EE700004F1240000F062F82046FFF74AFDBDE8E7
:10EE8000F081000070B504460025D4B11248006836
:10EE900008B9012000E0002050B900BF502080F3E5
:10EEA0001188BFF34F8FBFF36F8F00BF00BFFEE726
:10EEB00000F0C0F800212046FFF746F800F06EFF92
:10EEC00005463DB94FF0805004490860BFF34F8FAD
:10EED000BFF36F8F70BD0000280A002004ED00E032
:10EEE00003490968016003490968416070470000EF
:10EEF000180A0020040A0020012001490860704718
:10EF0000140A002070B504460D4654B900BF5020C5
:10EF100080F31188BFF34F8FBFF36F8F00BF00BF27
:10EF2000FEE70548016818312046FFF734FE01214D
:10EF30002846FFF709F870BDF009002070B50546B6
:10EF40000E46144655B900BF502080F31188BFF318
:10EF50004F8FBFF36F8F00BF00BFFEE70648016809
:10EF600018312846FFF731FE0CB14FF0FF3621462D
:10EF70003046FEF7E9FF70BDF009002010B586B0FD
:10EF800000200590049003AA04A905A8FFF7DAFD64
:10EF90000022DDE904101346CDE9002102901EA1F4
:10EFA0001F48039A00F048FD1E49086008460068A3
:10EFB00008B1012400E00024012C02D100F0C4FFBC
:10EFC0000446012C15D100BF502080F31188BFF3F7
:10EFD0004F8FBFF36F8F00BF4FF0FF3012490860B3
:10EFE00001201249086000201149086000F0AEF8C5
:10EFF00010E0601C08B1012000E0002050B900BF03
:10F00000502080F31188BFF34F8FBFF36F8F00BF85
:10F0100000BFFEE706B010BD49444C4500000000AB
:10F02000E1E20008240A0020200A00200C0A002047
:10F03000040A002002480068401C0149086070472B
:10F04000280A00201E48006818B101201D490860E8
:10F0500034E000201B4908601B4801680CE051B9EE
:10F0600000BF502080F31188BFF34F8FBFF36F8F25
:10F0700000BF00BFFEE7491E01EB8100134A52F8B2
:10F08000200008B9012000E000200028E7D101EBB2
:10F0900081020E4B03EB820042685268426000F12D
:10F0A00008024368934202D1426852684260426853
:10F0B000D268074B1A600448016000BF7047000027
:10F0C000280A0020140A0020080A00203C5A0020C8
:10F0D000F009002010B52020FFF75AFC044634B197
:10F0E00000202060201DFFF746FD002020772046ED
:10F0F00010BD38B5054655B900BF502080F31188C2
:10F10000BFF34F8FBFF36F8F00BF00BFFEE720201C
:10F1100000900098202801D1012000E0002050B983
:10F1200000BF502080F31188BFF34F8FBFF36F8F64
:10F1300000BF00BFFEE72C4634B100202060201D38
:10F14000FFF719FD01202077204638BD1CB538494E
:10F15000084600780190FF200A46107008460078A3
:10F1600000909DF8000000F0F0009DF80020904213
:10F1700001D1012000E0002050B900BF502080F3F1
:10F180001188BFF34F8FBFF36F8F00BF00BFFEE743
:10F190009DF8000000F05000264A10700720264A13
:10F1A000106009E024480068401E234A10609DF862
:10F1B00000004006000E00909DF8000000F0800066
:10F1C0008028EFD01C480068C0F10700042801D156
:10F1D000012000E0002050B900BF502080F31188CA
:10F1E000BFF34F8FBFF36F8F00BF00BFFEE7124822
:10F1F00000680002104A10601046008800F4E060C9
:10F2000010600B4A019810700C48006840F47000C0
:10F210000A4908600846006840F070400860FFF73F
:10F2200073FD002006490860F0F79EFF00201CBD1A
:10F2300000E400E0600A0020640A002020ED00E005
:10F240005C0A002070B505460E460DB1012000E0B5
:10F25000002050B900BF502080F31188BFF34F8FBA
:10F26000BFF36F8F00BF00BFFEE7AE4201D80120A1
:10F2700000E0002050B900BF502080F31188BFF398
:10F280004F8FBFF36F8F00BF00BFFEE70222002148
:10F29000284600F05DF8044604B1A663204670BD20
:10F2A000F8B505460E4617460DB1012000E00020D6
:10F2B00050B900BF502080F31188BFF34F8FBFF3C8
:10F2C0006F8F00BF00BFFEE7AE4201D8012000E013
:10F2D000002050B900BF502080F31188BFF34F8F3A
:10F2E000BFF36F8F00BF00BFFEE702203B46002246
:10F2F00011460090284600F05AF8044604B1A6636F
:10F300002046F8BD2DE9F04104460126002722469B
:10F310000021012000F01CF805462846FEF7F6FF04
:10F320002846BDE8F0812DE9F84304460D46012743
:10F330004FF000082B46002211460120009400F0F7
:10F3400036F806463046FEF7E1FF3046BDE8F88362
:10F350002DE9F84305460E4690460DB1012000E028
:10F36000002050B900BF502080F31188BFF34F8FA9
:10F37000BFF36F8F00BF00BFFEE70EB9002701E0AB
:10F3800005FB06F707F15000FFF702FB04465CB1EE
:10F3900004F15009002084F8460043464A463146AD
:10F3A00028460094FEF7C0FF2046BDE8F8832DE90B
:10F3B000F84380460E4617461D46DDF82090B8F10A
:10F3C000000F01D0012000E0002050B900BF502004
:10F3D00080F31188BFF34F8FBFF36F8F00BF00BF63
:10F3E000FEE70DB1012000E0002050B900BF502021
:10F3F00080F31188BFF34F8FBFF36F8F00BF00BF43
:10F40000FEE707B10EB1012000E0002050B900BFB7
:10F41000502080F31188BFF34F8FBFF36F8F00BF71
:10F4200000BFFEE707B90EB9012000E0002050B987
:10F4300000BF502080F31188BFF34F8FBFF36F8F51
:10F4400000BF00BFFEE7502000900098502801D177
:10F45000012000E0002050B900BF502080F3118847
:10F46000BFF34F8FBFF36F8F00BF00BFFEE72C4687
:10F470004CB1012084F846004B463A46314640469E
:10F480000094FEF751FF2046BDE8F88370B50546AD
:10F490000E462C4654B900BF502080F31188BFF3AC
:10F4A0004F8FBFF36F8F00BF00BFFEE7FFF79AFBE0
:10F4B000D4E90F12206801FB020060600020A06305
:10F4C0002068A060E06B401E226C216800FB0210E7
:10F4D000E060FF2084F8440084F845009EB920696C
:10F4E00008B9012000E00020A8B904F1100000F0E4
:10F4F00009FC80B14FF0805009490860BFF34F8F7D
:10F50000BFF36F8F07E004F11000FFF734FB04F145
:10F510002400FFF730FBFFF78FFB012070BD0000D8
:10F5200004ED00E02DE9FF4383B0064688461D4602
:10F530004FF00009344654B900BF502080F31188C1
:10F54000BFF34F8FBFF36F8F00BF00BFFEE7B8F16F
:10F55000000F01D1206C08B9012000E0002050B953
:10F5600000BF502080F31188BFF34F8FBFF36F8F20
:10F5700000BF00BFFEE7022D02D1E06B012801D1E0
:10F58000012000E0002050B900BF502080F3118816
:10F59000BFF34F8FBFF36F8F00BF00BFFEE700F0D8
:10F5A000A7FA08B9059808B9012000E0002050B971
:10F5B00000BF502080F31188BFF34F8FBFF36F8FD0
:10F5C00000BF00BFFEE700BFFFF70CFBA06BE16BC5
:10F5D000884201D3022D28D12A4641462046FEF713
:10F5E000C6FD0746606A08B9012000E0002068B93E
:10F5F00004F1240000F086FB88B14FF080503249BE
:10F600000860BFF34F8FBFF36F8F08E03FB14FF03B
:10F6100080502D490860BFF34F8FBFF36F8FFFF706
:10F620000BFB012007B0BDE8F083059818B9FFF780
:10F6300003FB0020F6E7B9F1000F04D101A8FFF7A2
:10F640004FFC4FF00109FFF7F7FAFFF7F3FCFFF764
:10F65000C9FA94F94400401C10B9002084F8440011
:10F6600094F94500401C10B9002084F84500FFF7CC
:10F67000E3FA05A901A800F059F9F0B92046FEF710
:10F680008CFFA0B104F110000599FFF73BFC204668
:10F69000FFF73FF900F082FB002895D14FF0805032
:10F6A00009490860BFF34F8FBFF36F8F8CE7204687
:10F6B000FFF72FF900F072FB86E72046FFF729F9E4
:10F6C00000F06CFB0020ADE704ED00E02DE9F05FF9
:10F6D00007468A4690461E463C4654B900BF502015
:10F6E00080F31188BFF34F8FBFF36F8F00BF00BF50
:10F6F000FEE7BAF1000F01D1206C08B9012000E04B
:10F70000002050B900BF502080F31188BFF34F8F05
:10F71000BFF36F8F00BF00BFFEE7022E02D1E06B88
:10F72000012801D1012000E0002050B900BF502085
:10F7300080F31188BFF34F8FBFF36F8F00BF00BFFF
:10F74000FEE7FFF7F5FA00BF5021EFF3118081F3D8
:10F750001188BFF34F8FBFF36F8F00BF0546A06BBB
:10F76000E16B884201D3022E23D194F945B0324691
:10F7700051462046FEF7FBFC0BF1010088B9606A98
:10F7800008B9012000E0002080B904F1240000F055
:10F79000B9FA58B1B8F1000F08D00120C8F800003C
:10F7A00004E00BF1010040B284F845004FF001097C
:10F7B00001E04FF0000900BF85F3118800BF484603
:10F7C000BDE8F09F2DE9F74183B005460E464FF0A6
:10F7D00000082C4654B900BF502080F31188BFF3B5
:10F7E0004F8FBFF36F8F00BF00BFFEE70EB9206CD5
:10F7F00008B9012000E0002050B900BF502080F37C
:10F800001188BFF34F8FBFF36F8F00BF00BFFEE7BC
:10F8100000F06EF908B9059808B9012000E0002051
:10F8200050B900BF502080F31188BFF34F8FBFF352
:10F830006F8F00BF00BFFEE700BFFFF7D3F9A76BD4
:10F84000F7B131462046FEF77DFC781EA0632069A3
:10F8500008B9012000E0002060B904F1100000F0B8
:10F8600051FA38B14FF080502F490860BFF34F8FE5
:10F87000BFF36F8FFFF7E0F9012006B0BDE8F0811C
:10F88000059818B9FFF7D8F90020F6E7B8F1000F8E
:10F8900004D101A8FFF724FB4FF00108FFF7CCF9D2
:10F8A000FFF7C8FBFFF79EF994F94400401C10B91C
:10F8B000002084F8440094F94500401C10B9002051
:10F8C00084F84500FFF7B8F905A901A800F02EF863
:10F8D000F0B92046FEF754FEA0B104F124000599CA
:10F8E000FFF710FB2046FFF714F800F057FA002846
:10F8F000A3D14FF080500C490860BFF34F8FBFF386
:10F900006F8F9AE72046FFF704F800F047FA94E774
:10F910002046FEF7FEFF00F041FA2046FEF730FEDB
:10F9200000288AD00020A8E704ED00E070B5064664
:10F930000C4656B900BF502080F31188BFF34F8F9B
:10F94000BFF36F8F00BF00BFFEE754B900BF502068
:10F9500080F31188BFF34F8FBFF36F8F00BF00BFDD
:10F96000FEE7FFF73FF9184802687068131A174856
:10F97000006890F85A0030B100201449096881F8F5
:10F980005A0001251CE02068401C08B9002517E03A
:10F990000F4930680968884204D07068904201D8E5
:10F9A00001250DE02068984207D92068C01A206020
:10F9B0003046FFF795FA002502E00020206001257F
:10F9C000FFF73AF9284670BD040A0020F00900202C
:10F9D000180A00202DE9FF4F85B08046894617465A
:10F9E000DDE912ABB800FEF7D3FF064656B15C2046
:10F9F000FEF7CEFF04460CB1266304E03046FFF765
:10FA000039F900E000248CB1002084F85900CDE9D8
:10FA100000ABCDE902403A4649464046089BFEF716
:10FA200098FC2046FEF7D4FA012501E04FF0FF359F
:10FA3000284609B0BDE8F08F2DE9F04F85B00746A4
:10FA4000884691469A46DDE90EB6109C0EB101201B
:10FA500000E0002050B900BF502080F31188BFF3B0
:10FA60004F8FBFF36F8F00BF00BFFEE70CB10120C7
:10FA700000E0002050B900BF502080F31188BFF390
:10FA80004F8FBFF36F8F00BF00BFFEE75C20039076
:10FA900003985C2801D1012000E0002050B900BF8C
:10FAA000502080F31188BFF34F8FBFF36F8F00BFDB
:10FAB00000BFFEE7B4B1AEB125462C462E6302204E
:10FAC00085F85900002004A953464A46CDE900B103
:10FAD000CDE9025041463846FEF73BFC2846FEF78A
:10FAE00077FA01E000200490049805B0BDE8F08F9B
:10FAF0000549096809B9012005E00449096809B9FF
:10FB0000022000E0002070470C0A0020280A002094
:10FB10000149086870470000040A00202DE9F041FF
:10FB20004FF0000843480068002876D1424800683A
:10FB3000451C4148056015BB40480068006808B98D
:10FB4000012000E0002050B900BF502080F3118850
:10FB5000BFF34F8FBFF36F8F00BF00BFFEE7374883
:10FB600007683748006835490860354807603548F8
:10FB70000068401C33490860FEF71EFE00BF324893
:10FB8000006885423BD300BF2C480068006808B974
:10FB9000012000E0002020B14FF0FF302A4908602A
:10FBA0002CE026480068C068C4686668B54202D286
:10FBB0002548066022E0201DFEF7B0FFA06A18B1BC
:10FBC00004F11800FEF7AAFF2049E06A096888429C
:10FBD00002D91E49E06A0860E16A01EB81011C4A12
:10FBE00002EB8100211DFEF7F0FF1A49E06A096867
:10FBF000C96A8842C8D34FF00108C5E700BF15485D
:10FC00000068C06A00EB8000114951F8200001280B
:10FC100001D94FF0010805E0FFE70F480068401CDC
:10FC20000D4908600D48006808B14FF001084046D2
:10FC3000BDE8F081280A0020040A0020F409002011
:10FC4000F8090020180A0020200A0020080A0020D5
:10FC50003C5A0020F0090020100A0020140A00205D
:10FC600070B505462C460026002D43D0224800687A
:10FC7000844201D1012000E0002050B900BF502093
:10FC800080F31188BFF34F8FBFF36F8F00BF00BFAA
:10FC9000FEE7206D50B900BF502080F31188BFF3FC
:10FCA0004F8FBFF36F8F00BF00BFFEE7206D401E78
:10FCB0002065E16CE06A88421CD0206DD0B9201D1F
:10FCC000FEF72CFFE06CE062E06AC0F13800A06152
:10FCD0000A49E06A0968884202D90849E06A08606E
:10FCE000E16A01EB8101064A02EB8100211DFEF76A
:10FCF0006CFF0126304670BDF0090020080A002084
:10FD00003C5A002070B50646F068C46854B900BF7C
:10FD1000502080F31188BFF34F8FBFF36F8F00BF68
:10FD200000BFFEE704F11800FEF7F8FE1548006872
:10FD3000A0B9201DFEF7F2FE1349E06A0968884267
:10FD400002D91149E06A0860E16A01EB81010F4ABA
:10FD500002EB8100211DFEF738FF04E004F11801D9
:10FD60000B48FEF732FF0B49E06A0968C96A88420E
:10FD700004D9012501200849086000E00025284633
:10FD800070BD0000280A0020080A00203C5A00200C
:10FD9000C45E0020F0090020140A002070B5002481
:10FDA00000263648006850B900BF502080F3118803
:10FDB000BFF34F8FBFF36F8F00BF00BFFEE7FEF7AB
:10FDC00011FF2E480068401E2C4908600846006854
:10FDD00000284ED12A48006800284AD023E029484C
:10FDE000C068C46804F11800FEF798FE201DFEF7F5
:10FDF00095FE2549E06A0968884202D92249E06AED
:10FE00000860E16A01EB8101204A02EB8100211DBB
:10FE1000FEF7DBFE1E49E06A0968C96A884202D320
:10FE200001201C4908601748006808B9012000E05B
:10FE300000200028D3D00CB1FEF7BEFC16480568A0
:10FE400065B100BFFFF76AFE10B1012011490860DB
:10FE50006D1E002DF6D100200F4908600D48006886
:10FE600038B1012630070D490860BFF34F8FBFF34B
:10FE70006F8FFEF7E1FE304670BD0000280A0020BB
:10FE8000000A0020C45E0020080A00203C5A00201E
:10FE9000F0090020140A0020100A002004ED00E000
:10FEA0002DE9FC4705460E4617469846DDF8289092
:10FEB0003020FEF76DFD044654B143463A463146C4
:10FEC0002846CDE90094FEF7A0FA002084F82C0023
:10FED0002046BDE8FC872DE9FC4706460F469046C4
:10FEE0009946DDE90AA5302001900198302801D11A
:10FEF000012000E0002050B900BF502080F311889D
:10FF0000BFF34F8FBFF36F8F00BF00BFFEE755B940
:10FF100000BF502080F31188BFF34F8FBFF36F8F66
:10FF200000BF00BFFEE72C4654B14B46424639465F
:10FF30003046CDE900A4FEF768FA012084F82C00D1
:10FF40002046BDE8FC87000010B586B00024FEF70F
:10FF50009BF816480068D0B100200590049003AAD1
:10FF600004A905A8FEF7FAFD0222DDE9041000232A
:10FF7000CDE9002102900EA10F48039AFFF75CFD26
:10FF80000E4908600846006800B1012400BF54B95A
:10FF900000BF502080F31188BFF34F8FBFF36F8FE6
:10FFA00000BF00BFFEE7204606B010BD340A0020A7
:10FFB000546D722053766300F9E80008380A002077
:10FFC0002DE9FF4704460D4616461F46DDF83080F2
:10FFD0004FF0000954B900BF502080F31188BFF3DF
:10FFE0004F8FBFF36F8F00BF00BFFEE7144800685C
:10FFF00010B3009501960294062D15DAFFF778FDEF
:020000040801F1
:10000000022808D10023424669460D480068FFF7E0
:1000100089FA814610E000231A46694608480068BC
:10002000FFF780FA814607E000233A466946044814
:100030000068FFF74BFB8146484604B0BDE8F087F7
:10004000340A002000C1814001C0804101C08041CC
:1000500000C1814001C0804100C1814000C1814098
:1000600001C0804101C0804100C1814000C1814088
:1000700001C0804100C1814001C0804101C0804178
:1000800000C1814001C0804100C1814000C1814068
:1000900001C0804100C1814001C0804101C0804158
:1000A00000C1814000C1814001C0804101C0804148
:1000B00000C1814001C0804100C1814000C1814038
:1000C00001C0804101C0804100C1814000C1814028
:1000D00001C0804100C1814001C0804101C0804118
:1000E00000C1814000C1814001C0804101C0804108
:1000F00000C1814001C0804100C1814000C18140F8
:1001000001C0804100C1814001C0804101C08041E7
:1001100000C1814001C0804100C1814000C18140D7
:1001200001C0804101C0804100C1814000C18140C7
:1001300001C0804100C1814001C0804101C08041B7
:1001400000C1814000C0C101C30302C2C60607C787
:1001500005C5C404CC0C0DCD0FCFCE0E0ACACB0BF7
:10016000C90908C8D81819D91BDBDA1A1EDEDF1F27
:10017000DD1D1CDC14D4D515D71716D6D21213D317
:1001800011D1D010F03031F133F3F23236F6F737C7
:10019000F53534F43CFCFD3DFF3F3EFEFA3A3BFBB7
:1001A00039F9F83828E8E929EB2B2AEAEE2E2FEF67
:1001B0002DEDEC2CE42425E527E7E62622E2E323D7
:1001C000E12120E0A06061A163A3A26266A6A76707
:1001D000A56564A46CACAD6DAF6F6EAEAA6A6BAB77
:1001E00069A9A86878B8B979BB7B7ABABE7E7FBFA7
:1001F0007DBDBC7CB47475B577B7B67672B2B37397
:10020000B17170B050909151935352929656579746
:10021000559594549C5C5D9D5F9F9E5E5A9A9B5B36
:1002200099595898884849894B8B8A4A4E8E8F4FE6
:100230008D4D4C8C44848545874746868242438356
:100240004181804090100108000000000000000083
:100250000000000000000000000200001800000084
:100260000000000000000000100E01080000000067
:10027000000000000000000000000000000400007A
:100280000800000000000000000000008C0E0108C3
:10029000000000000000000000000000000000005E
:1002A0000004000008000000000000000000000042
:1002B000FC0E01080000000000000000000000002B
:1002C0000000000000040000080000000000000022
:1002D000000000006C0F010800000000000000009A
:1002E0000000000000000000000200000800000004
:1002F0000000000000000000B80F0108000000002E
:1003000000000000000000000000000000020000EB
:10031000080000000000000000000000F80F0108C5
:1003200000000000000000000000000000000000CD
:1003300000020000080000000000000000000000B3
:10034000381001080000000000000000000000005C
:100350000000000000020000080000000000000093
:1003600000000000781001080000000000000000FC
:100370000000000000000000000200000800000073
:1003800000000000000000007C0D010800000000DB
:10039000000000000000000000000000000200005B
:1003A000080000000000000000000000F80D010837
:1003B000000000000000000000000000000000003D
:1003C0000002000008000000000000000000000023
:1003D000740E010800000000000000000000000092
:1003E0000000000000020000020000000000000009
:1003F00000000000940D0108000000000000000053
:10040000000000000000000000000000040E0108D1
:1004100000000000000000000000000000000000DC
:1004200000000000800E0108000000000000000035
:10043000000000000000000000000000F00E0108B5
:1004400000000000000000000000000000000000AC
:1004500000000000600F0108000000000000000024
:10046000000000000000000000000000AC0F0108C8
:10047000000000000000000000000000000000007C
:1004800000000000C00D0108000000000000000096
:10049000000000003C0E0108000000000000000009
:1004A00000000000B80E010800000000000000007D
:1004B00000000000280F01080000000000000000FC
:1004C00000000000880F010800000000000000008C
:1004D00000000000D40F0108000000000000000030
:1004E00000000000141001080000000000000000DF
:1004F000000000005410010800000000000000008F
:10050000000000008410010800000000000000004E
:1005100000000000880D010800000000000000003D
:1005200000000000EC0D01080000000000000000C9
:1005300000000000680E010800000000000000003C
:1005400000000000E40E01080000000000000000B0
:1005500000000000540F010800000000000000002F
:1005600000000000A00F01080000000000000000D3
:1005700000000000EC0F0108000000000000000077
:10058000000000002C100108000000000000000026
:10059000000000006C1001080000000000000000D6
:1005A00000000000D80D010801000000000000005C
:1005B00000000000540E01080100000000000000CF
:1005C00000000000D00E0108010000000000000043
:1005D00000000000400F01080100000000000000C2
:1005E00000000000B00D0108000000000000000045
:1005F000000000002C0E01080000000000000000B8
:1006000000000000A80E010800000000000000002B
:1006100000000000180F01080000000000000000AA
:1006200000000000780F010800000000000000003A
:1006300000000000C40F01080000000000000000DE
:10064000000000000410010800000000000000008D
:10065000000000004410010800000000000000003D
:1006600000000000A00D01080000000000000000D4
:10067000000000001C0E0108000000000000000047
:1006800000000000980E01080000000000000000BB
:1006900000000000080F010800000000000000003A
:1006A00000000000CC0D0108000000000000000068
:1006B00000000000480E01080000000000000000DB
:1006C00000000000C40E010800000000000000004F
:1006D00000000000340F01080000000000000000CE
:1006E00000000000940F010800000000000000005E
:1006F00000000000E00F0108000000000000000002
:1007000000000000201001080000000000000000B0
:100710000000000060100108000000000000000060
:100720000000000000000D05100513051605190551
:100730001C051F052205250528052B052E0531055D
:100740003305360539053C053F0542054505480595
:100750004B054E055105540557055A055D056005C5
:100760006305660569056C056F05720575057805F5
:100770007B057E058105840587058A058D05900525
:10078000930596059A059D05A005A305A605A9054F
:10079000AC05AF05B205B605B905BC05BF05C20578
:1007A000C505C805CC05CF05D205D505D805DB059F
:1007B000DF05E205E505E805EB05EF05F205F505C2
:1007C000F805FB05FF050206050608060C060F06E0
:1007D0001206150618061C061F06220625062906FF
:1007E0002C062F063306360639063C06400643061D
:1007F00046064A064D065006530657065A065E063A
:100800006106640668066B066F0672067606790650
:100810007D068106840688068B068F06930696065B
:100820009A069E06A106A506A906AD06B006B40660
:10083000B806BC06C006C306C706CB06CF06D3065D
:10084000D706DB06DF06E306E806EC06F006F4064C
:10085000F906FD06010706070A070F07140719071F
:100860001D07230728072D07330739073F074507CB
:100870000000000000000000000000000000000078
:100880000000000000000000000000000000000068
:100890000000000000000000000000000000000058
:1008A0000000000000000000000000000000000048
:1008B0000000000000002205250528052B052E0557
:1008C0003105340537053A053D0540054305460524
:1008D00049054C054F055205550558055B055E0554
:1008E0006105640567056A056D0570057305760584
:1008F00079057C057F058205850588058B058E05B4
:100900009205950598059B059E05A105A405A705DB
:10091000AA05AD05B005B405B705BA05BD05C00506
:10092000C305C605CA05CD05D005D305D605D9052D
:10093000DD05E005E305E605E905ED05F005F30550
:10094000F605FA05FD050006030606060A060D066D
:100950001006130617061A061D062106240627068A
:100960002A062E063106340638063B063E064206A7
:10097000450648064C064F065206560659065C06C2
:100980006006630667066A066D06710674067806D9
:100990007B067F06830686068A068D0691069506E7
:1009A00098069C06A006A406A706AB06AF06B306EB
:1009B000B706BB06BF06C206C606CA06CE06D306E3
:1009C000D706DB06DF06E306E706EB06F006F406CD
:1009D000F906FD06010706070B070F07140719079D
:1009E0001D07220727072B07300736073B0741075C
:1009F00048074E07550700000000000000000000F7
:100A000000000000000000000000000000000000E6
:100A100000000000000000000000000000000000D6
:100A200000000000000000000000000000000000C6
:100A300000000000000000000000000000000000B6
:100A40000000000000000C050F0512051505180533
:100A50001B051E0521052405270529052C052F0545
:100A60003205350538053B053E054105440547057A
:100A70004A054D0550055305560559055C055F05AA
:100A80006205650568056B056E05710574057705DA
:100A90007A057D0580058305860589058C05900509
:100AA0009305960599059C059F05A205A505A80532
:100AB000AB05AE05B105B405B805BB05BE05C1055E
:100AC000C405C705CA05CD05D005D405D705DA0587
:100AD000DD05E005E305E605EA05ED05F005F305AE
:100AE000F605FA05FD050006030606060A060D06CC
:100AF0001006130617061A061D06200624062706EA
:100B00002A062E063106340637063B063E06410607
:100B1000450648064B064F065206560659065D0620
:100B20006006640667066B066E0672067506790631
:100B30007C068006840687068B068F06930696063B
:100B40009A069E06A206A606A906AD06B106B50639
:100B5000B906BD06C106C406C806CC06D006D40632
:100B6000D806DD06E106E506E906ED06F206F6061C
:100B7000FB06FF06040708070D07120717071C07E7
:100B8000210726072B07310736073C074107470790
:100B90000000000000000000000000000000000055
:100BA0000000000000000000000000000000000045
:100BB0000000000000000000000000000000000035
:100BC0000000000000000000000000000000000025
:100BD00000000000000018051B051E052105240566
:100BE000260529052C052F053205350538053B0559
:100BF0003E0541054405460549054C054F0552058E
:100C0000550558055B055E056105640567056A05C0
:100C10006D0570057305760579057C057F058205F0
:100C2000850588058B058E059105940597059A0520
:100C30009D05A005A405A705AA05AD05B005B3054A
:100C4000B605B905BC05BF05C305C605C905CC0574
:100C5000CF05D205D605D905DC05DF05E205E5059A
:100C6000E905EC05EF05F205F605F905FC05FF05BC
:100C70000306060609060C061006130616061A06D3
:100C80001D062006240627062A062E0631063406EF
:100C900038063B063F064206450649064C06500606
:100CA000530657065A065E066106650668066C0618
:100CB0006F06730677067A067E0682068506890623
:100CC0008D069006940698069C06A006A306A70625
:100CD000AB06AF06B306B706BB06BF06C306C7061C
:100CE000CB06CF06D306D706DC06E006E406E90607
:100CF000ED06F206F606FB06FF06040709070D07D8
:100D0000120717071C07210726072B07300736078E
:100D10003B074107470700000000000000000000FB
:100D200000000000000000000000000000000000C3
:100D300000000000000000000000000000000000B3
:100D400000000000000000000000000000000000A3
:100D50000000000000000000000000000000000093
:100D60000000000000000000000000000102030479
:100D70000607080900000000010203046D795461B0
:100D8000736B3130000000006D7954696D6572310C
:100D9000300000006D7951756575653031000000D7
:100DA0006D79436F756E74696E6753656D30310090
:100DB0006D7942696E61727953656D303100000062
:100DC0006D7954696D657230310000006D7945763A
:100DD000656E7430310000006D7952656375727311
:100DE0006976654D75746578303100006D794D75A3
:100DF00074657830310000006D795461736B313166
:100E0000000000006D795175657565303200000095
:100E10006D795461736B3032000000006D79436F5F
:100E2000756E74696E6753656D3032006D79426915
:100E30006E61727953656D30320000006D795469CE
:100E40006D657230320000006D794576656E7430E4
:100E5000320000006D795265637572736976654D75
:100E600075746578303200006D794D757465783031
:100E7000320000006D795461736B31320000000064
:100E80006D79517565756530330000006D79546179
:100E9000736B3033000000006D79436F756E7469B9
:100EA0006E6753656D3033006D7942696E6172799A
:100EB00053656D30330000006D7954696D65723093
:100EC000330000006D794576656E743033000000A4
:100ED0006D795265637572736976654D7574657861
:100EE000303300006D794D75746578303300000043
:100EF0006D79517565756530340000006D79546108
:100F0000736B3034000000006D79436F756E746947
:100F10006E6753656D3034006D7942696E61727928
:100F200053656D30340000006D7954696D65723021
:100F3000340000006D794576656E74303400000031
:100F40006D795265637572736976654D75746578F0
:100F5000303400006D794D757465783034000000D0
:100F60006D79517565756530350000006D79546196
:100F7000736B3035000000006D7942696E617279E3
:100F800053656D30350000006D7954696D657230C0
:100F9000350000006D794576656E743035000000CF
:100FA0006D794D7574657830350000006D79517537
:100FB00065756530360000006D795461736B3036AD
:100FC000000000006D7942696E61727953656D3081
:100FD000360000006D7954696D657230360000008E
:100FE0006D794576656E7430360000006D794D750B
:100FF00074657830360000006D795461736B30375A
:10100000000000006D7942696E61727953656D3040
:10101000370000006D7954696D657230370000004B
:101020006D794576656E7430370000006D794D75C9
:1010300074657830370000006D795461736B303817
:10104000000000006D7942696E61727953656D3000
:10105000380000006D7954696D6572303800000009
:101060006D794576656E7430380000006D794D7588
:1010700074657830380000006D795461736B3039D5
:10108000000000006D7954696D6572303900000010
:1010900064656661756C745461736B00BC10010803
:1010A00000000020680A000050050008F412010842
:1010B000680A002068BC00002ED00008520001130E
:1010C00001390510091055090300D005010B003244
:1010D0003DAA55AA550102030405060708090A0B93
:1010E0000C0D0E0F101112131415161718191A1BC8
:1010F0001C1D1E1F202122232425262728292A2BB8
:101100002C000120118877AA990800002039019548
:101110005000010003140006ED9505AAAA00012263
:1011200011FA158134060D0A21032A1A100DAABBE3
:10113000CCDDEEDDCCBB0103000202111A72310AD4
:10114000524114212852E43A24057103003D4032F3
:10115000811020079BCA51040A0F2E175104E21177
:10116000082005610300046201FF010565D200FF4C
:1011700000401F541F681F7C1F901FA41FB81FCC66
:101180001FE01FF41F08201C203020442058206C32
:101190002080209420A820BC20D020E420F8200C1F
:1011A000212021342148215C21702184219821AC07
:1011B00021C021D421E821FC211022242238224CF4
:1011C000226022742288229C22B022C422D822ECDF
:1011D000220023142328233C235023642378238CC8
:1011E00023A023B423C823DC23F023042418242CB5
:1011F000244024542468247C249024A424B824CC9F
:1012000024E024F42408251C253025442558256C89
:101210002580259425A825BC25D025E425F8250C76
:10122000262026342648265C26702684269826AC5E
:1012300026C026D426E826FC261027242738274C4B
:10124000276027742788279C27B027C427D827EC36
:10125000270028142828283C285028642878288C1F
:1012600028A028B428C828DC28F028042918290434
:101270004DFF2C294029542968297C299029A4292B
:10128000B829CC29E029F429082A1C2A302A442A22
:10129000582A6C2A802A942AA82ABC2AD02AE42A0E
:1012A000F82A0C2B202B342B482B5C2B702B842BF7
:1012B000982BAC2BC02BD42BE82BFC2B102C90059F
:1012C00083900DFF20030DFF200305FF900D692083
:1012D00003231004023006980349075802052FCF54
:1012E0004324F4484D57080D6BFA068FAAAAC0098B
:0412F00000000000FA
:0400000508000131BD
:00000001FF
